:100000000C94030D0C94340D0C94340D0C94340D9D
:100010000C94340D0C948B620C94428F0C941F70D2
:100020000C94340D0C94340D0C94340D0C94340D4C
:100030000C94340D0C94340D0C94340D0C94340D3C
:100040000C94340D0C9462820C940E620C94340D5A
:100050000C94340D0C94340D0C94340D0C942D6EC2
:100060000C94340D0C94A94B0C94804B0C94340DCF
:100070000C94340D0C94340D0C94340D0C94340DFC
:100080000C94847E0C94340D0C94340D0C94340D2B
:100090000C94574B0C942E4B0C94340D0C94340D43
:1000A0000C94340D0C94340D0C94340D0C94340DCC
:1000B0000C94340D0C944D600C94340D0C94340D50
:1000C0000C94340D0C94340D0C94340D0C94054B9D
:1000D0000C94DC4A0C94340D0C94B34A0C948A4A68
:1000E0000C94340DFC1D2A1E611E981E731FAA1F3E
:1000F000D81F0620CC20CC20CC20CC20CC20CC205B
:10010000CC20CC20CC20CC20CC20CC20CC20CC208F
:10011000CC20CC20CC20CC20CC20CC20CC20CC207F
:10012000CC20CC20CC20CC20CC20CC20CC20CF1E6E
:10013000071F3E1F34206C20A320CB22D122D722C0
:10014000DD22E322E922EF22F522FB22012307230D
:100150000D231F2325232B23312337233D23432323
:1001600049234F2355235B23612367236D23732387
:1001700079237F238B2397239D23A323A923C123A3
:10018000C723CD23D323D923DF2399249F24A52458
:10019000B124B724BD24C924CF24D524DB24E124F1
:1001A000E724F924FF2429252F2535253B25532530
:1001B00059255F2565257D25832589258F2593254F
:1001C00097259B25A125A525A925AD25B125B525D3
:1001D000B925BF25C525CB25D125D725DD25E32587
:1001E000E925AF23E523EB23F123F723FD230324A4
:1001F000412547254D256B2571257725EF25F525CB
:10020000FB25ED24F32409240F2415241B24212489
:100210002724AB24C324912313231923B523BB2301
:10022000012607260D26852305250B2511251725D3
:100230001D2523252D24332439243F2445244B24F4
:10024000512457245D24632469246F2475247B245E
:10025000812487248D249324972C742C502CB42C27
:100260000B2DD32C022DF12CB92D9C2D782D092E80
:10027000D62DD62DF82DE12D8D338D33A7338D332B
:10028000B433CD33E8330334834786477547794722
:100290007F47BD478A478E47944798479C47A24768
:1002A000A647AA47BD47B047B447B847134D184DB6
:1002B0001D4D274D314DAA4D3B4D434D4B4D554D99
:1002C0005F4D694D784D824DAA4D8C4D964DA04D98
:1002D0007A6083608B609F60B160C360CE60BA73E8
:1002E000EE73237443747874AD74BD74E77531751F
:1002F0003B756F75A475B275E289F989108A278AF2
:100300003E8A558A6C8A838A9B8ABA8AD18AE88A0D
:10031000078B1D8B3400330032004E6F6E65005327
:10032000746F70706564004E65757472616C2054F2
:1003300075726E004D6F76696E67205265766572D4
:100340007365004D6F76696E6720466F72776172D4
:1003500064004272616B696E670054414E4B2052DB
:100360004553544F5245440025004865616C7468FC
:10037000204C6576656C3A200056454849434C450B
:100380002052455041495220434F4D504C45544511
:100390000054414E4B2044455354524F594544005C
:1003A00025004865616C7468204C6576656C3A2060
:1003B00000290056454849434C4520524550414983
:1003C0005220535441525445442028005245504134
:1003D0004952204F5045524154494F4E2043414EBF
:1003E00043454C4C45440029004D414348494E4546
:1003F0002047554E2048495421202800524550415D
:100400004952204F5045524154494F4E2043414E8E
:1004100043454C4C454400290043414E4E4F4E202D
:100420004849542120280054757272657420726FF7
:10043000746174696F6E206973206E6F74206F66CB
:10044000207479706520536572766F2E204E6F2070
:10045000736574757020617661696C61626C652E7C
:10046000004E6F207374656572696E6720736572E4
:10047000766F2061737369676E65642C2072652DD9
:10048000636865636B2076656869636C6520747961
:1004900070652E0054757272657420656C657661A6
:1004A00074696F6E206973206E6F74206F6620749C
:1004B00079706520536572766F2E204E6F207365BC
:1004C00074757020617661696C61626C652E005490
:1004D0006F70204C65667400546F702043656E74B5
:1004E000657200546F70205269676874004D6964CA
:1004F000646C65204C656674004D6964646C6520AD
:1005000043656E746572004D6964646C6520526960
:1005100067687400426F74746F6D204C6566740078
:10052000426F74746F6D2043656E74657200426F24
:1005300074746F6D205269676874004649524D5754
:100540004152452056455253494F4E3A2000694288
:10055000757300534275730050504D004E6F6E65B9
:1005600020446574656374656400417A696D7574CF
:10057000682020202000456C65766174696F6E20CC
:1005800020005475726E2020202020202000546806
:10059000726F74746C6520202000537469636B2043
:1005A0002020202020204D696E2020202043656ED1
:1005B0007465722020204D617820202020446561E0
:1005C0006462616E642020526576657273656400B2
:1005D000524144494F20494E464F202D20004E4F56
:1005E000542044455445435445440049474E4F52D6
:1005F000454400416E616C6F6700446967697461CE
:100600006C00417578204368616E2E2020204D6972
:100610006E20202020204D61782020202020547939
:100620007065004368616E6E656C73207574696CEB
:10063000697A65643A20004368616E6E656C732068
:1006400064657465637465643A20002028446973A6
:1006500061626C656429002028456E61626C656486
:1006600029004D656368616E6963616C2072656322
:100670006F696C00416972736F6674004D656368E1
:10068000616E6963616C2042617272656C3A200030
:1006900020284D31290020284D32290020284229C8
:1006A0000042617272656C20456C65766174696F99
:1006B0006E3A20200020284D30290020284D312975
:1006C00000202841290054757272657420526F749D
:1006D0006174696F6E3A202020004472697665204B
:1006E0004D6F746F72733A202020202020004D4FF0
:1006F000544F522054595045530054616E6B20287A
:1007000054616D69796120444D44290054616E6BD8
:100710002028444B4C4D2047656172626F78290058
:100720004361720048616C66747261636B0054616E
:100730006E6B00554E4B4E4F574E00596573004E31
:100740006F002900252C20446563656C6572617417
:10075000696F6E20666163746F72200020284B6998
:10076000636B6261636B2073706565642000547213
:1007700061636B205265636F696C20456E61626CCA
:1007800065643A202020004E2F4120666F7220764B
:10079000656869636C652074797065005475726E64
:1007A000204D6F64653A202020202020202020202A
:1007B00020202020004E2F4120666F722076656831
:1007C00069636C65207479706500596573202854DD
:1007D000616D69796129002500202D20004E657525
:1007E0007472616C205475726E20416C6C6F776509
:1007F000643A2020200020736563005472616E7398
:100800006D697373696F6E2044656C61793A20205D
:10081000202020002073656300456E67696E6520A7
:1008200050617573652054696D653A202020202041
:100830002000207365630053686966742054696DF5
:10084000653A202020202020202020202020200069
:100850004175746F6D61746963004D616E75616C93
:10086000005472616E736D697373696F6E20547991
:1008700070653A2020202020200025005965732033
:100880002D2000526576657273652053706565642E
:10089000204C696D697465643A2020002500596513
:1008A00073202D2000466F7277617264205370654B
:1008B0006564204C696D697465643A202000206D80
:1008C00073290025207468726F74746C6520666FDC
:1008D0007220002028004D6F746F72204E7564677F
:1008E0006520456E61626C65643A202020200029F5
:1008F000004E6F6E65004E6F6E65002C2050726565
:100900007365743A20002900202841646A75737465
:10091000656420746F200020284C6576656C3A2051
:1009200000446563656C2052616D7020456E6162A4
:100930006C65643A20202020200029004E6F6E65EF
:10094000004E6F6E65002C205072657365743A20FE
:10095000002900202841646A757374656420746FEF
:10096000200020284C6576656C3A20004163636561
:100970006C2052616D7020456E61626C65643A2036
:1009800020202020004163746976652044726976D6
:10099000696E672050726F66696C653A2000566513
:1009A0006869636C6520547970653A2020202020A6
:1009B00020202020202000445249564520534554F1
:1009C00054494E47530020736563005265636F6955
:1009D0006C2064656C61793A202020202020202042
:1009E00020202020202020202020200025005965C4
:1009F00073202D200042617272656C20456C657613
:100A00006174696F6E205370656564204C696D690F
:100A10007465643A20002500596573202D20005428
:100A2000757272657420526F746174696F6E2053B1
:100A300070656564204C696D697465643A202000B6
:100A40005455525245542053455454494E4753002F
:100A5000556E6B6E6F776E004865617679004D65F7
:100A60006469756D004C6967687400437573746FD1
:100A70006D00556E6B6E6F776E004E6F6E65004F3A
:100A800070656E2050616E7A65720054616D69798F
:100A90006120537065630020736563207265636F26
:100AA000766572792900207365632072656C6F61C9
:100AB000642C2000204D4720686974732C2000208E
:100AC00063616E6E6F6E20686974732C200028005D
:100AD00057656967687420436C6173733A202020FE
:100AE00020200044616D6167652050726F66696CFB
:100AF000653A202020005965732028004163636512
:100B00007074204D472044616D6167653A2000593B
:100B1000657320280053656E64204D47204952209C
:100B2000436F64653A2020004E2F4100526570618A
:100B3000697265642062793A202020202020004ECE
:100B40002F41004869742050726F746F636F6C207E
:100B5000323A20202000290020285465616D2000B1
:100B6000466972652050726F746F636F6C3A202013
:100B7000202000466972652050726F746F636F6C3D
:100B80003A2020202000497320526570616972204C
:100B900054616E6B3F202020004952202620546172
:100BA0006E6B20426174746C696E67204469736176
:100BB000626C656400424154544C4520494E464F96
:100BC00000554E4B4E4F574E0042656E6564696E40
:100BD0006920544253204D6963726F004265696514
:100BE000722055534D2D52432D3200546169676573
:100BF0006E20536F756E642043617264004F7065A0
:100C00006E2050616E7A657220536F756E6420435A
:100C10006172640042656E6564696E692054425376
:100C2000204D696E6900536F756E64206361726454
:100C30003A2000534F554E442043415244004869E6
:100C40006C6C205068797369637320456E61626CC7
:100C500065643A202020202020202020004261725C
:100C600072656C2053746162696C697A6174696F32
:100C70006E20456E61626C65643A200053656E7348
:100C80006F722064657465637465643A2020202067
:100C9000202020202020202020205965730053652B
:100CA0006E736F72206E6F74206465746563746513
:100CB000642100494E45525449414C204D45415311
:100CC0005552454D454E5420554E495400556E6B76
:100CD0006E6F776E0042617272656C20456C65764E
:100CE0006174696F6E20436F6D6D616E6400547541
:100CF0007272657420526F746174696F6E20436FF5
:100D00006D6D616E64005374656572696E67204332
:100D10006F6D6D616E640056656869636C65205324
:100D20007065656400456E67696E65205370656522
:100D300064005468726F74746C6520436F6D6D61EC
:100D40006E640053706565642064656372656173E9
:100D500065732062656C6F77200053706565642051
:100D6000696E637265617365732061626F76652079
:100D70000043616E6E6F6E2052656C6F61646564D6
:100D80000056656869636C652044657374726F7999
:100D900065640043616E6E6F6E2048697400427234
:100DA000616B6573204170706C6965640056617297
:100DB0006961626C6500290020286F662000506F11
:100DC000732000417578204368616E6E656C200069
:100DD0005661726961626C65004F6E004F66660015
:100DE0004200410045787465726E616C20496E70F6
:100DF00075742000070809090B0C0C0B0C0C5475BA
:100E00007272657420537469636B202D20004675DF
:100E10006E6374696F6E202300202D3E20002073C6
:100E2000656300547572726574206D6F76656D65CB
:100E30006E742064656C61793A2020004E6F6E6597
:100E40000059657300547572726574207374696318
:100E50006B2066756E6374696F6E733A2000465539
:100E60004E4354494F4E2054524947474552530030
:100E700076206375746F666629002028004C5643FF
:100E800020456E61626C65643A202020202020009D
:100E90007600566F6C746167653A20202020202010
:100EA0002020202000596573004E6F004261747449
:100EB0006572792044657465637465643A20004204
:100EC0004154544552590053657269616C20332076
:100ED000547820426175643A20200041757820538F
:100EE000657269616C20426175643A202020004D72
:100EF0006F746F722053657269616C204261756412
:100F00003A20005553422053657269616C2042615A
:100F100075643A20202000424155442052415445F6
:100F20005300212000464143544F5259205245530B
:100F30004554212000557365722046756E637469AF
:100F40006F6E203100557365722046756E6374694B
:100F50006F6E203200466F72776172642047656160
:100F600072004E65757472616C2047656172005243
:100F700065766572736520476561720053657420FC
:100F8000416363656C2052616D70204C6576656CC1
:100F90003A200053657420446563656C2052616D8E
:100FA00070204C6576656C3A200053657420426170
:100FB0007272656C2053656E7369746976697479B1
:100FC0003A20005365742048696C6C2053656E7339
:100FD000697469766974793A2000416E616C6F6753
:100FE00020557365722046756E6374696F6E20318B
:100FF000202D2000416E616C6F6720557365722053
:1010000046756E6374696F6E2032202D20002D00AE
:10101000202D20002000545255450046414C534598
:1010200000250057616974696E6720666F722072CF
:101030006164696F2E2E2E2000536D6F6B657220D8
:1010400064697361626C65640053657420766F6CCB
:10105000756D653A2000202D205374617274205202
:101060006570656174696E6700202D2053746F7020
:10107000005573657220536F756E64200046697267
:10108000652043616E6E6F6E004669726520526521
:1010900070616972205369676E616C004169727397
:1010A0006F6674202D204D616E75616C20547269DD
:1010B00067676572004D656368616E6963616C2086
:1010C0005265636F696C202D204D616E75616C20D7
:1010D0005472696767657200536572766F20526556
:1010E000636F696C202D204D616E75616C205472A8
:1010F0006967676572004869676820496E74656E44
:101100007369747920466C61736820556E69742028
:101110002D204D616E75616C205472696767657230
:10112000004D47205374617274004D472053746F13
:101130007000417578204F757470757420466C612D
:101140007368656400417578204F757470757420FC
:10115000496E766572736520466C617368656400DC
:1011600053746F7020417578204F757470757420BA
:10117000426C696E6B696E670053746F70205265C4
:10118000766F6C76696E6720417578204C69676868
:10119000740000002100240027002A002D003000E8
:1011A000330001010000040107010A0100002200D0
:1011B000250028002B002E00310034000201000021
:1011C000050108010B010000200023002600290072
:1011D0002C002F003200000100000301060109016C
:1011E00005050505070508080808020202020A0AA3
:1011F00008080404040401010101010101010303C1
:10120000030303030303040707070C0C0C0C0C0C6B
:101210000C0C0202020206060606060606060B0B68
:101220000B0B0B0B0B0B01021020200808102040A9
:10123000102040800201020108040201010204089A
:101240001020408080402010080402018004020128
:101250008040201008040201080402010102040871
:1012600010204080010204081020408000000A0B7A
:1012700002090C0D0E080703040100000000000025
:10128000000000000000000000000000000000005E
:10129000000000000000000012111000000000001B
:1012A000000000000000000000000000000000003E
:1012B0000000556E6B6E6F776E00446574616368F5
:1012C00065642F4E41005265636F696C20536572EF
:1012D000766F0050616E20536572766F00536572B1
:1012E000766F2F455343004F6E626F617264204DDD
:1012F0006F746F7220447269766572004F70656E0C
:101300002050616E7A65722053636F757420536547
:101310007269616C20455343005361626572746F5A
:101320006F74682053657269616C00506F6C6F6CEC
:10133000752053657269616C00536572766F203158
:1013400000536572766F203200536572766F2033DA
:1013500000536572766F203400536572766F2035C6
:1013600000536572766F203600536572766F2037B2
:1013700000536572766F2038005475726E20456E8A
:1013800067696E65204F6E004D616E75616C2074EB
:1013900072616E736D697373696F6E202D20707545
:1013A0007420696E206E65757472616C206765616A
:1013B00072206265666F7265207374617274696E03
:1013C0006720656E67696E6521005475726E2045F1
:1013D0006E67696E65204F666600456E67696E656B
:1013E000204175746F2053687574646F776E004583
:1013F0006E67616765205472616E736D697373699E
:101400006F6E00446973656E676167652054726131
:101410006E736D697373696F6E00536574205475D4
:10142000726E204D6F64653A20310053657420540C
:1014300075726E204D6F64653A20320053657420DA
:101440005475726E204D6F64653A203300456E61AD
:10145000626C65204E65757472616C205475726E95
:10146000730044697361626C65204E6575747261C6
:101470006C205475726E730042617272656C2053F9
:10148000746162696C697A6174696F6E3A2054752F
:10149000726E6564204F4E0042617272656C20531B
:1014A000746162696C697A6174696F6E3A2054750F
:1014B000726E6564204F46460048696C6C20506827
:1014C00079736963733A205475726E6564204F4E68
:1014D0000048696C6C20506879736963733A2054D2
:1014E00075726E6564204F464600494F20506F72FA
:1014F000742041204F7574707574202D204F6E003C
:10150000494F20506F72742041204F75747075746C
:10151000202D204F666600494F20506F7274204284
:10152000204F7574707574202D204F6E00494F2028
:10153000506F72742042204F7574707574202D2086
:101540004F6666004C56432045786974202D20561E
:101550006F6C7461676520526573746F72656400A7
:101560007629004C5643207468726573686F6C640A
:101570002072656163686564212028004C69676892
:10158000742031204F6E0052657665727365643A3F
:101590002020004D61782050756C73653A20004D15
:1015A000696E2050756C73653A2000456E64205654
:1015B000616C75657300456E64205265636F696C7C
:1015C00020536572766F20536574757000456E64A4
:1015D00020526F746174696F6E20536572766F204C
:1015E000536574757000456E6420456C6576617452
:1015F000696F6E20536572766F2053657475700045
:10160000536572766F20756E2D726576657273659F
:101610006400536572766F207265766572736564D7
:101620000052657665727365643A2020004D6178DA
:101630002050756C73653A20004D696E2050756CB2
:1016400073653A200053746172742056616C75653D
:101650007300494E56414C494420534552564F2E33
:10166000204E4F2053455455502E005365747570CD
:10167000205265636F696C20536572766F00536505
:101680007475702054757272657420526F74617431
:10169000696F6E2050616E20536572766F005365DE
:1016A000747570205374656572696E672053657236
:1016B000766F20284F757470757420322900536539
:1016C000747570205374656572696E672053657216
:1016D000766F20284F757470757420342900536517
:1016E0007475702054757272657420456C657661EE
:1016F00074696F6E20536572766F00401F7017D04B
:1017000007A00FA00FDC05D007C409102788139885
:101710003A10276C023A026C023A026C023A026CEE
:1017200002B036384A5C121C255C125C121C255C27
:1017300012BC7FC7F2C07887A5B7C5A00F8813B8C1
:101740000B401FB80BB80B7017401F5374617274B5
:10175000205265766F6C76696E6720417578204CF3
:101760006967687400536F6E790052435441204D8D
:10177000616368696E652047756E00436C61726BCA
:10178000204D616368696E652047756E0052435451
:10179000412052657061697200494255205265705E
:1017A00061697200436C61726B205265706169728D
:1017B000004F70656E50616E7A65720056735461A9
:1017C0006E6B00464F560054616967656E00486550
:1017D0006E67204C6F6E670054616D6979612031CE
:1017E0002F33350054616D69796120322D53686F54
:1017F000740054616D69796100556E6B6E6F776E20
:10180000003A200042697420004761703A20004C81
:10181000696768742031204F6666004C6967687498
:101820002032204F6E004C696768742032204F666A
:101830006600326E64204D472053746F7000326E24
:1018400064204D472053746172740052756E6E6946
:101850006E67204C6967687473204F6E0052756E16
:101860006E696E67204C6967687473204F66660006
:10187000417578204F7574707574204F6E004175F6
:1018800078204F7574707574204F66660053746FBE
:1018900070205265766F6C76696E6720417578208E
:1018A0004C696768740053746F7020417578204FDD
:1018B000757470757420426C696E6B696E67004157
:1018C0007578204F757470757420507265736574E7
:1018D0002044696D00537461727420417578204F03
:1018E000757470757420426C696E6B696E67004127
:1018F0006972736F6674202D20456E61626C656439
:10190000004D656368616E6963616C205265636F49
:10191000696C202D20456E61626C656400416972BE
:10192000736F6674202D2044697361626C65640076
:101930004D656368616E6963616C205265636F69B0
:101940006C202D2044697361626C656400436F6D87
:101950006D73206368616E67656420746F205553F2
:101960004200436F6D6D73206368616E676564202C
:10197000746F2053657269616C203100447269761E
:10198000696E672050726F66696C6520736574209C
:10199000746F202300536D6F6B657220656E6162FA
:1019A0006C656400524144494F204641494C5341C3
:1019B000464500526164696F205265616479202D4B
:1019C00020002900202D2041646A7573746564200D
:1019D000746F2000202853656E736974697669748A
:1019E0007920002900202D2041646A757374656494
:1019F00020746F2000202853656E736974697669BE
:101A0000747920001BA511241FBECFEFD1E2DEBFE9
:101A1000CDBF00E00CBF15E0A0E0B2E0E2ECFAE8D8
:101A200001E00BBF02C007900D92AC3EB107D9F7A1
:101A300023E1ACEEB5E001C01D92AE30B207E1F794
:101A40001DE0C3E0DDE000E006C021970109802F22
:101A5000FE010E9418B0C230D10780E00807A9F744
:101A60000E9444930C94D8B50C9400002F923F929E
:101A70004F925F926F927F928F929F92AF92BF929E
:101A8000CF92DF92EF92FF920F931F93CF93DF934A
:101A9000CDB7DEB7E6970FB6F894DEBF0FBECDBF69
:101AA00080919006909191060E94674A0E94773A31
:101AB0006BE375E080919006909191060E94094930
:101AC0006EEC75E0CE0101960E94CA480091900626
:101AD00010919106D801ED91FC914D815E81698153
:101AE0007A810280F381E02DC8011995C8010E9416
:101AF000674ACE0101960E949A480E948D9180917A
:101B0000900690919106DC01ED91FC910284F385A1
:101B1000E02D199580919006909191060E94674A58
:101B20000E94773A60ED75E0809190069091910661
:101B30000E940949E091DB0AE4300CF0E0E08CE51A
:101B400095E09A83898388E595E09C838B8383E580
:101B500095E09E838D838EE495E098878F83EE0FCA
:101B6000FF0B81E090E08C0F9D1FE80FF91F608153
:101B7000718180919006909191060E947A4A0E940C
:101B8000773A6AE975E080919006909191060E94FB
:101B90007A4A0E94773A6EE875E0809190069091BB
:101BA00091060E940949E0915B11F0915C118181DD
:101BB0009281883E934014F40E94673AE0915B1151
:101BC000F0915C11618172818091900690919106F3
:101BD0000E94657784E00E94DC7EE0915B11F091C9
:101BE0005C116581768180919006909191060E94AA
:101BF000657785E00E94DC7EE0915B11F0915C11DD
:101C00006381748180919006909191060E9465771E
:101C100084E00E94DC7EE0915B11F0915C116781B1
:101C200080919006909191060E944B7788E00E94E7
:101C3000DC7EE0915B11F0915C1180850E94533A4B
:101C400062E875E080919006909191060E940949A2
:101C5000E0916511F091661181819281883E9340F7
:101C600014F40E94673AE0916511F0916611618168
:101C7000728180919006909191060E94657784E030
:101C80000E94DC7EE0916511F0916611658176819C
:101C900080919006909191060E94657785E00E9460
:101CA000DC7EE0916511F091661163817481809111
:101CB0009006909191060E94657784E00E94DC7EF8
:101CC000E0916511F0916611678180919006909185
:101CD00091060E944B7788E00E94DC7EE0916511BE
:101CE000F091661180850E94533A66E775E0809115
:101CF0009006909191060E940949E0916F11F09130
:101D0000701181819281883E934014F40E94673A59
:101D1000E0916F11F0917011618172818091900654
:101D2000909191060E94657784E00E94DC7EE091AC
:101D30006F11F0917011658176818091900690917C
:101D400091060E94657785E00E94DC7EE0916F112C
:101D5000F091701163817481809190069091910649
:101D60000E94657784E00E94DC7EE0916F11F09123
:101D70007011678180919006909191060E944B7737
:101D800088E00E94DC7EE0916F11F09170118085F7
:101D90000E94533A6AE675E0809190069091910610
:101DA0000E940949E0917911F0917A118181928123
:101DB000883E934014F40E94673AE0917911F091C3
:101DC0007A116181728180919006909191060E94B2
:101DD000657784E00E94DC7EE0917911F0917A11C0
:101DE0006581768180919006909191060E94657739
:101DF00085E00E94DC7EE0917911F0917A11638197
:101E0000748180919006909191060E94657784E09C
:101E10000E94DC7EE0917911F0917A1167818091C6
:101E20009006909191060E944B7788E00E94DC7E9C
:101E3000E0917911F0917A1180850E94533A809156
:101E40009006909191060E94674A0E944885C82E8C
:101E500062E076E080919006909191060E947A4A25
:101E60000E94773A0AEF10E1E12CF12CD12C5701B6
:101E70002FEFA21AB20AB5018091900690919106B7
:101E80000E94657749E0E416F10410F48BE001C08C
:101E90008AE00E94DC7ED8012C918091900690917E
:101EA00091062223C9F11596ED91FC911697618157
:101EB00072810E946577D8011596ED91FC91169775
:101EC00081819281883E934014F40E94673A84E0B5
:101ED0000E94DC7ED8011596ED91FC9116976381E6
:101EE000748180919006909191060E94657784E0BC
:101EF0000E94DC7ED8011596ED91FC911697278102
:101F00008091900690919106222319F06AEF75E076
:101F10000BC063EF75E008C0EC14FD041CF46BEE1D
:101F200075E002C06EED75E00E947A4A095F1F4FAE
:101F30007501BCE0AB16B10409F099CF0E94773A65
:101F400067E376E080919006909191060E9409499E
:101F50000E944885682F80919006909191060E947A
:101F6000F67563E276E080919006909191060E946A
:101F700009496091D80A7091D90A80919006909190
:101F800091060E949B770E948D918091900690917E
:101F90009106DC01ED91FC910284F385E02D199509
:101FA00080919006909191060E94674A0E94773A2C
:101FB0006EEE76E080919006909191060E947A4AAA
:101FC0000E94773A6AED76E08091900690919106B2
:101FD0000E9409498091A30F0E945C4FBC0180912F
:101FE0009006909191060E947A4A66EC76E0809184
:101FF0009006909191060E9409498091A40F0E9439
:102000005C4FBC0180919006909191060E94094915
:102010002091A40F80919006909191062B303CF472
:10202000293054F4283069F465EB76E007C02B3092
:1020300041F461EC76E002C06BEB76E00E947A4AF4
:1020400002C00E94674A61EA76E080919006909112
:1020500091060E9409498091A50F0E945C4FBC0126
:1020600080919006909191060E9409492091A50FB8
:1020700080919006909191062B303CF4293054F4D5
:10208000283069F460E976E007C02B3041F46CE950
:1020900076E002C066E976E00E947A4A02C00E94B9
:1020A000674A6CE776E080919006909191060E94D5
:1020B00009492091B70F80919006909191062223B3
:1020C00019F064E776E002C062E676E00E94094912
:1020D00020913D0E8091900690919106222319F057
:1020E00067E576E002C06BE476E00E9409498091E2
:1020F0009006909191060E94674A0E948D9180916E
:10210000900690919106DC01ED91FC910284F3859B
:10211000E02D199580910002823011F40C945B1926
:10212000F090CE0F0091D10F11E080919006909128
:1021300091060E94674A0E94773A67EB79E08091A6
:102140009006909191060E947A4A0E94773A6EE931
:1021500079E080919006909191060E940949E09162
:10216000E40FE6300CF0E0E083E397E09A838983A4
:102170008EE297E09C838B8384E297E09E838D833D
:1021800080E297E098878F838CE097E09A87898731
:102190008AEF96E09C878B87EE0FFF0B81E090E043
:1021A0008C0F9D1FE80FF91F60817181809190064F
:1021B000909191060E947A4A65E879E080919006B4
:1021C000909191060E9409496091000280919006C9
:1021D000909191060E94F6756CE679E080919006E8
:1021E000909191060E9409498F2D0E943E3AFF204E
:1021F00009F44BC062E679E08091900690919106D7
:102200000E9409498091900690919106112339F01E
:102210006091CF0F0E944B779091CF0F06C06091D5
:10222000D50F0E944B779091D50F8091CB129813C8
:102230000C94621966E479E0809190069091910681
:102240000E9409498091900690919106112339F0DE
:102250006091D00F61110CC061E479E006C060911B
:10226000D60F611105C06CE379E00E94094905C0F1
:10227000062E000C770B0E9465776AE379E0809167
:102280009006909191060E94094980919006909144
:1022900091060E94674A61E279E0809190069091F0
:1022A00091060E940949802F0E943E3A002309F4BA
:1022B0004BC067E179E080919006909191060E9471
:1022C00009498091900690919106112339F060910F
:1022D000D20F0E944B779091D20F06C06091D80F19
:1022E0000E944B779091D80F8091CD1298130C9447
:1022F0007C196BEF78E080919006909191060E9496
:1023000009498091900690919106112339F06091CE
:10231000D30F61110CC066EF78E006C06091D90F51
:10232000611105C061EF78E00E94094905C0062EE1
:10233000000C770B0E9465776FEE78E08091900635
:10234000909191060E940949809190069091910682
:102350000E94674A66ED78E0809190069091910620
:102360000E9409498091ED0F811103C00E944C3AEF
:1023700035C06BE377E080919006909191060E94C2
:10238000094963ED78E080919006909191060E9452
:1023900009496091ED0F80919006909191060E94FD
:1023A0004B7763EC78E080919006909191060E94C3
:1023B00009494091EE0F5091EF0F60E070E02AE084
:1023C00080919006909191060E9442496EEB78E0D0
:1023D00080919006909191060E947A4A65EA78E091
:1023E00080919006909191060E9409498091E50F95
:1023F0008436C8F46EE978E0809190069091910659
:102400000E9409496091E50F809190069091910694
:102410000E944B776CE978E080919006909191064C
:102420000E947A4A03C080E00E944C3A63E878E058
:1024300080919006909191060E9409498091E60F43
:102440008436C8F46CE778E080919006909191060C
:102450000E9409496091E60F809190069091910643
:102460000E944B776AE778E0809190069091910600
:102470000E947A4A03C080E00E944C3A61E678E00C
:1024800080919006909191060E94094920918906B9
:102490008091900690919106222319F06AE578E0E8
:1024A00002C060E578E00E947A4A67E378E08091B4
:1024B0009006909191060E9409496091DB0F7091FE
:1024C000DC0F072E000C880B990B0E9438B420E01B
:1024D00030E04AE754E40E9491B0AB01BC0121E036
:1024E00080919006909191060E948A4962E378E07B
:1024F00080919006909191060E947A4A69E178E075
:1025000080919006909191060E9409496091DD0F9B
:102510007091DE0F072E000C880B990B0E9438B4C7
:1025200020E030E04AE754E40E9491B0AB01BC01E6
:1025300021E080919006909191060E948A4964E181
:1025400078E080919006909191060E947A4A6BEF14
:1025500077E080919006909191060E9409496091E0
:10256000DF0F7091E00F072E000C880B990B0E9473
:1025700038B420E030E04AE754E40E9491B0AB0167
:10258000BC0121E080919006909191060E948A49B9
:1025900066EF77E080919006909191060E947A4ACA
:1025A0006DED77E080919006909191060E94094927
:1025B0009091E40F913011F09430F9F48091E10F93
:1025C0000E943E3A8091E10F882329F169ED77E07E
:1025D00080919006909191060E9409496091E20FC6
:1025E00080919006909191060E944B7767ED77E07D
:1025F00080919006909191060CC0209190063091A8
:102600009106953019F46AEC77E002C065EB77E04B
:10261000C9010E94094980919006909191060E94FB
:10262000674A6CE977E080919006909191060E944C
:1026300009499091E40F2FEF290F80919006909116
:102640009106223028F46091EE050E94F67504C0D0
:1026500067E877E00E947A4A6EE677E0809190061C
:10266000909191060E9409498091F10F0E943E3A93
:102670008091F10F882341F16CE577E0809190061D
:10268000909191060E9409496091F20F8091900605
:10269000909191060E944B7764E477E080919006D8
:1026A000909191060E9409496091F30F80919006E4
:1026B000909191060E944B7762E477E080919006BA
:1026C000909191060E9409498091900690919106FF
:1026D0000E94674A0E948D91809190069091910688
:1026E000DC01ED91FC910284F385E02D1995809138
:1026F0009006909191060E94674A0E94773A60E4A2
:102700007AE080919006909191060E947A4A0E9408
:10271000773A6FE17AE080919006909191060E945D
:1027200009498091AC0F8436C8F468E17AE0809161
:102730009006909191060E9409496091AC0F80919A
:102740009006909191060E944B7766E17AE0809125
:102750009006909191060E947A4A03C080E00E9400
:102760004C3A65EF79E080919006909191060E9435
:1027700009498091AB0F8436C8F46EEE79E0809100
:102780009006909191060E9409496091AB0F80914B
:102790009006909191060E944B776CEE79E08091C3
:1027A0009006909191060E947A4A03C080E00E94B0
:1027B0004C3A6BEC79E080919006909191060E94E2
:1027C00009496091B90F7091BA0F1616170614F5E2
:1027D0000091900610919106072E000C880B990B22
:1027E0000E9438B420E030E04AE754E40E9491B0FF
:1027F000AB01BC0122E0C8010E948A49C8010E94C5
:10280000674A66EC79E080919006909191060E946B
:102810007A4A03C080E00E944C3A0E948D918091D8
:10282000900690919106DC01ED91FC910284F38574
:10283000E02D199580919006909191060E94674A2B
:102840000E94773A65EB7BE080919006909191062B
:102850000E947A4A0E94773A209110068091900651
:1028600090919106222309F4C3C166E87BE00E949F
:1028700009490E94BC700E944C3A0E94BC70209191
:10288000900630919106882389F063E77BE0C901C7
:102890000E940949809113060E94DA79BC01809157
:1028A0009006909191060E947A4A4FC060E67BE0C4
:1028B000C9010E940949809110060E94DA79BC0181
:1028C00080919006909191060E940949809111068D
:1028D0008823A9F168E57BE08091900690919106AC
:1028E0000E940949E0911106E4300CF0E0E08AE131
:1028F00093E09A83898388E193E09C838B8386E1CC
:1029000093E09E838D8384E193E098878F83EE0F1D
:10291000FF0B81E090E08C0F9D1FE80FF91F608195
:10292000718180919006909191060E94094966E517
:102930007BE080919006909191060E9409498091D8
:102940009006909191060E94674A63E47BE0809133
:102950009006909191060E9409498091120600917B
:10296000900610919106882321F00E94DA79BC012B
:1029700002C06FE37BE0C8010E947A4A6CE27BE010
:1029800080919006909191060E94094980911306CA
:102990000091900610919106882321F00E94DA7927
:1029A000BC0102C068E27BE0C8010E947A4A65E18E
:1029B0007BE080919006909191060E940949809158
:1029C00015068823E1F06FE07BE0809190069091FE
:1029D00091060E940949809114060E94DA79BC018F
:1029E00080919006909191060E94094966ED75E0EC
:1029F00080919006909191060E946A4A03C080E0FF
:102A00000E944C3A6CEF7AE080919006909191068A
:102A10000E940949809116068823E1F066EF7AE06A
:102A200080919006909191060E9409498091140628
:102A30000E94DA79BC0180919006909191060E94E3
:102A4000094966ED75E080919006909191060E948B
:102A50006A4A03C080E00E944C3A63EE7AE08091BB
:102A60009006909191060E940949E0911706E33083
:102A70000CF0E3E08BE89AE09A8389838FE79AE091
:102A80009C838B838AE79AE09E838D8382E79AE01A
:102A900098878F83EE0FFF0BA1E0B0E0AC0FBD1F56
:102AA000EA0FFB1F608171818091900690919106E1
:102AB0000E947A4A60ED7AE08091900690919106AA
:102AC0000E940949E0910906E4300CF0E4E08BE64D
:102AD0009AE09A83898385E69AE09C838B838EE5CE
:102AE0009AE09E838D8388E59AE098878F8380E5BE
:102AF0009AE09A878987EE0FFF0B81E090E08C0FB8
:102B00009D1FE80FF91F608171818091900690915F
:102B100091060E947A4A6EEC7AE08091900690913C
:102B200091060E94094960910E068091900690914D
:102B300091060E944B776FEB7AE08091900690911E
:102B400091060E94094980910906811110C0609187
:102B50000F0680919006909191060E944B7764EB4E
:102B60007AE080919006909191060E9409496091C7
:102B70000A0670910B06072E000C880B990B0E9419
:102B800038B420E030E04AE754E40E9491B0AB0151
:102B9000BC0121E080919006909191060E948A49A3
:102BA00066EA7AE080919006909191060E94094928
:102BB00060910C0670910D06072E000C880B990B86
:102BC0000E9438B420E030E04AE754E40E9491B01B
:102BD000AB01BC0121E080919006909191060E948A
:102BE0008A4967E97AE0809190069091910602C047
:102BF00069E97BE00E947A4A0E948D91809190065B
:102C000090919106DC01ED91FC910284F385E02D19
:102C1000199580919006909191060E94674A0E94B2
:102C2000773A63E37CE080919006909191060E9450
:102C30007A4A0E94773A66E27CE080919006909111
:102C400091060E940949E091FA0FE5300CF0E5E0A9
:102C500084E19CE09A8389838DEF9BE09C838B8346
:102C60008BEE9BE09E838D838CED9BE098878F831A
:102C700089EC9BE09A87898781EC9BE09C878B8716
:102C8000EE0FFF0B81E090E08C0F9D1FE80FF91F06
:102C90006081718180919006909191060E947A4A9C
:102CA0000E948D918091900690919106DC01ED91AA
:102CB000FC910284F385E02D199580919006909106
:102CC00091060E94674A0E94773A63EB7CE080910C
:102CD0009006909191060E947A4A0E94773A20913C
:102CE000EF0680919006909191062223C9F16CE73E
:102CF0007CE00E94094980919006909191060E9483
:102D0000674A6DE57CE080919006909191060E9463
:102D100009498091F40F0E943E3A8091F40F81118D
:102D20000E94169380919006909191060E94674AA6
:102D30006EE37CE080919006909191060E94094993
:102D40008091F60F0E943E3A8091F60F81110E9409
:102D5000E89280919006909191060E94674A04C083
:102D60006EE97CE00E947A4A0E948D9180919006E3
:102D700090919106DC01ED91FC910284F385E02DA8
:102D8000199580E49CE6A1E0BB278BAB9CABADAB77
:102D9000BEAB80919006909191060E94674A0E9476
:102DA000773A6EE57EE080919006909191060E94C0
:102DB0007A4A0E94773A65E47EE08091900690918D
:102DC00091060E9409492091D60A8091900690911F
:102DD0009106222319F061E47EE002C06CE37EE0FC
:102DE0000E947A4A8091D60A882349F163E27EE004
:102DF00080919006909191060E9409496091F80F88
:102E00007091F90F072E000C880B990B0E9438B4B3
:102E100020E030E04AE754E40E9491B0AB01BC01ED
:102E200022E080919006909191060E948A496EE17D
:102E30007EE080919006909191060E947A4A9DE2F0
:102E4000E92E9FE0F92E29E2222E38E1432E3CEFB5
:102E5000532E4AE0A42EB12C54E6C52ED12CD70116
:102E60002C91222309F4E5C1F701329700811181E9
:102E70000115110509F4DDC180EB9BE6A1E0BB273C
:102E8000820F911DA11DB11DABBFFC0187913324A1
:102E90003394811101C0312C20919006309191061C
:102EA000C8010197849790F56EEF7DE0C9010E94FB
:102EB000094909500C3148F4E02FF0E0EE0FFF1FF4
:102EC000E25EFD4F6081718102C06DEC7CE080911B
:102ED0009006909191060E9409490C3130F4E02F40
:102EE000F0E0EA5AFD4F808101C080E090E08C5014
:102EF000924F092E000CAA0BBB0BABBFFC018791B4
:102F00009EE0981B892F09F036C137C1C80184564D
:102F100091098438934008F03FC064EE7DE0C90118
:102F20000E940949C801B6010E94F1AF61307105E4
:102F300031F06230710559F460EE7DE002C062EE5E
:102F40007DE080919006909191060E9409490E942F
:102F50006F3A80909006909091063320B1F0C801AE
:102F60000E948944811107C06CED7DE0C4010E947C
:102F7000094987E000C1813009F0FFC069ED7DE0BB
:102F8000C4010E94094988E0F6C060ED7DE0C401FB
:102F90000E94094982E0EFC0C801885E93408035F5
:102FA000964408F05AC0C80168EE73E00E94F1AF81
:102FB0004B0163EC7DE0C9010E940949FAE08F16DC
:102FC000910410F40E94673AB401809190069091A8
:102FD00091060E9465770E946F3A6090900670900B
:102FE00091063320A1F1C8010E948944382E6EEB6E
:102FF0007DE0C3010E940949632D80919006909164
:1030000091060E944B7768EB7DE08091900690914D
:1030100091060E940949849CC001859C900D949C56
:10302000900D1124800F911FB5010E9405B07727E4
:1030300080919006909191060E94657766EB7DE005
:1030400080919006909191060E94094996C06DEA80
:103050007DE0C3010E94094946C0C80188539A44D3
:10306000883E934068F509338AE41807D9F058F48C
:1030700008331A4409F081C06EE97DE0C9010E945D
:1030800009498FE078C00A33BAE41B0791F00B338B
:103090001A4409F072C061E77DE0C9010E94094944
:1030A0008EE069C063E97DE0C9010E94094983E1BE
:1030B00062C061E87DE0C9010E9409498CE05BC003
:1030C000C80180529E44883E934078F400526AE5DD
:1030D0007DE0C9010E9409490A3010F40E94673A54
:1030E000802F0E94C23984E046C0C80188509245B2
:1030F000883E934020F4085063E47DE0EACF013F2E
:1031000085E5180719F462E37DE01CC0023F95E5F0
:10311000190739F465E27DE0C9010E94094981E19E
:103120002AC0033FA5E51A0739F467E17DE0C9012C
:103130000E94094980E11FC0043FB5E51B0739F42F
:1031400066E07DE0C9010E9409498DE014C0053F99
:10315000E5E51E0739F46EEE7CE0C9010E940949DD
:1031600086E009C0063F154541F465ED7CE0C901E4
:103170000E94094985E00E94DC7E69E17EE0809141
:103180009006909191060E9409496EE07EE0809140
:103190009006909191060E940949D7016C9170E0C8
:1031A00080919006909191060E946577F701808149
:1031B0008A3020F482E00E94DC7E04C0843610F461
:1031C0000E94673A0E946F3AD7014C91249EA00159
:1031D0001124052E000C660B770B8BA99CA9ADA9B9
:1031E000BEA9480F591F6A1F7B1FDE0111968A0175
:1031F0009B010F5F1F4F2F4F3F4F6BBFFA0187910E
:103200008D93B901A8018111F2CFBE016F5F7F4F8D
:1032100080919006909191060E946A4A8091900652
:1032200090919106DC01ED91FC910284F385E02DF3
:103230001995B3E0EB0EF11CE5EAEE16EFE0FE06A1
:1032400009F00DCE0E948D9180919006909191068B
:10325000DC01ED91FC910284F385E02D19958091BC
:103260009006909191060E94674A0E94773A6FEB10
:103270007EE080919006909191060E947A4A0E9489
:10328000773A6CEA7EE080919006909191060E94D8
:1032900009490E94985420E030E040E050E40E9448
:1032A00032B4209190063091910687FF3FC069EAC1
:1032B0007EE0C90159C0F090D40F0091D70F10E003
:1032C0000C94951063E579E08091900690919106B9
:1032D0000E9409496091CB128091900690919106CD
:1032E0000E944B7761E579E080919006909191067C
:1032F0000E9409490C941A1168E079E080919006C7
:10330000909191060E9409496091CD12809190069A
:10331000909191060E944B7766E079E0809190064B
:10332000909191060E9409490C94791165EA7EE01A
:10333000C9010E947A4A62E97EE0809190069091EC
:1033400091060E9409490E949854AB01BC0122E0F9
:1033500080919006909191060E948A4960E97EE0F2
:1033600080919006909191060E947A4A6DE77EE0E6
:1033700080919006909191060E9409498091421097
:103380000E943E3A209142108091900690919106C1
:10339000222379F06AE77EE00E9409490E94187FA3
:1033A00060E77EE080919006909191060E947A4AB3
:1033B00002C00E94674A0E948D9180919006909170
:1033C0009106DC01ED91FC910284F385E02D1995C5
:1033D00080919006909191060E94674A0E94773AE8
:1033E00067E17FE080919006909191060E947A4A71
:1033F0000E94773A63E07FE0809190069091910679
:103400000E9409494091321050913310609134105C
:103410007091351080919006909191060E9452779C
:103420006FEE7EE080919006909191060E9409498E
:1034300040913A1050913B1060913C1070913D10BA
:1034400080919006909191060E9452776BED7EE0FC
:1034500080919006909191060E9409494091361002
:10346000509137106091381070913910809190060A
:10347000909191060E94527767EC7EE080919006D1
:10348000909191060E94094940913E1050913F1041
:10349000609140107091411080919006909191063A
:1034A0000E9452770E948D91809190069091910692
:1034B000DC01ED91FC910284F385E02D199580915A
:1034C0009006909191060E94674A0E94773AE6968C
:1034D0000FB6F894DEBF0FBECDBFDF91CF911F9125
:1034E0000F91FF90EF90DF90CF90BF90AF909F90A3
:1034F0008F907F906F905F904F903F902F900895A6
:103500002F923F924F925F926F927F928F929F92F3
:10351000AF92BF92CF92DF92EF92FF920F931F93E1
:10352000CF93DF93CDB7DEB7AB970FB6F894DEBF7E
:103530000FBECDBF8CEC91E00E9463B56832734141
:103540008105910519F00E94137B08C040ED51E000
:1035500060E070E08AE89EE00E944BB540E052ECEB
:1035600061E070E08CEC98E00E94C06540913610FC
:103570005091371060913810709139108FE298E0B7
:103580000E94C06540913A1050913B1060913C10F0
:1035900070913D1082E997E00E94C06540913E1015
:1035A00050913F10609140107091411085EF96E06E
:1035B0000E94C0658EE29DE09093F3068093F20630
:1035C0008FEE9AE09093F1068093F0068CEC98E0F1
:1035D0009093F6128093F5121092F7121092330D19
:1035E0001092300D1092320D1092310D11E01093A7
:1035F000E10D0E94458E80915510809393061092A4
:1036000092061092800082E0809381008FE286BB58
:1036100010926F0010928500109284009BE29093AC
:10362000A00099E09093A10089BB109272001092C3
:10363000A5001092A4001092A9001092A800109268
:10364000AB001092AA001092AD001092AC0099EA63
:1036500090932001109321018ABB10927300109265
:103660002501109224011092290110922801109234
:103670002B0110922A0110922D0110922C018091A1
:10368000270F9091280F8093230690932406813072
:1036900071F461E08FE30E94B04C8091240688238E
:1036A00019F00E94C2530FC00E94AC530CC080910D
:1036B0002406882311F062E001C060E08FE30E94DD
:1036C000B04C0E9430558091290F90912A0F809321
:1036D0002A0690932B06813071F461E08EE30E94FC
:1036E000B04C80912B06882319F00E9495530FC08F
:1036F0000E947F530CC080912B06882311F062E05A
:1037000001C060E08EE30E94B04C0E94FF5460E074
:1037100085E40E94B04C62E08CE30E94B04C62E011
:103720008BE30E94B04C62E080E40E94B04C62E007
:1037300081E40E94B04C62E082E40E94B04C62E0FE
:1037400081E20E94B04C62E084E40E94B04C61E0EF
:1037500089E30E94B04C61E08AE30E94B04C0E9471
:10376000C0870E94F78761E085E30E94B04C61E06A
:1037700085E00E94B04C61E070E085E00E94EC4C76
:1037800061E084E00E94B04C61E087E00E94B04CB0
:1037900061E089E20E94814C61E089E20E94B04CC4
:1037A0006A9A60E085E30E94814C60E085E00E94B7
:1037B000814C60E084E00E94814C60E087E00E94E0
:1037C000814C729861E088E00E94B04C80E090E00B
:1037D0009C012657314FF901ED55FF4F40814F367F
:1037E00029F4329720813181232B31F403968837D5
:1037F000910571F760E001C061E088E00E94814CB2
:1038000061E08BE20E94B04C60E08BE20E94814C50
:103810000E94F7870E94DC768091DF0A813009F0F0
:103820006CC08091E20A9091E30AA091E40AB09101
:10383000E50A4091E60A5091E70A6091E80A709122
:10384000E90A841B950BA60BB70B84379E40A10594
:10385000B10500F30E94137B809190069091910630
:103860000E94674A80919006909191060E94674A53
:103870000E94773A65E27FE08091900690919106F0
:103880000E94094901E010E00E94C4870E94F78766
:103890006EEE72E080E090E00E94D24D62E27FE046
:1038A00080919006909191060E9409490E94C087DC
:1038B0000E94F3870530110531F064EF71E080E07C
:1038C00090E00E94D24D0F5F1F4F06301105E1F6C8
:1038D00080919006909191060E94674A0E94773AE3
:1038E00080919006909191060E94674A809190067F
:1038F000909191060E94674A02C081118BCF8091FE
:103900006F00826080936F008091840090918500A9
:103910008056904F90938900809388000E946A2877
:1039200080EF9AE09093A80D8093A70D1091F30F6C
:103930002091F20F8091E10F9091E30F3091E40F0D
:103940003093F4069093EE058093EF0530E0AFEFEF
:10395000B0E00E94C9B524E630E040E050E00E94AB
:103960007BB52093D412612F70E080E090E00E943C
:1039700036B423EC34E64AEA5AE30E9497B42AE9C3
:1039800039E949E55FE30E942DB06093CE12709350
:10399000CF128093D0129093D11210929500109272
:1039A0009400109290008CE08093910084EF90E05E
:1039B000909399008093980011E018BB82E0809367
:1039C0007100809100020E94E08D8091900690919C
:1039D0009106209193064091DD0F5091DE0F509398
:1039E0004212409341122093C90D9093C80D8093C9
:1039F000C70D1092F005109343128091FA0F853095
:103A000040F01092FA0F60E070E080E791E00E94D1
:103A100042761091FA0F123009F444C008F51123D0
:103A200009F466C0113009F05BC08CE090E00E94A0
:103A300032B12AE333E0DC0111963C932E9322E964
:103A400037E01B963C932E931A9790938D068093A4
:103A50008C0610935B0D10935E0D1093610D67C083
:103A6000133009F45EC01430D9F586E090E00E946E
:103A700032B18C012CE933E0DC012D933D93CD0173
:103A800041E060EF7AE00E94E05F86E792E0F801B3
:103A90009183808310938D0600938C0681E0809340
:103AA0005B0D41C086E090E00E9432B128ED32E02B
:103AB000FC013183208390938D0680938C068FB711
:103AC000F8942CED35E030937D1120937C11109209
:103AD00082118FBF81E080935B0D80935E0D25C0C6
:103AE0001092FA0F60E070E080E791E00E94427669
:103AF00086E090E00E9432B18C012CE933E0DC01D9
:103B00002D933D93CD0140E060EF7AE00E94E05FAD
:103B100086E792E0F8019183808310938D060093ED
:103B20008C0610925B0D10925E0D1092610D8091CB
:103B30008C0690918D06DC01ED91FC910190F08155
:103B4000E02D199580914F0D81111FC08091520D6C
:103B500081111BC08091550D811117C08091580DA6
:103B6000811113C080915B0D81110FC080915E0D9A
:103B700081110BC08091610D811107C081E00E940D
:103B8000418E882309F418C310C3A12CB12C612CD9
:103B9000912C1DA2712C812C412C512C06EC15E08E
:103BA000EE24EA94A3E0FA2ECC24CA94DD24D39424
:103BB0008AEB282E85E0382EC5018657914FFC01EF
:103BC000ED55FF4FE081EE2309F4E6C2DC01AF556D
:103BD000BF4F8D919C91892B09F4DEC28E2F90E00E
:103BE000FC01F797EB32F10508F0D6C28827EE58B2
:103BF000FF4F8F4F0C9418B080914F0D882309F41C
:103C0000CBC25110C9C289E190E00E9432B19C013F
:103C1000FC011183008387E090E093838283158207
:103C20001482F782E682D186C086108EC9012AA747
:103C30003BA70E9431832AA53BA5E2E2F4E0D9012B
:103C4000ED93FC933093400D20933F0DC9010E94EA
:103C5000C2667DC18091520D882309F49DC2411036
:103C60009BC289E190E00E9432B19C01DC01119677
:103C70001C930E93E6E0F0E01396FC93EE931297FC
:103C800015961C921E9214971796FC92EE92169718
:103C90001996DC92CE92189758961C922AA73BA7A9
:103CA0000E9431832AA53BA5E2E2F4E0D901ED931D
:103CB000FC933093420D2093410DC9010E94C266CE
:103CC00074C18091550D882309F466C2811064C2C5
:103CD00089E190E00E9432B19C01DC0111961C93B5
:103CE0000E93E5E0F0E01396FC93EE931297159691
:103CF0001C921E9214971796FC92EE9216971996A4
:103D0000DC92CE92189758961C922AA73BA70E9445
:103D100031832AA53BA5E2E2F4E0D901ED93FC93BF
:103D20003093440D2093430DC9010E94C2666BC1BC
:103D30008091580D882309F42FC271102DC289E19A
:103D400090E00E9432B19C01DC0111961C930E930D
:103D5000E4E0F0E01396FC93EE93129715961C9214
:103D60001E9214971796FC92EE9216971996DC9273
:103D7000CE92189758961C922AA73BA70E9431838F
:103D80002AA53BA5E2E2F4E0D901ED93FC93309340
:103D9000460D2093450DC9010E94C26662C1809103
:103DA0005B0D882309F4F8C12DA12111F5C189E12A
:103DB00090E00E9432B19C01DC0111961C930E939D
:103DC000E2E0F0E01396FC93EE93129715961C92A6
:103DD0001E9214971796FC92EE9216971996DC9203
:103DE000CE92189758961C922AA73BA70E9431831F
:103DF0002AA53BA5E2E2F4E0D901ED93FC933093D0
:103E0000480D2093470DC9010E94C26662C180918E
:103E10005E0D882309F4C0C19110BEC189E190E014
:103E20000E9432B19C01DC0111961C930E93E1E0DB
:103E3000F0E01396FC93EE93129715961C921E9247
:103E400014971796FC92EE9216971996DC92CE92E2
:103E5000189758961C922AA73BA70E9431832AA53F
:103E60003BA5E2E2F4E0D901ED93FC9330934A0DD7
:103E70002093490DC9010E94C26662C18091610D03
:103E8000882309F489C1611087C189E190E00E940B
:103E900032B19C01DC0111961C930E9313961C9277
:103EA0001E92129715961C921E9214971796FC92CA
:103EB000EE9216971996DC92CE92189758961C920D
:103EC0002AA73BA70E9431832AA53BA582E294E062
:103ED000F9019183808330934C0D20934B0DC901E0
:103EE0000E94C26657C180914F0D882309F454C1C6
:103EF000511052C18CE190E00E9432B19C01DC0172
:103F000011961C930E93E7E0F0E01396FC93EE936A
:103F1000129715961C921E9214971796FC92EE9289
:103F200016971996DC92CE92189758961C922AA74B
:103F30003BA70E9431832AA53BA5D9012D923C9233
:103F400030934E0D20934D0DC9010E948367552477
:103F5000539422C18091520D882309F41DC1411050
:103F60001BC18CE190E00E9432B19C01FC011183E5
:103F7000008386E090E09383828315821482F78227
:103F8000E682D186C086108EC9012AA73BA70E946F
:103F900031832AA53BA5D9012D923C923093510D36
:103FA0002093500DC9010E94836744244394F4C0B8
:103FB0008091550D882309F4EFC08110EDC08CE18C
:103FC00090E00E9432B19C01FC011183008385E0E6
:103FD00090E09383828315821482F782E682D186F1
:103FE000C086108EC9012AA73BA70E9431832AA54B
:103FF0003BA5D9012D923C923093540D2093530D43
:10400000C9010E94836788248394C6C08091580D9B
:10401000882309F4C1C07110BFC08CE190E00E94F8
:1040200032B19C01FC011183008384E090E0938312
:10403000828315821482F782E682D186C086108E32
:10404000C9012AA73BA70E9431832AA53BA5D90114
:104050002D923C923093570D2093560DC9010E942A
:1040600083677724739498C080915B0D882309F44B
:1040700093C02DA1211190C08CE190E00E9432B13B
:104080009C01DC0111961C930E93E2E0F0E0139684
:10409000FC93EE93129715961C921E921497179606
:1040A000FC92EE9216971996DC92CE92189758963B
:1040B0001C922AA73BA70E9431832AA53BA5D901C0
:1040C0002D923C9230935A0D2093590DC9010E94B4
:1040D000836721E02DA360C080915E0D882309F4E1
:1040E0005BC0911059C08CE190E00E9432B19C01FC
:1040F000DC0111961C930E93E1E0F0E01396FC9323
:10410000EE93129715961C921E9214971796FC9296
:10411000EE9216971996DC92CE92189758961C92AA
:104120002AA73BA70E9431832AA53BA5D9012D923E
:104130003C9230935D0D20935C0DC9010E94836712
:104140009924939429C08091610D882329F16110ED
:1041500023C08CE190E00E9432B19C01FC011183EC
:1041600000831382128215821482F782E682D1863E
:10417000C086108E2AA73BA70E9431832AA53BA5A3
:10418000D9012D923C923093600D20935F0DC901AF
:104190000E94836766246394B3E0AB0EB11CE8E72A
:1041A000AE16B10409F008CDE9CC82E00E94418E40
:1041B000882311F01FA216C081E00E94418E88233F
:1041C00029F082E00E94258E81113FC78CE30E9476
:1041D000594C892B09F02AC78CE30E94594C892B32
:1041E00009F02AC786E0E8E2F0E1DE01549601908A
:1041F0000D928A95E1F7B090211000913110109145
:10420000221070912310609124105091251040913C
:1042100026103091271020912E1080912F10909110
:104220003010A0918C06B0918D06BEA3ADA3E09195
:10423000B80DF091B90DF9A7E8A7909054106090CF
:104240004F10E0904810F0904910809052107090FC
:104250005110C090B90FD090BA0F5090BC0F409041
:10426000B70F3090B80FFFA1FB8BBA8E0B8F1C8F4E
:104270007D8F6E8F5F8F48A339A32AA39CA38BA346
:10428000F2E1AF2EFE017396DE01119601900D92C0
:10429000AA94E1F7E0EFFAE0F093F905E093F8056E
:1042A000AFA1A983B88609871A877B876C875D874A
:1042B0004E873F87288B9A8B898B82E1FE0131964E
:1042C000A9E0B6E001900D928A95E1F730923D0E9B
:1042D00040923E0E5092890ED092820EC092810E74
:1042E0006092BA0D7092860E8092850EF092840EC6
:1042F000E092830E90923C0E88A599A59093880E2B
:104300008093870E8DA19EA19093FB058093FA0563
:1043100087E08093ED091092EE0961E00E94B04CB5
:104320000E94B1761092EF091092F0098091140664
:10433000811102C01092150690911006911105C0CE
:10434000811103C01092C60AA3C081E08093C60AFF
:104350000091C10A1091C20A8091510A60E00E9446
:10436000B04CD801ED91FC910190F081E02DC80195
:10437000199580910906882359F1813071F08330B5
:10438000C1F488E293E290930B0680930A0689E0D9
:1043900080930E0680E197E217C088EB9BE0909334
:1043A0000B0680930A0683E080930E0688E99AE361
:1043B0000BC088E893E190930B0680930A0686E091
:1043C00080930E0680EE9EE290930D0680930C067D
:1043D000809110068823E9F18091140660910E0601
:1043E00070E08823C9F0809116068823A9F080E048
:1043F00090E00E9436B49B01AC0160E070E088EC74
:1044000092E40E9491B06093FC057093FD05809347
:10441000FE059093FF0525C080E090E00E9436B431
:104420009B01AC0160E070E088EC92E40E9491B0E6
:104430006093FC057093FD058093FE059093FF0546
:104440001092F3051092F4051092F5051092F605FE
:104450001FC01092FC051092FD051092FE051092EF
:10446000FF0560910F0670E080E090E00E9436B496
:104470009B01AC0160E070E088EC92E40E9491B096
:104480006093F3057093F4058093F5059093F6051A
:1044900010920606109200061092F705109201067F
:1044A0001092020610920306109204060E94E46A1B
:1044B0006E98769AEE9880916A008F7C80936A005D
:1044C00080913E0E882321F080916A00806203C0B3
:1044D00080916A00806380936A00EE980E94846DE8
:1044E00080E090E040E09C012657314FF901ED5506
:1044F000FF4F5081552331F0329720813181232B9A
:1045000009F04F5F03968837910569F740931D06C0
:10451000ACE2B6E020E030E08CE6282E89E3382ECD
:1045200096EE492E97E3592E4CE0642E48E3742E04
:104530005CEC852E57E3952E69EDA62E67E3B62E2B
:1045400048ED59E304E719E377E7E72E79E3F72E1F
:10455000EBE0CE2EEAE3DE2EC9018657914FFC0137
:10456000ED55FF4F6081662309F45CC38F559F4F63
:10457000FC0180819181892B09F454C370E0FB0117
:104580003197EF38F10508F04DC38827E356FF4F08
:104590008F4F0C9418B087E394E411969C938E93FC
:1045A00041C385E394E411969C938E933BC383E3CC
:1045B00094E411969C938E9335C38CE294E4119607
:1045C0009C938E932FC38AE294E411969C938E93CE
:1045D00029C383EB93E411969C938E9323C385EBBD
:1045E00093E411969C938E931DC387E993E41196EF
:1045F0009C938E9317C384E893E411969C938E93B7
:1046000011C386E793E411969C938E930BC38BE1C1
:1046100093E411969C938E9305C382EF91E41196D7
:104620009C938E93FFC28EE093E411969C938E939D
:10463000F9C280ED92E411969C938E93F3C283E0CD
:1046400093E411969C938E93EDC28CE093E41196C3
:104650009C938E93E7C285E093E411969C938E938E
:10466000E1C283EF92E411969C938E93DBC281EFBB
:1046700092E411969C938E93D5C28FEE92E411969C
:104680009C938E93CFC28FED92E411969C938E9360
:10469000C9C28DED92E411969C938E93C3C28EECA9
:1046A00092E411969C938E93BDC28EEB92E4119688
:1046B0009C938E93B7C28CEB92E411969C938E934D
:1046C000B1C28AEB92E411969C938E93ABC282E8BE
:1046D00091E411969C938E93A5C280E891E4119683
:1046E0009C938E939FC28EE791E411969C938E9338
:1046F00099C288E896E811969C938E9393C288EBB2
:1047000092E411969C938E938DC288EA92E411965E
:104710009C938E9387C28AE892E411969C938E9321
:1047200081C28CE692E411969C938E937BC28AE6BA
:1047300092E411969C938E9375C28BE392E411964A
:104740009C938E936FC28AEB91E411969C938E9307
:1047500069C281EC91E411969C938E9363C287E4C5
:1047600094E411969C938E935DC28CE795E4119628
:104770009C938E9357C28FE695E411969C938E93EB
:1047800051C281E695E411969C938E934BC280E3CF
:1047900095E411969C938E9345C286EF94E411960E
:1047A0009C938E933FC28FE595E411969C938E93D4
:1047B00039C28EE295E411969C938E9333C284EFB6
:1047C00094E411969C938E932DC28DE595E41196F9
:1047D0009C938E9327C28CE295E411969C938E93C2
:1047E00021C282EF94E411969C938E931BC28BE5B9
:1047F00095E411969C938E9315C28AE295E41196E6
:104800009C938E930FC280EF94E411969C938E93A9
:1048100009C289E595E411969C938E9303C288E2C0
:1048200095E411969C938E93FDC18EEE94E41196BF
:104830009C938E93F7C187E595E411969C938E9394
:10484000F1C186E295E411969C938E93EBC18CEEB8
:1048500094E411969C938E93E5C185E595E41196B9
:104860009C938E93DFC184E295E411969C938E9382
:10487000D9C18AEE94E411969C938E93D3C183E5BB
:1048800095E411969C938E93CDC182E295E41196A6
:104890009C938E93C7C188EE94E411969C938E935B
:1048A000C1C181E595E411969C938E93BBC180E2D2
:1048B00095E411969C938E93B5C186EE94E411967F
:1048C0009C938E93AFC18FE495E411969C938E9345
:1048D000A9C18EE195E411969C938E93A3C184EEB9
:1048E00094E411969C938E939DC18FEB99E311965E
:1048F0009C938E9397C189EB99E311969C938E9329
:1049000091C183EB99E311969C938E938BC18CEBB1
:1049100099E311969C938E9385C186EB99E311964A
:104920009C938E937FC180EB99E311969C938E9319
:1049300079C18CEA97E311969C938E9373C18AEAAE
:1049400097E311969C938E936DC188EA97E3119635
:104950009C938E9367C18BE999E311969C938E93F8
:1049600061C188E997E311969C938E935BC186E9B8
:1049700097E311969C938E9355C184E997E3119622
:104980009C938E934FC186E899E311969C938E93E6
:1049900049C181ED98E311969C938E9343C186E8BB
:1049A00098E311969C938E933DC186E394E511960E
:1049B0009C938E9337C182E294E511969C938E93DB
:1049C00031C18EE094E511969C938E932BC182E9C0
:1049D00091E411969C938E9325C182E897E31196FA
:1049E0009C938E931FC180E797E311969C938E93BF
:1049F00019C189EB96E311969C938E9313C18FE6B0
:104A000096E311969C938E930DC181E996E31196DE
:104A10009C938E9307C181E896E311969C938E93A5
:104A200001C183EA96E311969C938E93FBC087E4C1
:104A300096E311969C938E93F5C087E396E31196C7
:104A40009C938E93EFC089E596E311969C938E9389
:104A5000E9C08AE798E311969C938E93E3C08EE6B3
:104A600098E311969C938E93DDC082E698E31196AD
:104A70009C938E93D7C086E598E311969C938E9372
:104A8000D1C08AE498E311969C938E93CBC08EE3B9
:104A900098E311969C938E93C5C082E398E3119698
:104AA0009C938E93BFC087E397E311969C938E935C
:104AB000B9C085E297E311969C938E93B3C083E1CE
:104AC00097E311969C938E93ADC081E097E3119686
:104AD0009C938E93A7C08FEE96E311969C938E9332
:104AE000A1C08DED96E311969C938E939BC08BECA9
:104AF00096E311969C938E9395C083E899E3119663
:104B00009C938E938FC080E899E311969C938E932B
:104B100089C08AE799E311969C938E9383C011967E
:104B2000DC92CE927FC01196FC92EE927BC01196E1
:104B30001C930E9377C08EE699E311969C938E9307
:104B400071C011965C934E936DC01196BC92AE925B
:104B500069C011969C928E9265C011967C926E925D
:104B600061C011965C924E925DC011963C922E925D
:104B700059C0ECEEF3E51196FC93EE9353C089ED2A
:104B800093E511969C938E934DC0E4E0F4E5119665
:104B9000FC93EE9347C089E699E311969C938E931C
:104BA00041C0E6E6F9E31196FC93EE933BC08DE538
:104BB00099E311969C938E9335C0E2E5F9E3119643
:104BC000FC93EE932FC08BE599E311969C938E9303
:104BD00029C0E4E5F9E31196FC93EE9323C083E644
:104BE00097E311969C938E931DC0E6E5F7E311962B
:104BF000FC93EE9317C089E497E311969C938E93F0
:104C000011C0E0E4F9E31196FC93EE930BC08EE241
:104C100099E311969C938E9305C0ECE1F9E311960C
:104C2000FC93EE932D5F3F4F12962837310509F024
:104C300093CC10921E0680912306811114C080E04F
:104C400090E0FC01E55DF04F20813181245631096F
:104C50002436310528F003968837910591F703C073
:104C600081E080931E061092250680912A0681110C
:104C700014C080E090E0FC01E55DF04F20813181BF
:104C8000285C31092436310528F0039688379105D0
:104C900091F703C081E08093250680918C06909166
:104CA0008D06DC01ED91FC91E65BFF4F2091FD0F3D
:104CB0003091FE0F4091FB0F5091FC0F0190F0815D
:104CC000E02D61E0199580918C0690918D06DC01B4
:104CD000ED91FC91E65BFF4F2091011030910210A5
:104CE0004091FF0F509100100190F081E02D62E0A3
:104CF000199580918C0690918D06DC01ED91FC91C7
:104D0000E65BFF4F20910510309106104091031093
:104D1000509104100190F081E02D63E0199580918D
:104D20008C0690918D06DC01ED91FC91E65BFF4FC6
:104D3000209110103091111040910E1050910F10D1
:104D40000190F081E02D64E0199580918C0690919E
:104D50008D06DC01ED91FC91E65BFF4F2091141074
:104D60003091151040911210509113100190F08164
:104D7000E02D65E0199580918C0690918D06DC01FF
:104D8000ED91FC91E65BFF4F2091181030911910C6
:104D900040911610509117100190F081E02D66E0BF
:104DA000199580918C0690918D06DC01ED91FC9116
:104DB000E45BFF4F0190F081E02D4091071061E02E
:104DC000199580918C0690918D06DC01ED91FC91F6
:104DD000E45BFF4F0190F081E02D4091081062E00C
:104DE000199580918C0690918D06DC01ED91FC91D6
:104DF000E45BFF4F0190F081E02D4091091063E0EA
:104E0000199580918C0690918D06DC01ED91FC91B5
:104E1000E45BFF4F0190F081E02D40911A1064E0B7
:104E2000199580918C0690918D06DC01ED91FC9195
:104E3000E45BFF4F0190F081E02D40911B1065E095
:104E4000199580918C0690918D06DC01ED91FC9175
:104E5000E45BFF4F0190F081E02D40911C1066E073
:104E6000199580918C0690918D06DC01ED91FC9155
:104E700000ACF1ADE02D60910B10199580918C067E
:104E800090918D06DC01ED91FC9104ACF5ADE02D27
:104E900060912010199580918C0690918D06DC010F
:104EA000ED91FC9106A4F7A5E02D60910C101995E9
:104EB00080918C0690918D06DC01ED91FC9104A807
:104EC000F5A9E02D60910D10199580E090E09C010E
:104ED0002657314FF901ED55FF4F4081423731F4EC
:104EE000329720813181232B09F0B5C00396883792
:104EF000910569F70E94704580918C0690918D060E
:104F0000DC01ED91FC91E45AFF4F0190F081E02D1E
:104F100040E060911D10199580918C0690918D064E
:104F2000DC01ED91FC91E45AFF4F0190F081E02DFE
:104F300041E060911F10199580918C0690918D062B
:104F4000DC01ED91FC91E45AFF4F0190F081E02DDE
:104F500042E060911E1019958091F40F882331F082
:104F60008091A50F8D3011F01092F40F1092EF0682
:104F70001092CA0D8091F50F8093ED058091F70F87
:104F80008093EC052091461030E0AFEFB0E00E9436
:104F9000C9B524E630E040E050E00E947BB52093A4
:104FA000B5128091451081110E9450880E94D092C4
:104FB0000E94D36D6B017C0110E011110FC0809134
:104FC0009306882359F02CEB37E340ED57E060E07F
:104FD00070E080EF9AE00E94768011E00E94246ADF
:104FE000882351F00E946F870E9402570E94F78722
:104FF0000E94B2690E9489870E94F13B029711F0DA
:105000000E94CA3E0E948D910E94F13B0297A9F630
:105010000E94D36DDC01CB018C199D09AE09BF093B
:105020008C3B9240A105B10540F218C082E00E947D
:10503000418E81110DC0D0C882E00E94258E882348
:1050400009F4D0C883E08FA3CDC8F1E0FFA3CAC89C
:1050500022E02FA3C7C80E9463454ECF0E947D92D5
:105060000E94F7878091DA0A811102C00E94EA77D4
:105070000E94488586E30E94B34DBC01990F880BBE
:10508000990B611571058105910511F00E94BDB361
:1050900022E336E348EE53E060E070E080EF9AE010
:1050A000AB960FB6F894DEBF0FBECDBFDF91CF91A8
:1050B0001F910F91FF90EF90DF90CF90BF90AF9036
:1050C0009F908F907F906F905F904F903F902F9028
:1050D0000C9476808F929F92AF92BF92CF92DF9284
:1050E000EF92FF920F931F93CF93DF9381E0809312
:1050F0004F0D8093520D8093550D8093580D8093E2
:10510000640D8093670D9091E40F9150953040F0BD
:105110008093E40F61E070E08AE591E00E944276BE
:105120009091E40F2DEF290F8091A30F233008F009
:10513000D7C18A3079F03CF4883009F45BC08930FB
:1051400009F488C17EC18B3009F49AC08C3009F40F
:10515000DBC077C183E290E00E9432B1FC0188E0BD
:1051600090E0938382838824839499249A949582EF
:105170008482AA24AA94B12CB782A68211861086B2
:10518000108E93E8D92ED18E22E9E22E27E0F22E5E
:10519000F38EE28E02E514E011830083CAE3D0E1CE
:1051A000D1A3C0A312A2F0938206E0938106CF019F
:1051B0000E94A74E83E290E00E9432B1FC0189E098
:1051C00090E09383828395828482B782A68211863F
:1051D0001086108ED18EF38EE28E11830083D1A3C0
:1051E000C0A312A2F0938006E0937F06CF010E9435
:1051F000A74ED0C280E290E00E9432B1FC0188E06C
:1052000090E093838283AA24A394BB24BA94B582AA
:10521000A482CC24CA94D12CD782C682118610864F
:10522000108E1AE0F12EF18E02E917E0138F028F33
:10523000CAE3D4E0D183C083F0938206E093810671
:10524000CF010E94104E80E290E00E9432B1FC013A
:1052500089E090E093838283B582A482D782C6825C
:1052600011861086108EF18E138F028FD183C0832A
:10527000F0938006E0937F06CF010E94104E8AC211
:1052800089E190E00E9432B1FC0188E090E09383D4
:105290008283EE24E394FF24FA94F582E4820FEFF4
:1052A00010E01783068311861086108ECEE2D4E0BC
:1052B000D183C083F0938206E0938106CF010E94E0
:1052C00026681092640D8091E40F843009F062C268
:1052D00089E190E00E9432B1FC0189E090E0938383
:1052E0008283F582E4821783068311861086108EEE
:1052F000D183C083F0938006E0937F06CF010E94A4
:1053000026681092670D46C2943009F049C089E1C1
:1053100090E00E9432B1EC01E6ECAE2EE5E0BE2E4C
:10532000B982A88287E090E09B838A83CC24C394CF
:10533000DD24DA94DD82CC82EE24EA94F12CFF8223
:10534000EE8219861886188ECE010E94318302E201
:1053500014E019830883D0938206C0938106CE019E
:105360000E94C26610924F0D89E190E00E9432B116
:10537000EC01B982A88286E090E09B838A83DD827B
:10538000CC82FF82EE8219861886188ECE010E948A
:10539000318319830883D0938006C0937F064BC066
:1053A00085E08093E40F89E190E00E9432B1EC0146
:1053B00056ECA52E55E0B52EB982A88287E090E084
:1053C0009B838A83CC24C394DD24DA94DD82CC824F
:1053D000EE24EA94F12CFF82EE8219861886188E4C
:1053E000CE010E94318302E214E019830883D09336
:1053F0008006C0937F06CE010E94C26610924F0DB8
:1054000089E190E00E9432B1EC01B982A88286E085
:1054100090E09B838A83DD82CC82FF82EE821986B4
:105420001886188ECE010E94318319830883D09389
:105430008206C0938106CE010E94C2661092520D70
:10544000A9C189E08093A30F69E070E089E191E050
:105450000E94427680E290E00E9432B1FC0188E036
:1054600090E093838283AA24A394BB24BA94B58248
:10547000A482CC24CA94D12CD782C68211861086ED
:10548000108E40E8F42EF18E02E917E0138F028FA0
:10549000C6E4D4E0D183C083F0938206E093810612
:1054A000CF010E94524E80E290E00E9432B1FC0196
:1054B00089E090E093838283B582A482D782C682FA
:1054C00011861086108EF18E138F028FD183C083C8
:1054D000F0938006E0937F06CF010E94524E5AC19E
:1054E0008A3009F456C03CF4883009F49BC08930F6
:1054F00009F4FBC0F1C08B3009F4B5C08C3009F061
:10550000EBC089E190E00E9432B1EC0176ECA72E6D
:1055100075E0B72EB982A88287E090E09B838A83EA
:10552000CC24C394DD24DA94DD82CC82EE24EA9488
:10553000F12CFF82EE8219861886188ECE010E9409
:10554000318302E214E019830883D0938406C09368
:10555000830689E190E00E9432B1EC01B982A88211
:1055600086E090E09B838A83DD82CC82FF82EE829C
:1055700019861886188ECE010E94318319830883FC
:10558000D0938606C093850610924F0D1092520D4F
:10559000EBC083E290E00E9432B1FC01C091F00FB9
:1055A00088E090E0938382838824839499249A945A
:1055B00095828482AA24AA94B12CB782A6821186ED
:1055C0001086108ED3E8D18F82E9C82E87E0D82EBE
:1055D000D38EC28E92E5E92E94E0F92EF182E0821C
:1055E0000AE310E111A300A3C2A3F0938406E093A1
:1055F000830683E290E00E9432B1FC0189E090E0F2
:105600009383828395828482B782A68211861086D4
:10561000108ED18FD38EC28EF182E08211A300A3AF
:10562000C2A39EC080E290E00E9432B1FC0188E0FB
:1056300090E093838283AA24A394BB24BA94B58276
:10564000A482CC24CA94D12CD782C682118610861B
:10565000108EDAE0FD2EF18E02E917E0138F028F33
:10566000CAE3D4E062C089E190E00E9432B1FC015B
:1056700088E090E093838283EE24E394FF24FA94FD
:10568000F582E4820FEF10E01783068311861086FF
:10569000108ECEE2D4E0D183C083F0938406E093F1
:1056A000830689E190E00E9432B1FC0189E090E03C
:1056B00093838283F582E4821783068311861086A2
:1056C000108ED183C083F0938606E09385061092F6
:1056D000640D1092670D48C089E08093A30F69E0C4
:1056E00070E089E191E00E94427680E290E00E94C1
:1056F00032B1FC0188E090E093838283AA24A394D2
:10570000BB24BA94B582A482CC24CA94D12CD7826B
:10571000C68211861086108E60E8F62EF18E02E9A0
:1057200017E0138F028FC6E4D4E0D183C083F093D7
:105730008406E093830680E290E00E9432B1FC018F
:1057400089E090E093838283B582A482D782C68267
:1057500011861086108EF18E138F028FD183C08335
:10576000F0938606E09385068091850690918606E3
:10577000DC01ED91FC910280F381E02D199580917F
:10578000830690918406DC01ED91FC910280F38107
:10579000E02D19958091E40F833039F0823009F0C3
:1057A0006CC08091A30F8C3051F189E190E00E9490
:1057B00032B1EC0186EC95E09983888386E090E035
:1057C0009B838A8381E09FEF9D838C838FEF90E0A2
:1057D0009F838E8319861886188ECE010E9431838E
:1057E00082E294E099838883D0937D06C0937C06FF
:1057F000CE010E94C2661092520DC6E029C089E116
:1058000090E00E9432B1EC0186EC95E099838883A8
:1058100084E090E09B838A8381E09FEF9D838C836B
:105820008FEF90E09F838E8319861886188ECE01A5
:105830000E94318382E294E099838883D0937D062D
:10584000C0937C06CE010E94C2661092580DC4E03F
:105850006091B20F7091B30F8C2F0E944A826091B9
:10586000B40F7091B50F8C2F0E9446828091B60FB5
:10587000E0917C06F0917D06808FE091A40F8E2F41
:10588000EE0F990BAA0BBB0BFC013897E830F10522
:1058900008F0B8C08827E45DFE4F8F4F0C9418B015
:1058A00083E290E00E9432B1FC0188E090E09383B3
:1058B000828381E09FEF958384838FEF90E09783CD
:1058C000868311861086108E84E8818F82E997E0A6
:1058D000938F828F82E594E0918380838AE390E1C5
:1058E00091A380A312A21EC080E290E00E9432B178
:1058F000FC0188E090E09383828381E09FEF9583B1
:1059000084838FEF90E09783868311861086108EB4
:1059100087E8818F82E997E0938F828F86E494E015
:1059200091838083F0938B06E0938A0699C080E28E
:1059300090E00E9432B1FC0188E090E09383828382
:1059400081E09FEF958384838FEF90E09783868338
:1059500011861086108E8DE0818F82E997E0938FFB
:10596000828F8AE394E0DCCF89E190E00E9432B13B
:10597000FC0188E090E09383828381E09FEF958330
:1059800084838FEF90E09783868311861086108E34
:105990008EE294E091838083F0938B06E0938A06F5
:1059A0001092640D5DC08CE190E00E9432B1EC0178
:1059B00086EC95E09983888385E090E09B838A83D9
:1059C00081E09FEF9D838C838FEF90E09F838E8398
:1059D00019861886188ECE010E9431838AEB95E0D5
:1059E00037C089E190E00E9432B1FC01138212823B
:1059F000158214821782168211861086108E8EEF01
:105A000093E08ECF8CE08093A40F6CE070E08AE18D
:105A100091E00E94427689E190E00E9432B1EC016F
:105A200086EC95E09983888385E090E09B838A8368
:105A300081E09FEF9D838C838FEF90E09F838E8327
:105A400019861886188ECE010E94318382E294E076
:105A500099838883D0938B06C0938A061092550D44
:105A600080918A0690918B06DC01ED91FC91028079
:105A7000F381E02D19958091AC0F843658F485366A
:105A800008F084E664E6681B80918A0690918B0694
:105A90000E94304F8091A40F8C508230A8F4609106
:105AA000AD0F7091AE0F85E00E947C816091AF0FC9
:105AB0007091B00F85E00E9461818091B10FE091FB
:105AC0008A06F0918B06808F2091A50F822F022EDF
:105AD000000C990BAA0BBB0BFC013897E830F105C1
:105AE00008F086C08827EC5CFE4F8F4F0C9418B0EE
:105AF00083E290E00E9432B1FC0189E090E0938360
:105B0000828381E09FEF958384838FEF90E097837A
:105B1000868311861086108E84E8818F82E997E053
:105B2000938F828F82E594E0918380838AE390E172
:105B300091A380A312A257C080E290E00E9432B1EC
:105B4000FC0189E090E09383828381E09FEF95835D
:105B500084838FEF90E09783868311861086108E62
:105B600087E8818F82E997E0938F828F86E494E0C3
:105B700038C080E290E00E9432B1FC0189E090E000
:105B80009383828381E09FEF958384838FEF90E0FE
:105B90009783868311861086108E8DE0818F82E92F
:105BA00097E0938F828F8AE394E01BC08091E40F8B
:105BB000823009F0BAC18091A30F8C3009F0B5C1D1
:105BC0001FC089E190E00E9432B1FC011382128271
:105BD000158214821782168211861086108E8EEF1F
:105BE00093E091838083F0938F06E0938E065EC0EE
:105BF0008091E40F823061F58091A30F8C3041F5E4
:105C00008BE08093A50F6BE070E08BE191E00E9448
:105C1000427689E190E00E9432B1FC0189E090E097
:105C20009383828381E09FEF958384838FEF90E05D
:105C30009783868311861086108E8EE294E091837E
:105C40008083F0938F06E0938E061092670D2EC02E
:105C50008CE08093A50F6CE070E08BE191E00E94F6
:105C6000427689E190E00E9432B1EC0186EC95E049
:105C70009983888384E090E09B838A8381E09FEF0F
:105C80009D838C838FEF90E09F838E831986188687
:105C9000188ECE010E94318382E294E0998388833A
:105CA000D0938F06C0938E061092580D80918E0669
:105CB00090918F06DC01ED91FC910280F381E02D43
:105CC00019958091AB0F843658F4853608F084E638
:105CD00064E6681B80918E0690918F060E94304F7B
:105CE0008091A50F8C50823000F56091A60F7091C5
:105CF000A70F84E00E947C816091A80F7091A90F8A
:105D000084E00E9461818091AA0FE0918E06F0915B
:105D10008F06808F8091A50F8D3039F48091AA0F66
:105D2000E091D10DF091D20D808F8EE190E00E9434
:105D300032B1EC01F090BB0FC090BF0FD090C00FFC
:105D4000A090BD0FB090BE0F86EC95E0998388833C
:105D500083E090E09B838A8381E09FEF9D838C8327
:105D60000FEF10E01F830E8319861886188ECE0160
:105D70000E94318386E194E099838883BA8EA98E4C
:105D8000DC8ECB8EFD8ED093B90DC093B80D609193
:105D9000C10F7091C20F83E00E947C816091C30F9C
:105DA0007091C40F83E00E9461818091BB0FE091EC
:105DB000B80DF091B90D808F8091BB0F0E940D76C8
:105DC0008091B80D9091B90DDC01ED91FC910280AC
:105DD000F381E02D19958091C50F882339F185E273
:105DE00090E00E9432B1FC018091CA0F9091CB0FDC
:105DF0002091C80F3091C90F4091C60F5091C70F25
:105E000068E070E0738362831582148217830683CF
:105E100011861086108E6AE074E071836083528F61
:105E2000418F348F238F968F858F22C085E290E03B
:105E30000E9432B1FC018091C80F9091C90F20914E
:105E4000C60F3091C70F48E050E05383428315825C
:105E500014821783068311861086108E4AE054E060
:105E600051834083328F218F948F838F168F058FBC
:105E7000F0930806E09307068091070690910806C4
:105E80000E9404688091640D8823F9F089E190E014
:105E90000E9432B1FC0188E090E0938382831582F6
:105EA00014828FEF93E0978386838FEF91E0918741
:105EB0008087108E8EE294E091838083F093630D4F
:105EC000E093620DCF010E9426688091670D8823C0
:105ED00009F473C089E190E00E9432B1FC0189E0CD
:105EE00090E093838283158214828FEF93E09783EF
:105EF00086838FEF91E091878087108E8EE294E009
:105F000091838083F093660DE093650DCF01DF915F
:105F1000CF911F910F91FF90EF90DF90CF90BF90A6
:105F2000AF909F908F900C9426682C3009F499CEF6
:105F30008CE190E00E9432B1EC0186EC882E85E085
:105F4000982E9982888294E0A92EB12CBB82AA82D5
:105F5000CC24C394DD24DA94DD82CC82EE24EA944E
:105F6000F12CFF82EE8219861886188ECE010E94CF
:105F700031830AEB15E019830883D0938F06C09311
:105F80008E068CE190E00E9432B1EC019982888209
:105F9000BB82AA82DD82CC82FF82EE8219861886BD
:105FA000188E0E94318319830883D093D20DC09339
:105FB000D10DCE010E94836777CEDF91CF911F91E3
:105FC0000F91FF90EF90DF90CF90BF90AF909F9098
:105FD0008F9008952F923F924F925F926F927F928F
:105FE0008F929F92AF92BF92CF92DF92EF92FF92E9
:105FF0000F931F93CF93DF93CDB7DEB7C65AD10966
:106000000FB6F894DEBF0FBECDBFCDB6DEB6CC5511
:10601000DF4F1882C45AD040CD55DF4F1882C35A83
:10602000D0408091340D8A3709F447C0C0F48737D7
:1060300009F4D9C238F48F3109F430C5863709F430
:10604000E2C1F1C5883709F4DDC2893709F0EBC533
:106050000E9431850E94D36D2B013C0129C08E37EF
:1060600009F42EC338F48B3709F4CAC18C3709F40C
:10607000D8C2D9C5813809F402C5823809F4EDC403
:10608000803809F0D0C565C40E94D36DDC01CB0116
:1060900084199509A609B70980329340A105B10575
:1060A00008F007C50E94CA3E0E9431850E942E90CA
:1060B0000E94F13B029741F7FCC40E94F13B02971A
:1060C00029F060E084E80E94EE908BC18091DB0AA9
:1060D000823031F0833039F482E08093720D03C056
:1060E00081E08093921281E080933E0D8E010C55E9
:1060F0001F4F2BE0AE0144575F4F68E871E90E94E3
:106100006B900E944885893058F0015011092BE0AE
:10611000AE014F575F4F68E872E981E00E946B90D3
:1061200010923D0D772473940E94DA3B882309F482
:106130003DC1198222961FAE229780913D0D81119B
:106140000EC0BE0164577F4FCE018F5B9F4F0E94F0
:1061500050B3CC55DF4F0881C45AD0400FC0709265
:106160003D0DBE016F577F4FCE018F5B9F4F0E9449
:1061700050B3CD55DF4F0881C35AD04010913D0D2B
:10618000ADB6BEB68091D70AEDB7FEB722E0829FCA
:10619000E019F10911240FB6F894FEBF0FBEEDBF50
:1061A0008DB79EB701967C0166EE75E0CE018356F1
:1061B0009F4F0E94CA488091DB0A823089F0833069
:1061C00061F1813009F0A1C04091D70A50E0B701D8
:1061D00080916B1290916C120E94238F10E039C055
:1061E0002091D70A30E05FB7F89440E0842F90E028
:1061F0008217930774F4880F991FF701E80FF91FAE
:10620000DC01AF58BD4E8D919C91918380834F5F8F
:10621000EDCF5FBF109291121CC02091D70A30E0E1
:106220005FB7F89440E0842F90E08217930774F4EE
:10623000880F991FF701E80FF91FDC01A557B24F2E
:106240008D919C91918380834F5FEDCF5FBF1092C2
:10625000AD0D6DE270E0CE0183569F4F0E94F9476D
:106260002091D70A293048F0112321F0113021F470
:1062700018E004C028E001C020E010E0121758F533
:10628000F701E10FF11DE10FF11D608171814AE01D
:10629000CE0189569F4FCB55DF4F2883C55AD0403A
:1062A0000E949F48BE0169567F4FCE0183569F4F83
:1062B0000E942048CE0189569F4F0E949A48CE01E5
:1062C00083569F4F0E94F8881F5FCB55DF4F288170
:1062D000C55AD040D3CF40E450E0BE016F5F7F4F3E
:1062E000CE0183569F4F0E94EF88CF55DF4F188114
:1062F000C15AD040CE0183569F4F0E949A480FB694
:10630000F894BEBE0FBEADBE0BC0CE0183569F4FEC
:106310000E949A480FB6F894BEBE0FBEADBE10E004
:10632000BE016F5F7F4FCE018F5B9F4F0E9450B3C6
:10633000010F10E0E1E4F0E0EC0FFD1FE00FF11FB2
:106340001082BE016F5B7F4F8091F5129091F61223
:106350000E942D49B801CE018F5B9F4F0E944B9048
:10636000BC018091F5129091F6120E9465776AE067
:106370008091F5129091F6120E9402498091F512D7
:106380009091F612DC01ED91FC910284F385E02DF1
:1063900019950E944885893048F080913D0D811102
:1063A00003C070923D0D02C010923D0D0E943185D8
:1063B0000E942E900E94B06881110CDE8091330DF6
:1063C00081110FC080913E0D882359F08091F71202
:1063D000811107C08091310D9091320D0A970CF414
:1063E000A3CE8091DB0A823039F0833009F01BC4E0
:1063F00081E08093720D17C481E08093921213C4E0
:1064000010923E0D48C31091370D8FEF810F8530EC
:1064100028F060E089E80E94EE9005C4133079F01E
:1064200018F41230F9F004C0143079F0153099F0F6
:1064300040E6442E49E0542E612C712C19C0412CA9
:106440003BE4532E612C712C13C0412C26E9522EB3
:10645000612C712C0DC0412C92EC592E6624639452
:10646000712C06C080E8482E85E2582E612C712CD4
:1064700000E0E12EF12C5701BFE8AB0EB11C150175
:10648000E89427F83324E6E9EE0EF11CE894E7F8E7
:10649000FF24023091F018F4013051F004C00330B1
:1064A00089F00430A1F040E659E060E070E013C0EC
:1064B00040E855E260E070E00EC040E05BE460E080
:1064C00070E009C040E056E960E070E004C040E0E0
:1064D00052EC61E070E082E997E00E94C06582E9D9
:1064E00097E00E941E470E94D36D4B015C01F2E3CE
:1064F0008F0E911CA11CB11C0E94EE8F0E94D36DC7
:10650000681579058A059B05B8F360E870E082E9B3
:1065100097E00E94A36A6FE070E082E997E00E9432
:10652000A36A612F82E997E00E94D846B10182E90F
:1065300097E00E94A36A0E94D36D4B015C012AE0A0
:10654000820E911CA11CB11C0E94EE8F0E94D36D83
:10655000681579058A059B05B8F367E870E082E95C
:1065600097E00E94A36A6FE070E082E997E00E94E2
:10657000A36A612F82E997E00E94D846B70182E9B9
:1065800097E00E94A36A82E997E00E941E470E945A
:10659000D36D4B015C013EE5830E31E0931EA11CDF
:1065A000B11C0E94EE8F0E94D36D681579058A0593
:1065B0009B05B8F30F5F053009F06BCFB301A20163
:1065C00082E997E00E94C06540923A1050923B10D9
:1065D00060923C1070923D10B301A20180EB91E0FB
:1065E0000E942B8958C283E090E00E9432B12AE0D9
:1065F000DC012C9322E937E012963C932E931197FD
:106600006AE00CC083E090E00E9432B12DE0FC0112
:10661000208322E937E0328321836DE00E94F44039
:106620003AC24091370D5091380D0091390D1091BB
:106630003A0D6091350D7091360DCE010196CB5516
:10664000DF4F4883C55AD040CA55DF4F5883C65ADA
:10665000D0400E94927DCB55DF4F4881C55AD04033
:10666000CA55DF4F5881C65AD040892BE9F08D8139
:10667000873050F4853080F48130B0F0642F8B8106
:106680009C810E94D0770DC0893070F4B8018B8155
:106690009C810E942B8905C0BA018B819C810E943C
:1066A00042760E94699104C061E085E80E94EE9004
:1066B0008091300D8111B7C281E08093300DB3C25B
:1066C000B090350DE090360DC956DF4F1882C7598E
:1066D000D04066EE75E0CE018F579F4F0E94CA48AA
:1066E0006B2D7E2DCE0184579F4F0E94927D892B6A
:1066F00009F4C9C0C057DF4FE881C059D0404E2FC0
:1067000050E0FA013197E830F10508F0BCC0882765
:10671000E45CFE4F8F4F0C9418B0C257DF4F888156
:106720009981CE58D0400E945BB523961FAE1EAE15
:10673000239725961FAE1EAE259727961FAE1EAE39
:1067400027974AE0BE016F5F7F4F90E03EC0C2577F
:10675000DF4F88819981CE58D0400E945BB5682F69
:10676000880F770B4AE00AC0C257DF4F88819981B2
:10677000CE58D0400E9468B54AE0BC01CE010196D7
:106780000E949F48BE016F5F7F4FCE018F579F4F82
:106790000E94C047CE01019663C0C257DF4F888177
:1067A0009981CE58D0400E9468B523961FAE1EAE88
:1067B000239725961FAE1EAE259727961FAE1EAEB9
:1067C00027974AE0BE016F5F7F4F0E9409B435C032
:1067D000C257DF4F88819981CE58D0400E9463B55F
:1067E00023961FAE1EAE239725961FAE1EAE25978D
:1067F00027961FAE1EAE27972AE0AE014F5F5F4F70
:106800000E94DAB31AC0C257DF4F88819981CE58EF
:10681000D0400E9463B523961FAE1EAE23972596E7
:106820001FAE1EAE259727961FAE1EAE27972AE0F5
:10683000AE014F5F5F4F0E94E8B3BE016F5F7F4FB5
:10684000CE018F5B9F4F0E947A48BE016F5B7F4FE6
:10685000CE018F579F4F0E94C047CE018F5B9F4F45
:106860000E949A484BE050E0BE016F5B7F4FCE0123
:106870008F579F4F0E94EF88CB57DF4FF880C55846
:10688000D04011E002C0F12C10E0CE018F579F4F95
:106890000E949A48112309F4BCCD8E0109561F4F5E
:1068A00020E4AE014F5F5F4F68E87B2D8E2D0E9484
:1068B0006B90BE016F5B7F4FCE0101960E9450B37B
:1068C000C956DF4F8881C759D040F80E81E08F0D3F
:1068D000C956DF4F8883C759D040E1E0F0E0EC0FA4
:1068E000FD1FEF0DF11D9CE79083E1E0F0E0EC0F60
:1068F000FD1FE80FF11D1082BE016F5F7F4F809179
:10690000F5129091F6120E942D49C956DF4F688109
:10691000C759D04070E0CE0101960E944B90BC0157
:106920008091F5129091F6120E9465776AE080914D
:10693000F5129091F6120E9402498091F512909101
:10694000F612DC01ED91FC910284F385E02D19959E
:106950006AC18091350D9091360D8038910509F00E
:1069600062C18E0104571F4F20E4AE014F5F5F4F9D
:1069700068E870E880E00E946B906EEC75E0CE01F4
:106980008F579F4F0E94CA48CE018F579F4F0E943A
:10699000F888C457DF4F2881CC58D040CB57DF4F01
:1069A00088819981C558D040820F911DC457DF4F0F
:1069B0008883CC58D04022961FAE22974BE050E0FF
:1069C000BE016F5B7F4FCE018F579F4F0E946E7944
:1069D000BE016F5B7F4FCE0101960E9450B3C4573A
:1069E000DF4F8881CC58D040E1E0F0E0EC0FFD1F94
:1069F000E80FF11D1082BE016F5F7F4F8091F5128D
:106A00009091F6120E942D49C457DF4F6881CC58EF
:106A1000D04070E0CE0101960E944B90BC01809165
:106A2000F5129091F6120E9465776AE08091F51256
:106A30009091F6120E9402498091F5129091F612FF
:106A4000DC01ED91FC910284F385E02D1995CE01D6
:106A50008F579F4F0E949A48E6C08091350D9091C4
:106A6000360D8238910509F0DEC08E0104571F4FA4
:106A700020E4AE014F5F5F4F68E872E87BCF809102
:106A8000350D9091360D8138910509F0CCC080917B
:106A90003E0D8111C8C00E946991C5C08091350D1D
:106AA0009091360D4F9709F0BEC081E08093330D71
:106AB000BAC097D6029719F060E084E8ACCC809118
:106AC000DA0A811102C00E94EA770E944885F82EF6
:106AD00066EE75E0CE0184579F4F0E94CA48C956A2
:106AE000DF4F1882C759D0408E0109561F4F20E44E
:106AF000AE014F5F5F4F68E879E780E00E946B90DE
:106B0000CF57DF4F19821882C158D040CD57DF4F81
:106B100019821882C358D040CB57DF4F1982188290
:106B2000C558D0406F2D70E080E090E02AE0AE01C3
:106B30004F5B5F4F0E94DAB3BE016F5B7F4FCE01A8
:106B40008F579F4F0E947A48BE016F577F4FCE01EB
:106B500084579F4F0E94C047CE018F579F4F0E947E
:106B60009A484BE050E0BE016F5B7F4FCE018457E7
:106B70009F4F0E946E79C057DF4F1881C059D04097
:106B8000BE016F5B7F4FCE0101960E9450B3C95684
:106B9000DF4F8881C759D040810F91E0980FC956C7
:106BA000DF4F9883C759D040E1E0F0E0EC0FFD1FC4
:106BB000E80FF11D8CE78083E1E0F0E0EC0FFD1FB2
:106BC000E90FF11D1082BE016F5F7F4F8091F512BA
:106BD0009091F6120E942D49C956DF4F6881C7591E
:106BE000D04070E0CE0101960E944B90BC01809194
:106BF000F5129091F6120E9465776AE08091F51285
:106C00009091F6120E9402498091F5129091F6122D
:106C1000DC01ED91FC910284F385E02D1995CE0104
:106C200084579F4F17CF0FB6F894DEBE0FBECDBE70
:106C3000CA55DF4F0FB6F894DEBF0FBECDBFDF9150
:106C4000CF911F910F91FF90EF90DF90CF90BF9069
:106C5000AF909F908F907F906F905F904F903F90FC
:106C60002F900895809193068093920608958091C5
:106C7000670D882359F08091650D9091660DDC01B8
:106C8000ED91FC910480F581E02D19940895809197
:106C9000670D882369F08091650D9091660DDC0188
:106CA000ED91FC910190F081E02D6FEF73E019946C
:106CB00008958091670D882389F080916B0D88235A
:106CC00021F080E090E0D3DF03C080E090E0DFDFE0
:106CD00090916B0D81E0892780936B0D0895209131
:106CE000670D222369F0A091650DB091660DED91BD
:106CF000FC9111970190F081E02DBC01CD01199418
:106D000008958091640D882359F08091620D9091CF
:106D1000630DDC01ED91FC910480F581E02D199467
:106D200008958091640D882369F08091620D90919F
:106D3000630DDC01ED91FC910190F081E02D6FEF8E
:106D400073E0199408958091640D882389F08091EF
:106D50006A0D882321F080E090E0D3DF03C080E05B
:106D600090E0DFDF90916A0D81E0892780936A0DC2
:106D700008952091640D222369F0A091620DB091D5
:106D8000630DED91FC9111970190F081E02DBC0114
:106D9000CD01199408952091610D222369F0A091ED
:106DA0005F0DB091600DED91FC9111970190F08114
:106DB000E02DBC01CD011994089520915E0D222390
:106DC00069F0A0915C0DB0915D0DED91FC91119772
:106DD0000190F081E02DBC01CD011994089520911E
:106DE0005B0D222369F0A091590DB0915A0DED91E0
:106DF000FC9111970190F081E02DBC01CD01199417
:106E000008952091580D222369F0A091560DB0915C
:106E1000570DED91FC9111970190F081E02DBC018F
:106E2000CD01199408952091550D222369F0A09168
:106E3000530DB091540DED91FC9111970190F0819B
:106E4000E02DBC01CD01199408952091520D22230B
:106E500069F0A091500DB091510DED91FC911197F9
:106E60000190F081E02DBC01CD011994089520918D
:106E70004F0D222369F0A0914D0DB0914E0DED9173
:106E8000FC9111970190F081E02DBC01CD01199486
:106E9000089580918C0690918D06DC01ED91FC9116
:106EA000E65AFF4F0190F081E02D199480918C06F5
:106EB00090918D06DC01ED91FC91E85AFF4F019015
:106EC000F081E02D199480918C0690918D06DC0163
:106ED000ED91FC91EA5AFF4F0190F081E02D199459
:106EE0008091C50F81110DC0809107069091080611
:106EF000DC01ED91FC910190F081E02D60E070E00B
:106F0000199408958091C50F81110DC080910706D5
:106F100090910806DC01ED91FC910190F081E02D4B
:106F20006FEF70E0199408950C947F530C9495536F
:106F30008091690D882319F00E947F5302C00E943E
:106F400095539091690D81E089278093690D08958B
:106F50000C94AC530C94C2538091680D882319F0A3
:106F60000E94AC5302C00E94C2539091680D81E010
:106F700089278093680D089580919306882359F09E
:106F800030D4029741F063E270E1809190069091D5
:106F900091060C947A4A089580919206882341F0D4
:106FA00065E47FE080919006909191060C947A4A76
:106FB000089580919206882341F065E37FE08091F7
:106FC0009006909191060C947A4A0895CF93DF939E
:106FD00020916E0D30916F0D28173907D1F09093E5
:106FE0006F0D80936E0D20919206222391F0EC019B
:106FF00064EF7FE080919006909191060E9409498C
:10700000BE018091900690919106DF91CF910C94F2
:107010008373DF91CF910895CF93DF9320916C0D0F
:1070200030916D0D28173907D1F090936D0D809335
:107030006C0D20919206222391F0EC016AED7FE025
:1070400080919006909191060E940949BE0180911D
:10705000900690919106DF91CF910C948373DF910C
:10706000CF9108952091610D222339F0BC018091C8
:107070004B0D90914C0D0C94AA6A089520915E0DD1
:10708000222339F0BC018091490D90914A0D0C9456
:10709000AA6A089520915B0D222339F0BC018091EA
:1070A000470D9091480D0C94AA6A08952091580DAF
:1070B000222339F0BC018091450D9091460D0C942E
:1070C000AA6A08952091550D222339F0BC018091C0
:1070D000430D9091440D0C94AA6A08952091520D8D
:1070E000222339F0BC018091410D9091420D0C9406
:1070F000AA6A089520914F0D222339F0BC01809196
:107100003F0D9091400D0C94AA6A0895CF92DF92A2
:10711000EF92FF9220910002213019F42091D10FBB
:1071200004C02230C9F52091D70F2223A9F19C0178
:10713000211584E0380710F02FEF33E0ADE0B0E028
:107140000E94C9B52FEF33E040E050E00E947BB5CC
:1071500069017A018FEFC81AD80AE80AF80A809103
:10716000CD128C15C9F0C092CD1280919206882361
:1071700099F063E97FE080919006909191060E94DA
:1071800009496C2D8091900690919106FF90EF90A7
:10719000DF90CF900C94F675FF90EF90DF90CF903A
:1071A0000895CF92DF92EF92FF922091000221305A
:1071B00019F42091CE0F04C02230C9F52091D40FCC
:1071C0002223A9F19C01211584E0380710F02FEF4C
:1071D00033E0ADE0B0E00E94C9B52FEF33E040E00E
:1071E00050E00E947BB569017A018FEFC81AD80A76
:1071F000E80AF80A8091CB128C15C9F0C092CB1224
:1072000080919206882399F06CE77FE08091900648
:10721000909191060E9409496C2D80919006909161
:107220009106FF90EF90DF90CF900C94F675FF9051
:10723000EF90DF90CF90089581E0809389060E94BF
:107240001A5680919206882341F062E67FE0809191
:107250009006909191060C947A4A089583E0809369
:1072600089060E944A5480919206882341F06FE675
:107270007FE080919006909191060C947A4A08954F
:1072800082E0809389060E944A5480919206882366
:1072900041F065E57FE080919006909191060C9415
:1072A0007A4A08950C946C918091010281110C949A
:1072B00005460C946C910C94054680910002813037
:1072C00011F482E001C081E00C94E08D82E00C9426
:1072D000E08D81E00C94E08D0C94360D9091F60FCA
:1072E00081E089270C94615580E00C94615581E020
:1072F0000C9461559091F40F81E089270C9493557B
:1073000080E00C94935581E00C94935580912B066A
:10731000882329F00E947F5325E933E504C00E94A9
:1073200095532FE733E54CE251E060E070E080EFE9
:107330009AE00C94768080912406882329F00E949C
:10734000AC5322EC33E504C00E94C2532CEA33E56F
:107350004CE251E060E070E080EF9AE00C947680BF
:107360008CE00C94BE448BE00C94BE448CE00C94F6
:10737000F8448BE00C94F8448CE00C9432458BE09C
:107380000C943245682F80919006909191060E944E
:107390004B7761E270E180919006909191060C9498
:1073A0000949F0DF80919006909191060C94674A0C
:1073B000CF92DF92EF92FF929C01A3E6B0E00E9491
:1073C000C9B52FEF33E040E050E00E947BB5690182
:1073D0007A018FEFC81AD80AE80AF80A8091EC05FA
:1073E0008C15A1F0C092EC0580919206882371F073
:1073F00063EC7FE080919006909191060E9409498C
:107400008C2DFF90EF90DF90CF90CBCFFF90EF903F
:10741000DF90CF900895CF92DF92EF92FF929C0180
:10742000A3E6B0E00E94C9B52FEF33E040E050E0A2
:107430000E947BB569017A018FEFC81AD80AE80A61
:10744000F80A8091ED058C15A1F0C092ED058091B0
:107450009206882371F06AEA7FE08091900690910D
:1074600091060E9409498C2DFF90EF90DF90CF90FC
:1074700098CFFF90EF90DF90CF90089520919006E5
:1074800030919106882319F06BE377E002C06FE337
:1074900077E0C9010C940949F1DF80919006909141
:1074A00091060C94674A20919006309191068823AA
:1074B00019F066E170E102C06BE170E1C9010E9460
:1074C000094980919006909191060C94674A64E175
:1074D00070E180919006909191060C94094960E1C9
:1074E00070E180919006909191060C940949CF9398
:1074F000CDE26EE070E180919006909191060E943D
:107500000949C150B1F780919006909191060E946F
:10751000674A8091900690919106DC01ED91FC9173
:107520000284F385E02DCF9119948091D50A8111C1
:1075300057C0E0915B11F0915C1185819681909329
:1075400058118093571110925A1110925911E091CD
:107550006511F091661185819681909362118093F7
:1075600061111092641110926311E0916F11F0910A
:1075700070118581968190936C1180936B1110929C
:107580006E1110926D11E0917911F0917A1185814F
:1075900096819093761180937511109278111092C4
:1075A000771182E190E090934F1180934E1181E02A
:1075B0008093541180935E118093681180937211AF
:1075C0008093501180E090E021E0FC01E650FF4EF6
:1075D0002183079684359105C1F781E08093D50A10
:1075E000089510927411089510926A1108958F925F
:1075F0009F92AF92BF92CF92DF92EF92FF921F9332
:10760000CF93DF93EC0111E08E819F81892B09F4E8
:1076100010E02C813D81E885F985C580D680878181
:1076200090E0A601480F591F2417350764F18085A3
:107630000D2C000CEE08FF08A901330F660B770B29
:107640000380F481E02D9A01AB012C193D094E090C
:107650005F09882329F0A1E0BFEF0E94A3B504C011
:10766000AFEFB0E00E9497B54F01FF0FAA08BB082B
:10767000A50194012C193D094E095F090E947BB5B3
:107680003F832E834BC0A601481B590B421753075B
:107690000CF43FC080850D2C000CEE08FF08A901FA
:1076A000330F660B770B81809280092C000CAA089F
:1076B000BB089A01AB01281939094A095B098823DB
:1076C00099F0A1E0BFEF0E94A3B5A7019601281988
:1076D00039094A095B090E947BB5DA01C901815069
:1076E0009F4FAF4FBF4F12C0AFEFB0E00E9497B5B2
:1076F000A7019601281939094A095B090E947BB53F
:10770000DA01C9018F5F9109A109B1099F838E83B5
:1077100005C01F821E82111101C019828E819F81B6
:10772000009789F08F3F910519F014F08FEF90E0EA
:1077300081305FEF950714F481E09FEF9F838E8384
:1077400081E018271A83DF91CF911F91FF90EF906E
:10775000DF90CF90BF90AF909F908F90089581E081
:107760008093D20A089581E08093D30A089581E03E
:107770008093D40A0895CF93DF93C091A70DD09141
:10778000A80D6091B40D7091B50DCE010E940F80CF
:1077900081110DC025E93AE34CE251E060E070E070
:1077A000CE010E9476809093B50D8093B40DDF9149
:1077B000CF9108958091DB0A823039F0833051F007
:1077C000813069F48091AE0D08950E9427858091E3
:1077D000911208950E941C858091AD0D089580E05E
:1077E00008958091DB0A823049F0833071F0813056
:1077F00099F48091A90D9091AA0D08950E94278572
:10780000809195129091961208950E941C85809106
:10781000AB0D9091AC0D089581E090E008952F920A
:107820003F925F926F927F928F929F92AF92CF9290
:10783000DF92EF92FF920F931F93CF93DF931F92EC
:107840001F92CDB7DEB76DB67EB60E9427850E9427
:107850001C85C7DF029709F01FC2ACDF882309F43B
:1078600016C2C090B40DD090B50DE090A70DF09069
:10787000A80DB601C7010E940F808823F1F0F7011F
:10788000E250FE4F00E010E0819191918C159D0532
:1078900071F40E94D36D000F111F000F111FF7012B
:1078A000E00FF11F608371838283938307C00F5FB2
:1078B0001F4F0E31110541F701C05DDF1092D50A4F
:1078C000EDB6FEB64091D80A5091D90ACA01880F88
:1078D000991F2DB73EB7281B390B0FB6F8943EBF42
:1078E0000FBE2DBF0DB71EB70F5F1F4F8091DB0A74
:1078F000823069F0833029F1813009F071C0B8011C
:1079000080916B1290916C120E94238F33C03FB70D
:10791000F89420E0822F90E08417950774F4880F84
:10792000991FF801E80FF91FDC01AF58BD4E8D918A
:107930009C91918380832F5FEDCF3FBF1092911276
:1079400019C03FB7F89420E0822F90E08417950784
:1079500074F4880F991FF801E80FF91FDC01A5578F
:10796000B24F8D919C91918380832F5FEDCF3FBF6C
:107970001092AD0D20E06AE071E0822F90E040911E
:10798000D80A5091D90A8417950754F5689FF001D9
:10799000699FF00D1124E65AFF4EA085B1858C91A8
:1079A0008823E1F0A081B1813C91C801830F911D32
:1079B000830F911DDC0112978D919C91A281B3815F
:1079C0004D915C9111970480F581E02D481759077E
:1079D00011F4108203C070838D939C932F5FCDCFE1
:1079E0000FB6F894FEBE0FBEEDBE809154118823F1
:1079F00019F083E591E1FBDD80915E11882319F098
:107A00008DE591E1F4DD80916811882319F087E616
:107A100091E1EDDD80917211882319F081E791E108
:107A2000E6DD8091D60A882309F465C0809168114B
:107A3000811105C080917211882309F450C0809192
:107A40006B1190916C11E0916F11F0917011238185
:107A500034812817390724F48085811109C00EC0AC
:107A6000218132818217930734F48085811106C009
:107A700088E090E005C080E190E002C080E290E004
:107A80002091751130917611E0917911F0917A1170
:107A9000438154814217530724F42085222349F05F
:107AA0000AC041815281241735073CF420852223E6
:107AB00011F0816003C0846001C0826020914E118A
:107AC00030914F112817390719F41092501107C03F
:107AD00090934F1180934E1181E0809350118091CB
:107AE0004E1190914F11429709F4DAC081E08093D2
:107AF000741180936A11EBEFF0E18EEF90E19A83BD
:107B0000898398EE892E93E0992E55245394CF01C2
:107B10000197DC018C91882309F4ACC0E480F580E6
:107B2000D70117968C911797882309F4A3C08081F9
:107B3000882309F49FC04181528118966C91840179
:107B4000041B150B101611061CF08A01085E134069
:107B500020E030E022242394312C8FE097E2A12C06
:107B6000C62ED12C2C143D04ACF56430A9F040F4A1
:107B7000623071F0633019F5C90184559A4F13C012
:107B8000653071F06630D9F4C90182579A4F0BC045
:107B9000C9018E549A4F07C0C9018C559A4F03C032
:107BA000C90186569A4FDC0112968D919C911397CC
:107BB000841B950B97FF03C09195819591098017C0
:107BC000910714F4A22C8C01BFEF2B1A3B0A2E5FF5
:107BD0003F4FC8CF81E08A0DD70119969C91992318
:107BE000F1F1643099F028F4623041F0633049F0EB
:107BF00036C06530A1F06630D9F031C0813021F552
:107C00002DC0813049F1833051F51EC0813011F112
:107C1000823011F1833011F1843009F515C08130C3
:107C2000B9F08230B9F08430C9F08530C1F40CC0AD
:107C3000813061F0823061F0833061F0843061F036
:107C4000853061F0863059F481E009C086E007C0D4
:107C500085E005C084E003C083E001C082E0A98123
:107C6000BA819C91981302C0108204C05082A981ED
:107C7000BA818C93379629813A81295F3F4F3A83A5
:107C8000298331E1EF34F30709F041CF03C00E94AB
:107C9000338571DD81E066C00E94338580E062C07B
:107CA000E0905111F09052111E141F040CF055C0B9
:107CB000809169110091A70D1091A80D6091B20DEE
:107CC0007091B30D8823B1F081E080936A11C801EF
:107CD0000E940F80811115C0A701FF0C660B770B66
:107CE00024EF3AE3C8010E9476809093B30D80930D
:107CF000B20D07C0C8010E940F80811102C010920E
:107D00006A11809173110091A70D1091A80D6091D7
:107D1000B00D7091B10D8823D1F081E08093741182
:107D2000C8010E940F808111E6CE409151115091FF
:107D30005211052E000C660B770B21EF3AE3C801B8
:107D40000E9476809093B10D8093B00DD4CEC8017F
:107D50000E940F808111CFCE02C010926A11109242
:107D60007411C9CE0FB6F8947EBE0FBE6DBE0F90D3
:107D70000F90DF91CF911F910F91FF90EF90DF90C7
:107D8000CF90AF909F908F907F906F905F903F903B
:107D90002F900895CF938091AF0DC0910A02811169
:107DA00001C1C23009F450C0C33009F49DC0C130D4
:107DB00009F028C18091D40A811124C181E090E0AA
:107DC0000E9432B190936C1280936B1262E083E058
:107DD0000E94B04C1092880D1092AA0D1092A90D1D
:107DE0001092AE0D80E090E0FC01EE0FFF1FEA580C
:107DF000F24F11821082019688309105A9F71092F6
:107E0000870D1092860D80916A008C6080936A00C5
:107E1000ED9A8FB7F89420918400309185003093CB
:107E2000710D2093700D8FBF27EB3BE34AEF50E0BD
:107E300060E070E08091A70D9091A80D0E9476807F
:107E400081E08093AF0DDEC08091D30A8111DAC04A
:107E500081E090E00E9432B190936E1280936D1297
:107E6000809104018E7F80930401809105018160DF
:107E70008093050185EF96E0909398128093971276
:107E80002EE240EA56E861E070E00E94F44B8091F7
:107E900065008B7F809365001092350189E08093A7
:107EA00034018EE2809332018CEF8093300180E9BF
:107EB00080933101109296121092951210929412A2
:107EC0001092931210929112E1E7F2E18CED95E09D
:107ED0008193919322E1E139F207D1F7C1E0C09398
:107EE000921223EB3BE351C08091D20A81118AC0E8
:107EF00081E090E00E9432B19093701280936F12F3
:107F0000809104018E7F809304018091050181603E
:107F10008093050185EF96E090938A0D8093890DFB
:107F200026E040E052EC61E070E00E94F44B80916A
:107F300065008B7F809365001092350180E180930E
:107F4000340186E0809332018EEF8093300180E926
:107F5000809331011092AC0D1092AB0D1092750D03
:107F60001092740D1092AD0DEBE8FDE08CED95E0F4
:107F7000819391932DE0E73AF207D1F71092730DB8
:107F8000C1E0C093720D2FEA3BE34AEF50E060E09E
:107F900070E08091A70D9091A80D0E947680C0930B
:107FA000AF0D30C0C23069F0C330D1F0C13051F5EF
:107FB0008091D40A811126C08091A90D9091AA0DBB
:107FC0001DC08091D30A81111DC080916D129091C6
:107FD0006E120E94298480919512909196120EC083
:107FE0008091D20A81110EC080916F12909170120F
:107FF0000E94337A8091AB0D9091AC0D029711F4F1
:10800000C093DB0A80910A028230A1F1833009F427
:1080100054C0813009F074C08091D40A882309F4D7
:108020006FC0ED98E59A1092880D10926A12109226
:10803000AA0D1092A90D1092AE0D80E090E0FC0107
:10804000EE0FFF1FEA58F24F11821082019688301E
:108050009105A9F71092870D1092860D80916B12F1
:1080600090916C120E94C7B11092AF0D1092D30A7A
:1080700082E044C08091D30A882309F441C08091F2
:108080009712909198120E94D24B809131018F7774
:1080900080933101809131018F7E80933101109264
:1080A000300180916D1290916E120E94C7B11092B2
:1080B000AF0D1092D20A83E021C08091D20A8823AA
:1080C000F9F08091890D90918A0D0E94D24B809198
:1080D00031018F7780933101809131018F7E8093C0
:1080E00031011092300180916F12909170120E94B4
:1080F000C7B11092AF0D1092D40A81E080930A02AA
:108100008091A70D9091A80DCF910C948680AF928D
:10811000BF92CF92DF92EF92FF920F931F93CF9374
:10812000DF937C016B015A01D0E0C0E08D2F90E01D
:10813000F701A181B2818A159B05D0F4F601E80F01
:10814000F91F608100E513E821E03327C6270C0FF3
:10815000111D211D311D2BBFF801C791ED91FC911F
:1081600011970190F081E02DCD011995DF5FDECFF1
:10817000ED91FC9111970190F081E02D6C2FCD01D4
:10818000DF91CF911F910F91FF90EF90DF90CF90F3
:10819000BF90AF901994CF93DF9300D01F921F929E
:1081A000CDB7DEB7FE01319625E0DF011D922A959D
:1081B000E9F724E8298325E52C832AE22D836A83C5
:1081C0004B8345E050E0BF01A2DF65E070E080E056
:1081D00090E00E94D24D80E00F900F900F900F9092
:1081E0000F90DF91CF910895EF92FF921F93CF935D
:1081F000DF931F92CDB7DEB77C01162FFC016181A2
:1082000072810E94807665E070E080E090E00E94DC
:10821000D24D42E462E4C701BEDF412F60E0C701F6
:10822000BADF811163C040E061E0C701B4DF8111B2
:108230005DC040E062E0C701AEDF811157C046E09B
:1082400062E0C701A8DF811151C040E063E0C701CF
:10825000A2DF81114BC040E064E0C7019CDF11E068
:10826000811110E040E065E0C70195DF811101C098
:108270001F5F40E066E0C7018EDF811101C01F5F14
:1082800040E067E0C70187DF811101C01F5F40E068
:1082900068E0C70180DF811101C01F5F40E069E035
:1082A000C70179DF811101C01F5F44E06AE0C701A7
:1082B00072DF811101C01F5F44E06AE0C7016BDF1C
:1082C000811101C01F5F62E370E080E090E00E94D6
:1082D000D24D82E8898341E050E0BE016F5F7F4F5D
:1082E000C70115DF81E0183011F0111180E00F9007
:1082F000DF91CF911F91FF90EF9008950C94B78676
:108300000C94F0868091C30D882319F00E94B786E3
:1083100002C00E94F0869091C30D81E0892780936E
:10832000C30D08950F931F93CF93DF932091C50F33
:1083300021111BC0C0910706D09108060881198140
:108340009C01AFEFB0E00E94C9B52FEF33E040E0F1
:1083500050E00E947BB5D801ED91FC91B901CE01AE
:10836000DF91CF911F910F911994DF91CF911F91C0
:108370000F91089580913D12811102C00C94F07EFE
:108380000895CF93DF9380913D12882321F11092BD
:108390003D1260E088E00E94814CC0913E12D09175
:1083A0003F12BE0180EF9AE00E940F80882329F0DF
:1083B000BE0180EF9AE00E94278080919206882378
:1083C00071F069E771E18091900690919106DF91DB
:1083D000CF910C947A4ADF91CF910C94F07EDF918B
:1083E000CF9108950F931F93CF93DF930091BE0D0C
:1083F0001091BF0DC091F805D091F905B801CE01DB
:108400000E940F80882379F0B801CE010E94278056
:108410008091FA059091FB05DC01ED91FC9100A0A3
:10842000F1A1E02D19950091BC0D1091BD0DC091E9
:10843000F805D091F905B801CE010E940F8088237C
:1084400021F0B801CE010E94278072988091920697
:10845000882361F06AE271E1809190069091910623
:10846000DF91CF911F910F910C947A4ADF91CF91B8
:108470001F910F910895CF93DF938091401288232D
:1084800011F10E94B78610924012C0913E12D09115
:108490003F12BE0180EF9AE00E940F80882329F0EE
:1084A000BE0180EF9AE00E94278080919206882387
:1084B00071F060E671E18091900690919106DF91F4
:1084C000CF910C947A4ADF91CF910C940587DF917C
:1084D000CF9108950C9405870E94B786409148106B
:1084E0005091491060E070E020EF36E880EF9AE0AC
:1084F0000E94768090933F1280933E128091920664
:10850000882339F065E471E180919006909191069D
:10851000F1C708950E94F08640914810509149108B
:1085200060E070E027EB36E880EF9AE00E9476800A
:1085300090933F1280933E1280919206882339F0E7
:1085400062E371E18091900690919106D3C70895FE
:108550008091C40D882319F00E94B78602C00E9442
:1085600026889091C40D81E089278093C40D0895D9
:108570000C9426880C9439880C9450888091C20DF4
:10858000882319F00E94398802C00E945088909177
:10859000C20D81E089278093C20D08950C947A88DA
:1085A0000E947A8880918C0690918D06DC01ED9175
:1085B000FC9104A0F5A1E02D19940C94B78880914A
:1085C000C10D882319F00E947A8802C00E94B788E2
:1085D0009091C10D81E089278093C10D08950C947D
:1085E000D3880C947D548091C00D882319F00E948B
:1085F000D38802C00E947D549091C00D81E08927EC
:108600008093C00D08950C94F18E80913D0E8111E0
:108610000C94DB8E0C94F18E0C94DB8E0E944087C0
:1086200080918C0690918D06DC01ED91FC9102A069
:10863000F3A1E02D1994CF93DF93C091F805D09169
:10864000F9056091BE0D7091BF0DCE010E940F80A3
:10865000811129C04091BA0D50E060E070E027EB35
:108660003AE6CE010E947E809093BF0D8093BE0DAE
:108670008091FA059091FB05DC01ED91FC91068C4F
:10868000F78DE02D199580911506882361F0609192
:10869000BC0D7091BD0D8091F8059091F9050E9477
:1086A0000F80882369F0809192068823E1F061E2CF
:1086B00071E18091900690919106DF91CF911AC758
:1086C0000E94A76D27EA3DE644E650E060E070E0D6
:1086D0008091F8059091F9050E947E809093BD0DE0
:1086E0008093BC0DE0CFDF91CF9108950E940F7071
:1086F00080919206882339F066EF70E180919006B0
:1087000090919106F7C60895E091B80DF091B90DDA
:1087100082810E94E58180919206882339F068ED7C
:1087200070E18091900690919106E4C60895809141
:108730003E0E882319F00E94787002C00E94627079
:1087400080919206882371F02091B70F8091900656
:1087500090919106222319F06CE970E102C065EB5B
:1087600070E1C8C608950C941A56CF938091C70A39
:10877000882309F46DC00E94BC709091C50A8823BB
:1087800039F0911165C080911C06882331F160C0D9
:1087900091115EC080919206882339F06DE770E1F7
:1087A0008091900690919106A5D60E945D7181E01E
:1087B0008093050680910702813009F049C08091BD
:1087C000F10F882309F444C08091B70F8823E9F0A2
:1087D00080913D0E81112EC018C082E080931C064E
:1087E00080919206882339F069E870E180919006C3
:1087F000909191067FD6C1E0C0931B060E941A5645
:108800000E945D71C093050623C04091B90F50913D
:10881000BA0F141615065CF4052E000C660B770BC8
:1088200021EA3DE880EF9AE0CF910C947680CF91D9
:108830000C94A18D2CEA3DE842E350E060E070E04A
:1088400080EF9AE00E947E809093B70D8093B60DE2
:10885000CF9108950C944A548091880681110C940C
:108860001A560C944A540C94BE560C94B0570E945D
:10887000427E8091F00581110C94BE560C94B05745
:1088800061E770E18091900690919106C2C4CF9308
:108890009C01A4E6B0E00E94C9B52FEF33E040E0B0
:1088A00050E00E947BB5C22F30E08091BB0D281BA9
:1088B000310937FF03C03195219531092330310546
:1088C00034F1C33020F0C23618F0C4E601C0C0E075
:1088D00080918C0690918D06DC01ED91FC91EC5A13
:1088E000FF4F0190F081E02D6C2F1995C093BB0DC7
:1088F00080919206882359F069E470E18091900696
:108900009091910686D48C2FCF910C94D139CF9130
:1089100008959C010197849710F4822F0895C9014E
:10892000845691098438934040F4C90164E670E0AC
:108930000E94F1AF822F94E61BC0283E43E034072B
:10894000D8F0C90168EE73E00E94F1AF48E15CEF36
:10895000649FC001659F900D749F900D1124280F96
:10896000391FC9016AE070E00E9405B0822F9AE0C9
:10897000699F80191124089580E00895CF93C82F2E
:1089800080918C0690918D06DC01ED91FC91EE5B5F
:10899000FF4F0190F081E02D6C2F19958091920688
:1089A000882381F06DDF6C2F809190069091910665
:1089B0000E944B7769E670E1809190069091910654
:1089C000CF9198C5CF9108958AE0D8CF89E0D6CFCE
:1089D00088E0D4CF87E0D2CF86E0D0CF85E0CECF7D
:1089E00084E0CCCF83E0CACF82E0C8CF81E0C6CF9D
:1089F000CF93C82F80918C0690918D06DC01ED916C
:108A0000FC91E05CFF4F0190F081E02D6C2F1995F7
:108A100080919206882381F033DF6C2F809190063D
:108A2000909191060E944B7766E570E180919006E7
:108A300090919106CF915EC5CF9108958AE0D8CFED
:108A400089E0D6CF88E0D4CF87E0D2CF86E0D0CF00
:108A500085E0CECF84E0CCCF83E0CACF82E0C8CF20
:108A600081E0C6CFCF93C82F80918C0690918D0660
:108A7000DC01ED91FC9106ACF7ADE02D6C2F199562
:108A800080919206882349F0FBDE6C2F809190063E
:108A900090919106CF910C94F675CF9108958AE04C
:108AA000E1CF89E0DFCF88E0DDCF87E0DBCF86E074
:108AB000D9CF85E0D7CF84E0D5CF83E0D3CF82E094
:108AC000D1CF81E0CFCF80918C0690918D06DC01D3
:108AD000ED91FC910484F585E02D60E01994F3CFCD
:108AE00080918C0690918D06DC01ED91FC910484BF
:108AF000F585E02D61E01994F3CFCF93DF9380915A
:108B0000C50F882349F180910102882329F1C09182
:108B10000706D09108068BA19CA1892B11F01CA2FD
:108B20001BA22D8D3E8D8B8D9C8D9B878A873D87CB
:108B30002C879F878E87E881F9810190F081E02D55
:108B400060E070E0CE0119951F8A1E8A0E94D36DE5
:108B50006F8F78A389A39AA3DF91CF910895CF93C4
:108B6000DF938091C50F882349F18091010288230A
:108B700029F1C0910706D09108068BA19CA1892BF1
:108B800011F01CA21BA22D8D3E8D898D9A8D9B8785
:108B90008A873D872C879F878E87E881F98101909E
:108BA000F081E02D60E070E0CE0119951F8A1E8AE9
:108BB0000E94D36D6F8F78A389A39AA3DF91CF9181
:108BC00008951F93CF93DF939091C50F9923C9F018
:108BD000182FC0910706D0910806CE010E94B265F9
:108BE0008E899F89892B49F4112319F0898D9A8DDB
:108BF00002C08B8D9C8D9F8B8E8B81E090E09CA31F
:108C00008BA3DF91CF911F9108958091010288235A
:108C1000B1F01092010280919206882339F069E345
:108C200070E1809190069091910664D40E94427EFA
:108C30008091F005882319F080918806C2CF0895AD
:108C40000895CF92DF92EF92FF920F931F93CF93ED
:108C5000DF936C017A018B01C0E0D0E0CE15DF0517
:108C600089F0D8016D918D01D601ED91FC910190B3
:108C7000F081E02DC6011995892B11F47E0102C007
:108C80002196ECCFC701DF91CF911F910F91FF90FB
:108C9000EF90DF90CF900895FC01A089B1898C916D
:108CA000A689B78982FD0FC09C91818D8F5F8F73DC
:108CB000228D821749F0218DDF01A20FB11D5D9633
:108CC0009C93818F08958C910895FC01918D828DE4
:108CD000981761F0828DDF01A80FB11D5D968C9110
:108CE000928D9F5F9F73928F90E008958FEF9FEF1B
:108CF0000895FC01918D828D981731F0828DE80FD7
:108D0000F11D858D90E008958FEF9FEF0895FC0190
:108D1000918D228D892F90E0805C9F4F821B91095D
:108D20008F739927089585EF96E0F1DF21E0892B75
:108D300009F420E0822F089582E997E0E8DF21E03E
:108D4000892B09F420E0822F08958FE298E0DFDF7D
:108D500021E0892B09F420E0822F08958CEC98E023
:108D6000D6DF21E0892B09F420E0822F0895FC0151
:108D7000848DDF01A80FB11DA35ABF4F2C91848DA4
:108D800090E001968F739927848FA689B7892C93D9
:108D9000A089B1898C9180648C93938D848D981374
:108DA00006C00288F389E02D80818F7D808308953D
:108DB000EF92FF920F931F93CF93DF93EC0181E02B
:108DC000888F9B8D8C8D981305C0E889F9898081E7
:108DD00085FD23C0F62E0B8D10E00F5F1F4F0F7324
:108DE0001127E02E8C8DE8120BC00FB607FCFACFCE
:108DF000E889F989808185FFF5CFCE01B8DFF2CF10
:108E00008B8DFE01E80FF11DE35AFF4FF0820B8FAF
:108E1000EA89FB898081806207C0EE89FF896083CF
:108E2000E889F98980818064808381E090E0DF9126
:108E3000CF911F910F91FF90EF900895CF93DF9303
:108E4000EC01888D8823C1F0EA89FB89808185FD4A
:108E500005C0A889B9898C9186FD0EC00FB607FCA4
:108E6000F5CF808185FFF2CFA889B9898C9185FFE4
:108E7000EDCFCE017CDFE8CFDF91CF91089580E088
:108E800090E0892B19F06ADF811116C080E090E034
:108E9000892B19F05ADF811112C080E090E0892BF4
:108EA00019F04ADF81110EC080E090E0892B79F043
:108EB0003ADF81110AC008950E940000E7CF0E94A6
:108EC0000000EBCF0E940000EFCF0C94000008954B
:108ED00090E0FC013197E231F10508F04EC088279F
:108EE000EC5BFE4F8F4F0C9418B0809180008F7711
:108EF00003C0809180008F7D8093800008958091D1
:108F00008000877FF9CF84B58F7702C084B58F7DCD
:108F100084BD08958091B0008F7703C08091B00028
:108F20008F7D8093B0000895809190008F7707C067
:108F3000809190008F7D03C080919000877F809307
:108F4000900008958091A0008F7707C08091A000C5
:108F50008F7D03C08091A000877F8093A00008953B
:108F6000809120018F7707C0809120018F7D03C001
:108F700080912001877F8093200108950E9443B350
:108F80000F931F93CF93DF938C01EB01FC01808142
:108F900091810097B1F0688179816115710579F04F
:108FA000428153812C813D814217530740F00E943A
:108FB0005BB38C819D81F8019583848313C00E94EB
:108FC000C7B188819981F801918380838A819B81CF
:108FD000938382838C819D819583848319821882F7
:108FE0001B821A821D821C82DF91CF911F910F91EB
:108FF00008950F931F93CF93DF93EC01888199819C
:10900000009729F02A813B812617370788F48B01C6
:109010006F5F7F4F0E945FB2009761F099838883F2
:109020001B830A832C813D81232B11F4FC011082C8
:1090300081E001C080E0DF91CF911F910F910895F1
:10904000EF92FF920F931F93CF93DF93FB01248145
:109050003581E080F180FC0104811581E114F10487
:1090600011F480E016C02115310591F0EC01020FDA
:10907000131FB801BEDF8823A1F3288139818C81B9
:109080009D81B701820F931F0E945BB31D830C83E8
:1090900081E0DF91CF911F910F91FF90EF900895A4
:1090A000EF92FF920F931F93CF93DF93EC017B011D
:1090B0008A01BA019EDF2881398181110DC02115F5
:1090C000310519F0C9010E94C7B1198218821D82A9
:1090D0001C821B821A8206C01D830C83B701C90142
:1090E0000E945BB3CE01DF91CF911F910F91FF9052
:1090F000EF900895CF93DF93EC016115710551F066
:10910000FB0101900020E9F73197AF01461B570B97
:10911000C7DF0CC088819981009711F00E94C7B108
:10912000198218821D821C821B821A82CE01DF9155
:10913000CF910895FC01808191810C94C7B10F9368
:109140001F93CF93DF93CDB7DEB762970FB6F89436
:10915000DEBF0FBECDBF8C01CB01F80111821082A2
:10916000138212821582148250E0BE016F5F7F4F1E
:109170000E94C6B3BE016F5F7F4FC801BBDF62961E
:109180000FB6F894DEBF0FBECDBFDF91CF911F9118
:109190000F910895FC0111821082138212821582B0
:1091A00014826115710549F0FB0101900020E9F777
:1091B0003197AF01461B570B73CF0895CF93DF93C1
:1091C00000D01F92CDB7DEB76115710581059105FD
:1091D00079F09B01AC0169833A834B835C830E94E5
:1091E000BAB329813A814B815C810E947BB503C06F
:1091F00060E070E0CB010F900F900F900F90DF9127
:10920000CF910895DC01ED91FC910190F081E02D6A
:109210001994EF92FF920F931F93CF93DF938C01DA
:109220007B01C0E0D0E0F701EC0FFD1F64916623E5
:1092300061F0D801ED91FC910190F081E02DC80121
:109240001995892B11F02196EECFCE01DF91CF91A8
:109250001F910F91FF90EF9008956115710579F0BE
:10926000FB0101900020E9F73197AF01461B570B36
:10927000DC01ED91FC910280F381E02D199480E0F6
:1092800090E008954F925F926F927F92EF92FF92DB
:109290000F931F93CF93DF93CDB7DEB7A1970FB690
:1092A000F894DEBF0FBECDBF7C01FA01CB0119A23D
:1092B000223008F42AE08E010F5D1F4F422E512C00
:1092C000612C712CBF01A30192010E94A7B5F90185
:1092D000CA01015011096A3014F4605D01C0695C73
:1092E000D8016C93232B242B252B61F7B801C701E0
:1092F000B4DFA1960FB6F894DEBF0FBECDBFDF91ED
:10930000CF911F910F91FF90EF907F906F905F90A2
:109310004F9008954F925F926F927F928F929F929B
:10932000AF92BF92CF92DF92EF92FF92CF93DF93F3
:10933000EC016A017B01B22E9A01AB01C701B601B3
:109340000E942EB1882319F068ED75E027C0260130
:109350003701E89477F82FEF3FEF4FE75FE7C3015E
:10936000B2010E942EB181110DC02FEF3FEF4FE7E8
:109370005FE7C301B2010E9432B418161CF46CED11
:1093800075E00CC02FEF3FEF4FE75FE4C701B60178
:109390000E942AB1181694F460EE75E0CE01DF91B8
:1093A000CF91FF90EF90DF90CF90BF90AF909F90C4
:1093B0008F907F906F905F904F904FCF2FEF3FEF48
:1093C0004FE75FECC701B6010E9432B487FDE4CFDE
:1093D00020E030E0A901C701B6010E9432B487FF46
:1093E00009C06DE2CE010EDF4C01F7FAF094F7F8F8
:1093F000F09402C0812C912CA12C60E070E080E000
:109400009FE3AB1441F020E030E040E251E40E94E1
:1094100091B0A394F6CF9B01AC01C701B6010E94A5
:109420002DB02B013C010E94FEB06B017C010E941B
:1094300036B49B01AC01C301B2010E942CB02B01D8
:109440003C012AE0B701A601CE011CDF7C01E80C3B
:10945000F91CBB2029F06EE2CE01D4DEE80EF91E25
:10946000DB2CDD2021F120E030E040E251E4C301BB
:10947000B2010E9497B42B013C010E94FEB04B0147
:10948000A12CB12C2AE0B501A401CE01FBDEE80E2F
:10949000F91EC501B4010E9436B49B01AC01C301A1
:1094A000B2010E942CB02B013C01DA94DACFC70143
:1094B000DF91CF91FF90EF90DF90CF90BF90AF9072
:1094C0009F908F907F906F905F904F90089564EE83
:1094D00075E0C3CE0F931F93CF93DF93EC01BDDEF6
:1094E0008C01CE01F4DF800F911FDF91CF911F918E
:1094F0000F9108950F931F93CF93DF93EC0189DEB3
:109500008C01CE01E4DF800F911FDF91CF911F917D
:109510000F9108951F920F920FB60F9211240BB660
:109520000F922F933F934F935F936F937F938F93FC
:109530009F93AF93BF93EF93FF9385EF96E017DC74
:10954000FF91EF91BF91AF919F918F917F916F911B
:109550005F914F913F912F910F900BBE0F900FBED7
:109560000F901F9018951F920F920FB60F92112413
:109570000BB60F922F933F934F935F936F937F930D
:109580008F939F93AF93BF93EF93FF9385EF96E0F5
:1095900083DBFF91EF91BF91AF919F918F917F916D
:1095A0006F915F914F913F912F910F900BBE0F9054
:1095B0000FBE0F901F9018951F920F920FB60F922B
:1095C00011240BB60F922F933F934F935F936F939A
:1095D0007F938F939F93AF93BF93EF93FF9382E912
:1095E00097E0C5DBFF91EF91BF91AF919F918F9174
:1095F0007F916F915F914F913F912F910F900BBE93
:109600000F900FBE0F901F9018951F920F920FB6DC
:109610000F9211240BB60F922F933F934F935F93AA
:109620006F937F938F939F93AF93BF93EF93FF932A
:1096300082E997E031DBFF91EF91BF91AF919F916C
:109640008F917F916F915F914F913F912F910F90EB
:109650000BBE0F900FBE0F901F9018951F920F9288
:109660000FB60F9211240BB60F922F933F934F9387
:109670005F936F937F938F939F93AF93BF93EF937A
:10968000FF938FE298E073DBFF91EF91BF91AF9171
:109690009F918F917F916F915F914F913F912F910A
:1096A0000F900BBE0F900FBE0F901F9018951F923A
:1096B0000F920FB60F9211240BB60F922F933F9378
:1096C0004F935F936F937F938F939F93AF93BF93CA
:1096D000EF93FF938FE298E0DFDAFF91EF91BF9174
:1096E000AF919F918F917F916F915F914F913F913A
:1096F0002F910F900BBE0F900FBE0F901F901895DB
:109700001F920F920FB60F9211240BB60F922F9348
:109710003F934F935F936F937F938F939F93AF93F9
:10972000BF93EF93FF938CEC98E021DBFF91EF91D7
:10973000BF91AF919F918F917F916F915F914F9169
:109740003F912F910F900BBE0F900FBE0F901F9067
:1097500018951F920F920FB60F9211240BB60F920D
:109760002F933F934F935F936F937F938F939F9329
:10977000AF93BF93EF93FF938CEC98E08DDAFF915A
:10978000EF91BF91AF919F918F917F916F915F9179
:109790004F913F912F910F900BBE0F900FBE0F90E6
:1097A0001F901895CF93DF93EC01E881F981028433
:1097B000F385E02D1995EA89FB8980818F7E80836E
:1097C000EA89FB898081877F8083EA89FB898081A0
:1097D0008F778083EA89FB8980818F7D80838A8D62
:1097E000898FDF91CF910895CF92DF92EF92FF9210
:1097F0001F93CF93DF93EC016A017B01122FE8895D
:10980000F98982E080834115514E61057105B1F0FF
:1098100060E079E08DE390E0A70196010E94A7B592
:10982000DA01C9010197A109B109B695A7959795E4
:109830008795AC01411580E15807A8F0E889F989BE
:10984000108260E874E88EE190E0A70196010E9422
:10985000A7B5BA01A901415051096109710976956D
:10986000679557954795EC85FD855083EE85FF8577
:109870004083188EEC89FD891083EA89FB898081F9
:1098800080618083EA89FB89808188608083EA899E
:10989000FB89808180688083EA89FB8980818F7D54
:1098A0008083DF91CF911F91FF90EF90DF90CF9059
:1098B0000895CF93DF93282F30E0F901E459FD4E4E
:1098C0008491F901EA5DFD4ED491F901E052FE4E1A
:1098D000C491CC2389F08111FBDAEC2FF0E0EE0F7C
:1098E000FF1FEA53FE4EA591B491EC91ED2381E068
:1098F00090E021F480E002C080E090E0DF91CF9121
:1099000008951F93CF93DF93282F30E0F901E45996
:10991000FD4E8491F901EA5DFD4ED491F901E052CA
:10992000FE4EC491CC23C1F0162F8111D1DAEC2F59
:10993000F0E0EE0FFF1FE455FE4EA591B4918FB7F6
:10994000F894111105C09C91ED2FE095E92302C018
:10995000EC91ED2BEC938FBFDF91CF911F91089588
:10996000CF93DF9390E0FC01EA5DFD4E2491FC0172
:10997000E052FE4E8491882361F190E0880F991F98
:10998000FC01EE56FE4EC591D491FC01E455FE4E0D
:10999000A591B491611109C09FB7F8948881209571
:1099A00082238883EC912E230BC0623061F49FB731
:1099B000F8943881822F809583238883EC912E2B15
:1099C0002C939FBF06C08FB7F894E8812E2B288375
:1099D0008FBFDF91CF9108951F93CF93DF93182FFF
:1099E000EB0161E0BDDF209711F460E004C0CF3FE0
:1099F000D10531F461E0812FDF91CF911F9181CFAB
:109A0000E12FF0E0E459FD4EE4914E2F50E0FA01D1
:109A10003197E231F10508F09DC08827EA5AFE4FE0
:109A20008F4F0C9418B084B5806884BDC7BD97C0B3
:109A300084B5806284BDC8BD92C08091800080687A
:109A400080938000D0938900C093880088C0809163
:109A50008000806280938000D0938B00C0938A0046
:109A60007EC080918000886080938000D0938D00BC
:109A7000C0938C0074C08091B00080688093B00067
:109A8000C093B3006CC08091B00080628093B0003E
:109A9000C093B40064C0809190008068809390006F
:109AA000D0939900C09398005AC080919000806232
:109AB00080939000D0939B00C0939A0050C08091F7
:109AC0009000886080939000D0939D00C0939C008C
:109AD00046C08091A00080688093A0008091A00083
:109AE0008F7B8093A000D093A900C093A80037C0BB
:109AF0008091A00080628093A000D093AB00C093BF
:109B0000AA002DC08091A00088608093A000D0930F
:109B1000AD00C093AC0023C0809120018068809389
:109B20002001D0932901C093280119C08091200100
:109B3000806280932001D0932B01C0932A010FC033
:109B400080912001886080932001D0932D01C093E3
:109B50002C0105C0C038D1050CF04CCF46CFDF91A9
:109B6000CF911F910895863308F0865390917B0022
:109B7000282F2870977F922B90937B0087708064AA
:109B800080937C0080917A00806480937A00809139
:109B90007A0086FDFCCF809178002091790090E0DA
:109BA000922B08958F929F92AF92BF92CF92DF92A5
:109BB000EF92FF926B017C010E94AE6D4B015C0144
:109BC000C114D104E104F104F1F00E94AE6DDC0196
:109BD000CB0188199909AA09BB09883E9340A105C0
:109BE000B10570F321E0C21AD108E108F10888EE4E
:109BF000880E83E0981EA11CB11CC114D104E1049D
:109C0000F10419F7DDCFFF90EF90DF90CF90BF9078
:109C1000AF909F908F9008950895089508950895A6
:109C2000CF93DF93EC018091C60D811109C06A8D3D
:109C30007B8DCE0149960E94807681E08093C60D8F
:109C400021E83FEF3B872A878FE790E09D878C874D
:109C50001F861E86398B288B9B8B8A8B1D8A1C8ABC
:109C6000DF91CF9108950F931F93CF93DF93EC0172
:109C70001F8A1E8A8C01075E1F4F40E060E0C8010A
:109C80000E94EC8340E064E0C8010E94EC830E94E3
:109C9000D36D6C8F7D8F8E8F9F8FDF91CF911F91B2
:109CA0000F9108950F931F93CF93DF93EC01809151
:109CB000C50D811112C00A8D1B8D6AEA70E0C801C2
:109CC0000E94A36AD801ED91FC910284F385E02DF6
:109CD000C801199581E08093C50D4AE06EE0CE0180
:109CE00049960E94EC8321E83FEF3B872A878FE764
:109CF00090E09D878C871F861E86398B288B9B8BD7
:109D00008A8B1D8A1C8ADF91CF911F910F91089534
:109D10000F931F93CF93DF93EC011F8A1E8A8C0150
:109D2000075E1F4F40E060E0C8010E94AF8340E043
:109D300064E0C8010E94AF830E94D36D6C8F7D8F59
:109D40008E8F9F8FDF91CF911F910F9108950F9369
:109D50001F93CF93DF93EC01E8A1F9A1808191815A
:109D6000A281B3818E01075E1F4F81159649A1051F
:109D7000B10509F44FC040E056E960E070E082E9C7
:109D800097E00E94C06564E170E080E090E00ADF47
:109D9000E8A1F9A180819181A281B38181152BE491
:109DA0009207A105B105E9F068F4803629E0920731
:109DB000A105B105A1F080389542A105B105C1F416
:109DC00042E012C0811521EE9207A105B10559F0BC
:109DD0008115924CA140B10559F445E005C041E020
:109DE00003C043E001C046E06FE0C8010E94AF83BA
:109DF00082E997E023D8E8A1F9A1408151816281ED
:109E0000738182E997E00E94C06564E170E080E0C0
:109E100090E0C8DE4AE06EE0C8010E94AF8341E0F6
:109E200067E1C8010E94AF834AA168E1C8010E94AE
:109E3000AF8321E83FEF3B872A878FE790E09D873C
:109E40008C871F861E86398B288B9B8B8A8B1D8A5D
:109E50001C8ADF91CF911F910F9108950C94AA6AEB
:109E6000EF92FF920F931F93CF93DF93EC01662342
:109E7000E1F0262F653608F024E60A891B89E88878
:109E8000F988D801AE19BF0930E00E9426B028EC4D
:109E900030E040E050E00E94A7B5E20EF31EFB86E2
:109EA000EA86021B130B1D870C87DF91CF911F9150
:109EB0000F91FF90EF900895CF93DF93CDB7DEB76A
:109EC000A2970FB6F894DEBF0FBECDBF80310CF065
:109ED00080E121E733E13A83298329E633E13C83BA
:109EE0002B8321E633E13E832D8329E533E1388757
:109EF0002F8321E533E13A87298729E433E13C8741
:109F00002B8721E433E13E872D8729E333E1388B2A
:109F10002F872BE233E13A8B298B29E133E13C8B0C
:109F20002B8B2CEF32E13E8B2D8B27EE32E1388FDD
:109F30002F8B2DED32E13A8F298F23ED32E13C8FCB
:109F40002B8F26EC32E13E8F2D8F2AEB32E138A3A6
:109F50002F8F22EB32E13AA329A3E82FEE0FFF0B5C
:109F6000EC0FFD1F81819281A2960FB6F894DEBF9F
:109F70000FBECDBFDF91CF9108958F929F92AF9288
:109F8000BF92CF92DF92EF92FF920F931F93DC016B
:109F900018968D919C9119971E96CD90DC901F97E5
:109FA0006817790709F456C05896FC9058974C01E9
:109FB000092E000CAA08BB088B01072E000C220BEF
:109FC000330B861797073CF41696ED91FC91179783
:109FD000FF2039F015C01496ED91FC911597FF20E4
:109FE00079F00D2C000CEE08FF08A9019801281942
:109FF00039094A095B091C966D917C911D970EC029
:10A000000D2C000CEE08FF08A90198012819390948
:10A010004A095B091A966D917C911B97CB01770FCA
:10A02000AA0BBB0BBC01CD016C197D098E099F09E0
:10A030000E94E2AF8F01FF0F220B330BA9019801A1
:10A04000281939094A095B090E947BB5C20ED31E43
:10A05000E41EF51EC6011F910F91FF90EF90DF9057
:10A06000CF90BF90AF909F908F900895EF92FF9206
:10A070000F931F93CF93DF938C01FC01778B668B3B
:10A080007CDFEC01F801828193818830910531F504
:10A090007801F9E1EF0EF11CD7FF06C06AE0C13884
:10A0A0008FEFD80754F001C068E02C2F9D2FC038E7
:10A0B000D1052CF02FE790E002C021E89FEF422F5E
:10A0C000592F57FF03C0519541955109C7010E946F
:10A0D000088FCD2B69F54FE766E027C0099741F55A
:10A0E0007801E9E1EE0EF11CD7FF06C06EE0C13841
:10A0F000FFEFDF0754F001C06CE02C2F9D2FC0381C
:10A10000D1052CF02FE790E002C021E89FEF422F0D
:10A11000592F57FF03C0519541955109C7010E941E
:10A12000088FCD2B29F44FE767E0C7010E94088F05
:10A130000E94D36DF801648F758F868F978FDF91A2
:10A14000CF911F910F91FF90EF900895CF93DF93E0
:10A15000EC017F8B6E8B11DF9C018A819B818830A3
:10A160009105C1F437FF06C061E021388FEF380751
:10A170004CF001C060E0A901203831052CF04FE718
:10A1800050E002C041E85FEF57FF1FC05195419575
:10A1900051091BC00997E9F4922F832F203831050C
:10A1A00014F09FE780E0492F582F41388FEF580770
:10A1B00014F441E85FEF57FF03C0519541955109F1
:10A1C000632F661F6627661F6C5FCE0149960E944B
:10A1D000EC830E94D36D6C8F7D8F8E8F9F8FDF916C
:10A1E000CF9108950F931F93CF93DF93EC010E94BB
:10A1F000D36D0C8D1D8D2E8D3F8DDC01CB01801B11
:10A20000910BA20BB30B853F9140A105B10540F026
:10A210006E897F89CE01DF91CF911F910F9196CFEB
:10A22000DF91CF911F910F910895CF93DF93EC01B0
:10A230007F8B6E8BA2DE9C018A819B818830910589
:10A24000C1F437FF06C061E021388FEF38074CF0CA
:10A2500001C060E0A901203831052CF04FE750E043
:10A2600002C041E85FEF57FF1FC05195419551096A
:10A270001BC00997E9F4922F832F2038310514F081
:10A280009FE780E0492F582F41388FEF580714F48B
:10A2900041E85FEF57FF03C0519541955109632F86
:10A2A000661F6627661F6C5FCE0149960E94AF83CA
:10A2B0000E94D36D6C8F7D8F8E8F9F8FDF91CF919A
:10A2C00008950F931F93CF93DF93EC010E94D36DFA
:10A2D0000C8D1D8D2E8D3F8DDC01CB01801B910BD4
:10A2E000A20BB30B853F9140A105B10540F06E89EB
:10A2F0007F89CE01DF91CF911F910F9196CFDF9192
:10A30000CF911F910F910895CF93DF93EC0161E0FE
:10A3100089E026DB60E089E0F4DA1092D60980E17A
:10A3200095E099838883DF91CF910895CF92DF9252
:10A33000EF92FF928091D709833009F061C080913C
:10A34000D8098130D1F488EE93E0A0E0B0E08093AA
:10A35000690990936A09A0936B09B0936C0980E72F
:10A3600097E1A0E0B0E080936D0990936E09A0930F
:10A370006F09B093700932E001C030E0E091D80974
:10A38000F0E0E752F64F2081A0E1A30F48EE53E042
:10A3900060E070E088EBC82E8BE0D82EE12CF12C29
:10A3A000832F90E0FC01EE0FFF1FEE0FFF1FE75918
:10A3B000F64F27FF10C0C082D182E282F382880F5D
:10A3C000991F880F991FFC01E359F64F4083518371
:10A3D000628373830FC04083518362837383880FCA
:10A3E000991F880F991FFC01E359F64FC082D18253
:10A3F000E282F3823E5F220F3A13D2CF3093D2092A
:10A40000FF90EF90DF90CF900895CF93DF938091EE
:10A41000D609811151C01092D4091092D109C1E01E
:10A42000C093D609D091D50961E089E099DA60E05E
:10A4300089E067DA2D2F30E040E050E060E47FE112
:10A4400080E090E00E947BB5C093B00089E08093EB
:10A45000B1002093B3008BEA289F212D112426956B
:10A460002093B40080916F008B7F80936F00809168
:10A47000B00080628093B00020918400309185000C
:10A48000E091D10981E08E0F8093D10984E0E89FAB
:10A49000F0011124E759F64F80819181A281B381A7
:10A4A000820F931F90938B0080938A00B29A8091C1
:10A4B0006F00846080936F00DF91CF9108954F9279
:10A4C0005F926F927F928F929F92AF92BF92CF9244
:10A4D000DF92EF92FF928AE18093D2092093D30911
:10A4E00088E28093D50981E08093D8098093D909C7
:10A4F0008EE08093D70980EC92E1A0E0B0E08093F9
:10A50000690990936A09A0936B09B0936C0980EB79
:10A5100094E0A0E0B0E080936D0990936E09A09361
:10A520006F09B0937009A4E1440F551F661F771F90
:10A53000AA95D1F722E030E0B0EBCB2EB4E0DB2ED1
:10A54000E12CF12C80E6482E89E0582E612C712CEC
:10A5500090E4892E9CE9992EA12CB12CC901880F79
:10A56000991F880F991FFC01E759F64F77FF05C027
:10A57000408251826282738204C0C082D182E282B0
:10A58000F382C9010196880F991F880F991FFC015A
:10A59000E759F64F283129F0C082D182E282F38256
:10A5A00004C080829182A282B382440F551F661F2D
:10A5B000771F2E5F3F4F2A31310581F6FF90EF90D4
:10A5C000DF90CF90BF90AF909F908F907F906F90D3
:10A5D0005F904F901ACF8F929F92AF92BF92CF927F
:10A5E000DF92EF92FF9282E18093D20986E080931E
:10A5F000D30996E29093D50991E09093D80990936E
:10A60000D9098093D70988ED90E4A0E0B0E0809369
:10A61000690990936A09A0936B09B0936C098CE166
:10A620009CE0A0E0B0E080936D0990936E09A09348
:10A630006F09B0937009742F66275527442722E0CD
:10A6400030E0ACE1CA2EACE0DA2EE12CF12CB8E31C
:10A650008B2EB8E19B2EA12CB12CC901880F991F1C
:10A66000880F991FFC01E759F64F77FF05C08082DC
:10A670009182A282B38204C0C082D182E282F3823C
:10A68000F901EE0FFF1FEE0FFF1FE359F64FC082D7
:10A69000D182E282F382440F551F661F771F2E5F1F
:10A6A0003F4F22313105C9F68CE199E8A0E0B0E0D6
:10A6B0008093AD099093AE09A093AF09B093B00910
:10A6C000FF90EF90DF90CF90BF90AF909F908F90D2
:10A6D0009CCE80918C0690918D06DC01ED91FC91D1
:10A6E0000084F185E02D199580918C0690918D065E
:10A6F000DC01ED91FC910480F581E02D19948091AD
:10A70000070180FF11C060E08EE3FBD8109229069C
:10A7100080919206882341F06DE275E18091900668
:10A72000909191060C947A4A08958091070180FFD8
:10A7300012C061E08EE3E5D881E080932906809124
:10A740009206882341F067E175E18091900690912F
:10A7500091060C947A4A08958091070181FF11C0F7
:10A7600060E08FE3CED81092220680919206882373
:10A7700041F060E075E180919006909191060C9413
:10A780007A4A08958091070181FF12C061E08FE34A
:10A79000B8D881E08093220680919206882341F008
:10A7A0006AEE74E180919006909191060C947A4A39
:10A7B00008958091EF05882371F01092EF05809144
:10A7C0009206882341F062E674E1809190069091B0
:10A7D00091060C947A4A08958091E40F833099F0A1
:10A7E0008091EF0581110FC081E08093EF0580918A
:10A7F0009206882341F06DE474E180919006909177
:10A8000091060C947A4A08958091EF05882319F0F7
:10A8100080E090E0CECF80E090E0DECF8091EE054A
:10A82000833079F083E08093EE058091920688234F
:10A8300041F06CE374E180919006909191060C9444
:10A840007A4A08958091EE05823079F082E0809313
:10A85000EE0580919206882341F06BE274E18091CD
:10A860009006909191060C947A4A08958091EE0595
:10A87000813079F081E08093EE0580919206882303
:10A8800041F06AE174E180919006909191060C94F8
:10A890007A4A08950E94427E8091F005882361F1F2
:10A8A0008091C50A811128C080918806811124C039
:10A8B00081E0809388060E94AF4580911B06882323
:10A8C00019F010921B060CC080918C0690918D0699
:10A8D000DC01ED91FC910088F189E02D61E0199592
:10A8E00080919206882341F06FEE73E1809190068B
:10A8F000909191060C947A4A089561E085E301D81D
:10A9000080918C0690918D06DC01ED91FC9106A85A
:10A91000F7A9E02D199580919206882341F06CE704
:10A9200075E180919006909191060C947A4A089571
:10A930008F929F92AF92BF92CF92DF92EF92FF924F
:10A9400085E411D9BC01990F880B990B0E9438B48A
:10A9500020E030E040E85AE30E9497B420E030E085
:10A9600040EA50E40E9497B46B017C0180910C0294
:10A97000882351F0C092CD0DD092CE0DE092CF0D34
:10A98000F092D00D10920C0226E636E646E65FE322
:10A990006091CD0D7091CE0D8091CF0D9091D00D25
:10A9A0000E9497B44B015C0120ED3CEC4CEC5DE364
:10A9B000C701B6010E9497B49B01AC01C501B40167
:10A9C0000E942DB06093CD0D7093CE0D8093CF0D6E
:10A9D0009093D00D2DE33CE248E450E40E9497B4FC
:10A9E0002AE939E949E95EE30E942DB0FF90EF9032
:10A9F000DF90CF90BF90AF909F908F900895CF93AE
:10AA0000DF938091070180FD28C0C0912606D09178
:10AA1000270680912B06882369F08EE3A4D8813025
:10AA200092402CF0109227061092260609C081E071
:10AA300090E002C08EE397D8909327068093260675
:10AA400080912606909127068C179D0719F4109285
:10AA5000280603C081E080932806DF91CF910895F6
:10AA6000CF93DF938091070181FD28C0C0911F061D
:10AA7000D091200680912406882369F08FE373D853
:10AA8000813092402CF01092200610921F0609C0CF
:10AA900081E090E002C08FE366D890932006809317
:10AAA0001F0680911F06909120068C179D0719F4B0
:10AAB0001092210603C081E080932106DF91CF919F
:10AAC0000895909192068823D9F08091EF0688230B
:10AAD000B9F081E08093F60F8093CA0D992311F1AC
:10AAE00069EB74E180919006909191060E9409496A
:10AAF0000E94E89280919006909191060C94674A8A
:10AB00001092F60F992341F061ED74E18091900667
:10AB1000909191060E947A4A8091F40F811102C0AF
:10AB20001092CA0D0895909192068823F9F08091B1
:10AB3000EF068823D9F08091A50F8D30B9F481E01C
:10AB40008093F40F8093CA0D992311F168E774E1A3
:10AB500080919006909191060E9409490E94169357
:10AB600080919006909191060C94674A1092F40F90
:10AB7000992341F068E974E18091900690919106E3
:10AB80000E947A4A8091F60F811102C01092CA0D7C
:10AB900008958091E40F833041F12CF48130A9F0C5
:10ABA000823099F02DC086305CF5809181069091BD
:10ABB0008206DC01ED91FC910480F581E02D199570
:10ABC00080917F069091800614C0809185069091B7
:10ABD0008606DC01ED91FC910480F581E02D19954C
:10ABE000809183069091840604C0809181069091A3
:10ABF0008206DC01ED91FC910480F581E02D199530
:10AC000080918C0690918D06DC01ED91FC91EA5BC0
:10AC1000FF4F0190F081E02D199580918C06909165
:10AC20008D06DC01ED91FC910284F385E02D60E05E
:10AC300070E019940E94427E8091F0058823D1F043
:10AC4000809188068823B1F0109288060E947D4585
:10AC500080911B06882389F010921B068091920632
:10AC6000882341F063E074E1809190069091910611
:10AC70000E947A4A10928806089580918C069091DD
:10AC80008D06DC01ED91FC910088F189E02D60E0FA
:10AC90001995E4CFCF93DF93C091CB0DD091CC0D1C
:10ACA000BE0180EF9AE00E940F80882329F0BE0148
:10ACB00080EF9AE00E9427801092CC0D1092CB0D6D
:10ACC000DF91CF9108950F931F93CF93DF938091DE
:10ACD000E90F9091EA0FA091EB0FB091EC0F1816CD
:10ACE00019061A061B060CF044C00E94427E809191
:10ACF000F0058823C9F10091CB0D1091CC0DB8015E
:10AD000080EF9AE00E940F808823D9F0EEEEFCE0FD
:10AD1000C0E0D0E0819191918017910769F40E9481
:10AD2000D36DCC0FDD1FCC0FDD1FC051D54F688315
:10AD300079838A839B831DC02196CE31D10551F73B
:10AD400018C04091E90F5091EA0F6091EB0F70919C
:10AD5000EC0F2CE937E580EF9AE00E947680909323
:10AD6000CC0D8093CB0D05C0DF91CF911F910F913A
:10AD700091CFDF91CF911F910F9108958091C50AD6
:10AD800081113FC00E94427E809143128823B1F01E
:10AD90008091F005882391F01092F00510924312F3
:10ADA0000E94697E8091C90D882341F06AEC73E1AD
:10ADB0008091C70D9091C80D0E947A4A80918806B3
:10ADC000882311F081E001C080E00E94E14581E02C
:10ADD00080931B062FDF8091FA0F81110FC08091A5
:10ADE0000606882359F029E633E544E650E060E0A2
:10ADF00070E080EF9AE00E94768001C06ADCC9DED4
:10AE000062CF0895C6DE0E94E96F0E94427E809163
:10AE1000F0058111B3DF80918E0690918F06DC01E1
:10AE2000ED91FC910480F581E02D199580918A06C1
:10AE300090918B06DC01ED91FC910480F581E02D71
:10AE400019958091C50F882359F08091070690913C
:10AE50000806DC01ED91FC910480F581E02D199448
:10AE6000089580910B02882351F062DD20E030E0EC
:10AE700040E050E40E9432B487FF39C0089558DDA5
:10AE800020E030E04AE754E40E9497B40E94FEB00C
:10AE9000209143103091441040919506621773073A
:10AEA00010F4442351F1442309F445C041DD20E06E
:10AEB00030E04AE754E40E9497B40E94FEB020912B
:10AEC00043103091441062177307A8F11092950651
:10AED00081E08093940680919206882361F164E476
:10AEE00075E180919006909191060C947A4A1092A7
:10AEF0000B0281E080939406089581E0809395068B
:10AF00001092940680919206882391F063E675E191
:10AF100080919006909191060E9409490E94187FA5
:10AF200060E675E180919006909191060E947A4AC0
:10AF300069DF0C942C8608950E94427E8091F00572
:10AF4000882369F01BDF80919206882341F06AED27
:10AF500073E180919006909191060C947A4A08953D
:10AF60008091C50A811155C080918906823068F0B0
:10AF700080919206882309F44CC068E873E18091BF
:10AF80009006909191060C947A4A0E94427E80919C
:10AF90004312882309F43DC08091F005811139C026
:10AFA00081E08093F005109243120E94697E8091A7
:10AFB000C90D882341F069E773E18091C70D909135
:10AFC000C80D0E947A4A80918C0690918D06DC0112
:10AFD000ED91FC910280F381E02D19958091890615
:10AFE000811116C04091DF0F5091E00F81E08093F6
:10AFF0001B064115510559F060E070E02AE434E584
:10B0000080EF9AE00E9476800E947D4501C042DC7C
:10B010005ACE08952F923F924F925F926F927F92F5
:10B020008F929F92AF92BF92CF92DF92EF92FF9258
:10B030000F931F93CF93DF9300D01F92CDB7DEB74E
:10B040005C01E0DE0E94C0870E94F7878091900635
:10B05000909191060E94674A0E94773A24E0A216D6
:10B06000B10409F49CC00CF04FC0A3E0AA16B104CF
:10B0700009F03CC18CE190E00E9432B19C838B834B
:10B0800086EC95E0AB81BC8111969C938E931396D0
:10B09000BC92AE92129781E09FEF15969C938E938F
:10B0A00014978FEF90E017969C938E9316971996AE
:10B0B0001C921E92189758961C925897CD010E9488
:10B0C00031838AEB95E0EB81FC8191838083E09171
:10B0D000B80DF091B90DD08C0091BF111091C01135
:10B0E00016950795E090BD11F090BE11F694E79487
:10B0F0006BE676E180919006909191060E947A4AE3
:10B10000812C9924939412C1B5E0AB16B10409F4D3
:10B11000A6C0E6E0AE16B10409F0E8C08CE190E00C
:10B120000E9432B19C838B8386EC95E0AB81BC811D
:10B1300011969C938E931396BC92AE92129781E0D7
:10B140009FEF15969C938E9314978FEF90E0179630
:10B150009C938E93169719961C921E921897589648
:10B160001C925897CD010E9431838AEB95E0EB81C8
:10B17000FC8191838083E0917C06F0917D06D08CE8
:10B180000091FE111091FF1116950795E090FC11AA
:10B19000F090FD11F694E7946EE976E1A0C08CE1A1
:10B1A00090E00E9432B19C838B8386EC95E0AB816A
:10B1B000BC8111969C938E931396BC92AE9212977B
:10B1C00081E09FEF15969C938E9314978FEF90E0FC
:10B1D00017969C938E93169719961C921E92189709
:10B1E00058961C925897CD010E9431838AEB95E0C6
:10B1F000EB81FC81918380830091D4111091D51152
:10B2000016950795E090D211F090D311F694E7943B
:10B210008091A50F8C50823040F4E0918E06F09121
:10B220008F06D08C6EED76E15AC08091E40F8230AB
:10B2300009F07AC08091A30F8C3009F075C0E091BD
:10B240007C06F0917D06D08C6EEB76E180919006C5
:10B25000909191060E947A4A8824839466C08CE17A
:10B2600090E00E9432B19C838B8386EC95E0AB81A9
:10B27000BC8111969C938E931396BC92AE921297BA
:10B2800081E09FEF15969C938E9314978FEF90E03B
:10B2900017969C938E93169719961C921E92189748
:10B2A00058961C925897CD010E9431838AEB95E005
:10B2B000EB81FC8191838083E0918A06F0918B067B
:10B2C000D08C0091E9111091EA1116950795E09044
:10B2D000E711F090E811F694E7946EE776E180913B
:10B2E0009006909191060E947A4A1EC062E576E12E
:10B2F00080919006909191060F900F900F900F9073
:10B30000DF91CF911F910F91FF90EF90DF90CF9041
:10B31000BF90AF909F908F907F906F905F904F9075
:10B320003F902F900C947A4A812C912C0E94773A6E
:10B3300065E476E180919006909191060E947A4AA8
:10B3400069E376E180919006909191060E94094907
:10B35000B80180919006909191060E949B776DE2D2
:10B3600076E180919006909191060E940949B7017B
:10B3700080919006909191060E949B7761E276E120
:10B3800080919006909191060E9409498D2D0E940E
:10B39000533A80919006909191060E94674AAB8142
:10B3A000BC81ED91FC9111970280F381E02DCD01DC
:10B3B0001995CA2C8A2D0E944E828D3D9540A8F485
:10B3C00064E378E08A2D0E944682EB81FC81F78A53
:10B3D000E68AB70182810E945E826CED75E08A2D5B
:10B3E0000E944A82DD20C1F01AC064E873E08A2D11
:10B3F0000E944A82AB81BC8157961C930E9356974C
:10B40000B80112968C910E945E826CED75E08A2DD7
:10B410000E944682DD2019F03324339401C0312C80
:10B4200021E02983212C2A830E940F3C80916811FE
:10B43000882359F1AB81BC81ED91FC91119760910A
:10B440006D1170916E110190F081E02DCD01199573
:10B450008C2D0E944E828D3DB5E09B075CF48438B4
:10B46000E3E09E0784F08C018D3D954074F00CED77
:10B4700015E00BC07C01853398403CF064E3E62E78
:10B4800068E0F62E02C004E813E02A8121111FC0F3
:10B4900080915E118823C9F1E0916511F0916611E8
:10B4A0008581968140916111509162119C012153D7
:10B4B0003109421753074CF1C196841795072CF1B7
:10B4C0000E94D36D6415750586059705F0F080918F
:10B4D0005E118823C1F04091611150916211E09199
:10B4E0006511F0916611858196819C01285C310976
:10B4F000421753072CF088539F4F841795071CF46D
:10B5000081E0382605C021E02A83222009F47CC08E
:10B51000332009F445C0DD20F9F064E873E08C2D98
:10B520000E944A82992009F458C06091BF0F70911F
:10B53000C00F41E08C2D0E9405820E948D91AB814D
:10B54000BC8112968C910E944E8208171907ACF3A9
:10B550008C2D0E94D78141C064E378E08C2D0E943D
:10B5600046829920B1F06091BF0F7091C00F40E00A
:10B570008C2D0E9405820E948D91AB81BC81129618
:10B580008C910E944E828E159F05ACF38C2D0E94EB
:10B59000D781EB81FC81F78AE68AB701828110C0EE
:10B5A000DD20B1F064E378E08C2D0E944682AB810F
:10B5B000BC815796FC92EE925697B70112968C91E9
:10B5C0000E945E826CED75E08C2D0E944A8212C052
:10B5D00064E873E08C2D0E944A82EB81FC81178B1A
:10B5E000068BB80182810E945E826CED75E08C2D25
:10B5F0000E9446820E94D36D2B013C01F8EC4F0E55
:10B60000511C611C711C1A8229812223D9F180915D
:10B6100054118823A9F14091571150915811E0918C
:10B620005B11F0915C11858196819C01285C310948
:10B63000421753072CF088539F4F8417950704F542
:10B6400081E0D8268091900690919106DD2039F016
:10B6500062E176E10E947A4A82E090E006C060E012
:10B6600076E10E947A4A81E090E00E94C8870E94B9
:10B67000D36DAB81BC815896DC922224239403C005
:10B68000212C1EC0212C80915411882309F472C2F0
:10B69000E0915B11F0915C11858196814091571189
:10B6A000509158119C0121533109421753070CF452
:10B6B00061C2C19621E02983841795070CF45AC210
:10B6C0000E9431850E94DC7680EF9AE00E9486809D
:10B6D0008091DF0A882309F4A7CE8091E10A8823AC
:10B6E00009F4A2CE0E94DC760E94B8898823D1F3A7
:10B6F00084E0A816B104D9F134F4B3E0AB16B10478
:10B7000009F438C1C4C1E5E0AE16B10409F4CDC0F6
:10B71000F6E0AF16B10409F0BAC11093B30F00936D
:10B72000B20FF092B50FE092B40FD092B60FB801FD
:10B7300088E291E00E944276B7018AE291E00E949D
:10B7400042766D2D8CE291E00E94D077B80186E0C0
:10B750000E947C81B70186E00E946181E0917C06B5
:10B76000F0917D06D08E6CED75E086E091C088206A
:10B77000C1F01093B30F0093B20FF092B50FE092A7
:10B78000B40FD092B60FB80188E291E00E944276E1
:10B79000B7018AE291E00E9442766D2D8CE291E041
:10B7A00017C01093A70F0093A60FF092A90FE09275
:10B7B000A80FD092AA0FB8018CE191E00E944276C6
:10B7C000B7018EE191E00E9442766D2D80E291E01A
:10B7D0000E94D077B80184E00E947C81B70184E0A8
:10B7E0000E946181882049F0E0917C06F0917D06FD
:10B7F000D08E6CED75E084E04BC0E0918E06F09148
:10B800008F06D08E8091A50F8D3029F4E091D10D57
:10B81000F091D20DD08E6CED75E084E00E945E82D6
:10B8200066E970E080E090E00E94D24D8091A50F23
:10B830008D3011F584E00E944E82A0918E06B09169
:10B840008F068D3D95404CF0ED91FC911197019044
:10B85000F081E02D6FEF7FEF08C0ED91FC91119723
:10B860000190F081E02D61E070E0CD0119958091AB
:10B870008E0690918F066FC080918E0690918F06F4
:10B88000DC01ED91FC910480F581E02D1995FFC05C
:10B890000E945E8266E970E080E090E00E94D24DF6
:10B8A00080917C0690917D06EBCF1093AE0F0093B4
:10B8B000AD0FF092B00FE092AF0FD092B10FB80180
:10B8C00083E291E00E944276B70185E291E00E9416
:10B8D00042766D2D87E291E00E94D077B80185E035
:10B8E0000E947C81B70185E00E946181E0918A0617
:10B8F000F0918B06D08E6CED75E085E00E945E8243
:10B9000066E970E080E090E00E94D24D8091A40F43
:10B910008D3059F585E00E944E82A0918A06B09143
:10B920008B068D3D95404CF0ED91FC911197019067
:10B93000F081E02D6FEF7FEF08C0ED91FC91119742
:10B940000190F081E02D61E070E0CD0119958091CA
:10B950008A0690918B06DC01ED91FC910190F081BB
:10B96000E02D60E070E0199592C080918A06909178
:10B970008B0686CF1093C20F0093C10FF092C40FB5
:10B98000E092C30FD092BB0FB80187E391E00E9411
:10B990004276B70189E391E00E9442766D2D81E302
:10B9A00091E00E94D077B80183E00E947C81B701CA
:10B9B00083E00E9461818091BB0FE091B80DF0910E
:10B9C000B90D808F8091BB0F0E940D7683E00E949D
:10B9D0004E822091BB0F222369F1B9E0BC1538F0EB
:10B9E0002091BF113091C0113695279502C02EEEDF
:10B9F00032E08217930709F44AC06091BF0F70913B
:10BA0000C00F41E083E00E9405820E948D91EB818E
:10BA1000FC8182810E944E8208171907B4F383E0EB
:10BA20000E94D781AB81BC8157961C930E93569789
:10BA3000B80129C029E02C1508F49EC02091BD1141
:10BA40003091BE11369527958217930701F16091C9
:10BA5000BF0F7091C00F40E083E00E9405820E94FA
:10BA60008D91EB81FC8182810E944E828E159F0513
:10BA7000B4F383E00E94D781AB81BC815796FC92DE
:10BA8000EE925697B70112968C910E945E82809139
:10BA90009006909191060E94674A0E94773AB4E01E
:10BAA000AB16B10459F0E5E0AE16B10451F0F3E085
:10BAB000AF16B10471F466EB75E105C066EE75E191
:10BAC00002C06DEC75E180919006909191060E9404
:10BAD0007A4A0E94773A6BEA75E1809190069091DC
:10BAE00091060E947A4A6FE975E1809190069091E3
:10BAF00091060E940949B8018091900690919106A3
:10BB00000E949B7763E975E1809190069091910680
:10BB10000E940949B70180919006909191060E9478
:10BB20009B7767E875E180919006909191060E945D
:10BB300009498D2D0E94533A80919006909191066B
:10BB40000E94674A0F900F900F900F90DF91CF9156
:10BB50001F910F91FF90EF90DF90CF90BF90AF902B
:10BB60009F908F907F906F905F904F903F902F901D
:10BB70000C94F3871982A4CD2AEC38E065CF80912C
:10BB8000DD0D9091DE0D91609093DE0D8093DD0DC3
:10BB900008958091DD0D9091DE0D80689093DE0D0B
:10BBA0008093DD0D08958091DD0D9091DE0D806113
:10BBB0009093DE0D8093DD0D0895FC018281882332
:10BBC00071F08381882359F013828091DD0D90916B
:10BBD000DE0D24E082279093DE0D8093DD0D089525
:10BBE000FC018281882371F0838181110BC081E087
:10BBF00083838091DD0D9091DE0D84609093DE0D46
:10BC00008093DD0D0895FC018481882371F0858186
:10BC1000882359F015828091DD0D9091DE0D28E08A
:10BC200082279093DE0D8093DD0D0895FC018481C1
:10BC3000882371F0858181110BC081E0858380911B
:10BC4000DD0D9091DE0D88609093DE0D8093DD0D0B
:10BC500008958091DD0D9091DE0D20E28227909372
:10BC6000DE0D8093DD0D08958091DD0D9091DE0D48
:10BC700080629093DE0D8093DD0D0895DC01ED91DF
:10BC8000FC910680F781E02D60E070E0199477FF69
:10BC900003C07195619571096F3F710519F014F03A
:10BCA0006FEF70E08091DD0D9091DE0D8C7B9170D7
:10BCB0009093DE0D8093DD0D8091DD0D9091DE0D72
:10BCC0006F30710514F480641FC06733710514F47C
:10BCD00081641AC06F3571051CF48164906114C0D1
:10BCE000673871051CF4816490630EC06F3A71056A
:10BCF0001CF48164906408C0673D71051CF4816484
:10BD0000906502C0816490669093DE0D8093DD0D96
:10BD1000089580E094E09093DE0D8093DD0D08950A
:10BD20008091DD0D9091DE0D92609093DE0D8093F9
:10BD3000DD0D8091DD0D9091DE0D80649093DE0D20
:10BD40008093DD0D08950895089508950895089548
:10BD50000895089508950895089580E00895089538
:10BD600008950895089508950895089508950895EB
:10BD700008950895089508950895089508950895DB
:10BD800080E0089508950895FC0164830895FC01FE
:10BD900062830895FC011382148215821682178231
:10BDA000108611860895089508950895FC018381F1
:10BDB0000895FC0165830895FC0164830895FC01E6
:10BDC00060870895FC0166830895FC0182810895CF
:10BDD0006CED75E080E00C949781FC011282138277
:10BDE0001482158261E086E10E94B04C61E086E138
:10BDF0000E94814CE2E7F0E08081816080831092B4
:10BE0000DE0D1092DD0D0895FF920F931F93CF93D7
:10BE1000DF938C01C62FF42ED22F6AED70E0DC0187
:10BE20001A968D919C911B970E94A36AF8018285B6
:10BE30009385DC01ED91FC910190F081E02D6C2F58
:10BE40001995F80182859385DC01ED91FC910190B3
:10BE5000F081E02D6F2D1995F80182859385DC0125
:10BE6000ED91FC910190F081E02D6D2F1995EC2F53
:10BE7000F0E0BF0166527F4F6F0D711D6D0F711D98
:10BE80006F777727F80182859385DF91CF911F9196
:10BE90000F91FF900C94A36A242F462F6CE4B4CF2B
:10BEA00077FF03C071956195710920E0462F6EE21E
:10BEB000ABCF462F20E067E4A7CF462F20E066E413
:10BEC000A3CF262F64E4A0CFCF92DF92FF920F93EF
:10BED0001F93CF93DF938C01F62E443F81E05807E8
:10BEE00038F0413187E2580728F040E157E202C0BC
:10BEF00044EF51E0243F81E0380738F0E901213177
:10BF0000374228F0C0E1D7E202C0C4EFD1E0CA0155
:10BF1000845F914022E3C22ED12CB6010E94F1AF82
:10BF2000462F2F2D62E4C8016FDFCE01845F914060
:10BF3000B6010E94F1AF462F2F2D63E4C801DF91B7
:10BF4000CF911F910F91FF90DF90CF905DCF262F63
:10BF500040E06FE359CF262F40E06EE355CF262F08
:10BF600040E06DE351CF462F20E06FE44DCF462FE8
:10BF700020E06DE449CFFC016283611104C020E040
:10BF800040E06BE441CF089577FF03C07195619560
:10BF9000710920E0462F6BE437CF1092600E25EB3D
:10BFA00030E744EF51E060E070E08091790E9091CD
:10BFB0007A0E0E9476809093D50D8093D40D0895CB
:10BFC0000F931F93CF93DF93EC0170937A0E6093DE
:10BFD000790E4093800E81E090E00E9432B18C0196
:10BFE0000E9431831093E00D0093DF0D91E0909358
:10BFF000600E9093610E1092D50D1092D40D109298
:10C00000640E1092630E1092650E1092620E24EF71
:10C0100031E030936C0E20936B0E28EB3BE03093B5
:10C020006E0E20936D0E20E233E03093730E20935A
:10C03000720E2CEA3DE03093750E2093740E28E0CA
:10C0400037E030937C0E20937B0E24E931E130936E
:10C050007E0E20937D0E1092680E1092670E109245
:10C06000660E10926F0E1092760E10927F0E109246
:10C07000D30D10926A0E1092690E1092710E1092EA
:10C08000700E1092780E1092770E988399839A838F
:10C09000DF91CF911F910F9108951F920F920FB6CC
:10C0A0000F9211240BB60F922F933F934F935F93F0
:10C0B0006F937F938F939F93AF93BF93EF93FF9370
:10C0C0008091DC0D8F5F8093DC0D9091DB0D8917E3
:10C0D00008F401C11092DC0D8091DA0D90E08730F8
:10C0E000910508F0F8C0FC018827E859FE4F8F4FF2
:10C0F0000C9418B060E086E10E94814C80E480934B
:10C10000DB0D81E048C061E086E10E94814C88E05F
:10C110008093DB0D36C060E086E10E94814C809107
:10C12000D80D9091D90D97FF05C088E18093DB0D64
:10C1300084E031C088E08093DB0D83E02CC061E0B7
:10C1400086E10E94814C88E18093DB0D8091D70DC0
:10C150008F5F8093D70D803150F01092D70D85E01E
:10C160001AC061E086E10E94814C88E0EDCF8091A9
:10C17000D80D9091D90D880F991F9093D90D809368
:10C18000D80D82E008C060E086E10E94814C88E022
:10C190008093DB0D86E08093DA0D9DC061E086E13F
:10C1A0000E94814C80EC8093DB0D8091DD0D90919D
:10C1B000DE0D9093D90D8093D80D8091DD0D909177
:10C1C000DE0D91FF1DC08091D60D8823B1F08091C6
:10C1D000DD0D9091DE0D22E092279093DE0D80938D
:10C1E000DD0D8091DD0D9091DE0D80649093DE0D6C
:10C1F0008093DD0D1092D60D03C081E08093D60DA3
:10C200008091DD0D9091DE0D92FF0EC08091D60DD4
:10C21000882339F01092DE0D1092DD0D1092D60DAC
:10C2200003C081E08093D60D8091DD0D9091DE0DED
:10C2300084FF14C08091D60D882369F08091DD0DB4
:10C240009091DE0D20E182279093DE0D8093DD0D2D
:10C250001092D60D03C081E08093D60D8091DD0D44
:10C260009091DE0D87FF13C08091D60D882361F079
:10C270008091DD0D9091DE0D80589093DE0D8093BE
:10C28000DD0D1092D60D03C081E08093D60D809114
:10C29000DD0D9091DE0D90FF14C08091D60D8823A6
:10C2A00069F08091DD0D9091DE0D21E09227909351
:10C2B000DE0D8093DD0D1092D60D03C081E08093DA
:10C2C000D60D8091DD0D9091DE0D9093D90D809368
:10C2D000D80D1092DA0DFF91EF91BF91AF919F9120
:10C2E0008F917F916F915F914F913F912F910F901F
:10C2F0000BBE0F900FBE0F901F90189520E040E0EE
:10C3000083CD65E4FBCF68E4F9CFCF93DF93FC01E5
:10C310002381222321F0EC0161E4F0DF1B82DF9115
:10C32000CF910895CF93DF93FC012381211105C0A4
:10C33000EC0160E4E3DF81E08B83DF91CF9108952E
:10C34000FC012581222311F060E5D8CF0895FC017E
:10C350002481222311F06CE3D1CF0895FC012085C4
:10C36000222331F02185222319F011866BE3C6CFF9
:10C370000895FC012085222339F02185211104C074
:10C3800021E021876AE3BACF0895FC0126812223A8
:10C3900031F02781222319F0178269E3AFCF089586
:10C3A000FC012681222339F02781211104C021E0DC
:10C3B000278368E3A3CF089567E3A0CF6AE49ECF05
:10C3C00069E49CCF66E39ACF65E398CF6EE496CF9D
:10C3D00064E394CF63E392CF62E390CF61E38ECFC7
:10C3E00060E38CCF6FE28ACF6DE288CF1092BF0AF4
:10C3F0000895CF93DF93C1E5DAE081E090E09A837E
:10C4000089831092BF0A0E94AE6D6C837D838E83F8
:10C410009F83E49AEC9ADF91CF9108951F920F9237
:10C420000FB60F9211240BB60F922F933F934F9399
:10C430005F936F937F938F939F93AF93BF93EF938C
:10C44000FF939091D1098091D209981317C010924F
:10C45000D1098091D8098F5F8093D8099091D8092C
:10C460008091D909891740F481E08093D80980919F
:10C47000D4098F5F8093D4090E9496519091D4097A
:10C480008091D30998130DC08091B0008F7D809367
:10C49000B00080916F008B7F80936F001092D6095F
:10C4A00027C08091B00085FF04C08091B0008F7DCF
:10C4B00003C08091B00080628093B000209184001E
:10C4C00030918500E091D10981E08E0F8093D109F0
:10C4D00084E0E89FF0011124E759F64F80819181B3
:10C4E000A281B381820F931F90938B0080938A0067
:10C4F000FF91EF91BF91AF919F918F917F916F913C
:10C500005F914F913F912F910F900BBE0F900FBEF7
:10C510000F901F9018951F920F920FB60F92112433
:10C520000BB60F921F932F933F934F935F936F938D
:10C530007F938F939F93AF93BF93EF93FF93CF938B
:10C54000DF9300D01F92CDB7DEB78091510A0E94D1
:10C55000594C11E0892B09F010E00E94AE6D6983FF
:10C560007A838B839C8389819A81AB81BC81409142
:10C57000550A5091560A6091570A7091580A841BC7
:10C58000950BA60BB70B2091520A3091530A243019
:10C59000310509F44CC02530310521F02130310539
:10C5A000E9F414C02091540A222339F02091BF0AE3
:10C5B00020FF02C0289A01C02898112379F0813EFB
:10C5C0002EE29207A105B10548F02BC0112379F1A5
:10C5D00025E030E03093530A2093520A2091520A0A
:10C5E0003091530A2530310511F5E091BF0AF0E092
:10C5F000EE0FFF1FE75AF54F9183808389819A815F
:10C60000AB81BC818093550A9093560AA093570A38
:10C61000B093580A8091BF0A8F5F8093BF0A83331B
:10C6200030F084E090E09093530A8093520A0F9088
:10C630000F900F900F90DF91CF91FF91EF91BF91ED
:10C64000AF919F918F917F916F915F914F913F91AA
:10C650002F911F910F900BBE0F900FBE0F901F9048
:10C66000189508950895089508950895623039F051
:10C67000633041F0613041F44093680E0895409377
:10C68000670E08954093660E0895623069F0633036
:10C69000A1F06130D1F450936C0E40936B0E309347
:10C6A0006E0E20936D0E08955093730E4093720E8C
:10C6B0003093750E2093740E089550937C0E409322
:10C6C0007B0E30937E0E20937D0E0895FC018581B4
:10C6D0000895089508952091800E211102C0FC0153
:10C6E000628308952091800E211102C0FC016483B1
:10C6F00008952091800E211102C0FC0163830895EA
:10C70000089508958091800E811102C00C94B57037
:10C710000895089580E0089508950895089508956E
:10C72000089508958091800E811104C08FE090E0FB
:10C730000C94B77108958091800E811121C06330EF
:10C7400091F028F4613049F0623051F0089565307D
:10C7500081F060F0663081F0089589E090E00EC0CD
:10C760008AE090E00BC08BE090E008C08CE090E0A5
:10C7700005C08DE090E002C08EE090E00C94B771AF
:10C7800008952091800E211108C0FC018481882326
:10C7900021F082E090E00C94B77108952091800E12
:10C7A000211108C0FC018381882321F081E090E001
:10C7B0000C94B77108958091800E811104C08BE0B4
:10C7C00090E00C94B77108958091800E811105C09E
:10C7D00060E080E190E00C94F57108958091800E06
:10C7E000811105C060E08FE090E00C94F571089530
:10C7F0008091800E811127C06330A1F028F4613050
:10C8000049F0623059F008956530A1F078F0663053
:10C81000A9F0089560E089E090E013C060E08AE04C
:10C8200090E00FC060E08BE090E00BC060E08CE037
:10C8300090E007C060E08DE090E003C060E08EE033
:10C8400090E00C94F57108958091800E811127C0BD
:10C850006330A1F028F4613049F0623059F0089556
:10C860006530A1F078F06630A9F0089561E089E0C4
:10C8700090E013C061E08AE090E00FC061E08BE0DF
:10C8800090E00BC061E08CE090E007C061E08DE0DB
:10C8900090E003C061E08EE090E00C94F5710895A3
:10C8A0002091800E211109C0FC018281882329F08A
:10C8B00061E088E090E00C94F57108952091800E7D
:10C8C000211109C0FC018481882329F061E082E004
:10C8D00090E00C94F57108952091800E211109C00B
:10C8E000FC018381882329F061E081E090E00C94D1
:10C8F000F57108958091800E811105C061E086E098
:10C9000090E00C94F57108958091800E811105C01E
:10C9100060E08BE090E00C94F57108958091800EBA
:10C92000811105C061E087E090E00C94F5710895F5
:10C930008091800E811105C061E085E090E00C944B
:10C94000F5710895CF93DF93FC0125812223A1F196
:10C95000EC018091800E81112EC06091690E709162
:10C960006A0E8091790E90917A0E0E942780109223
:10C970006F0E8091800E81110CC06091700E7091CD
:10C98000710E8091790E90917A0E0E9427801092FC
:10C99000760E8091800E81110CC06091770E70919F
:10C9A000780E8091790E90917A0E0E9427801092D5
:10C9B0007F0E1092D30D1D82DF91CF910895CF93FA
:10C9C000DF93FC01258121111EC0EC018091800EB6
:10C9D000811117C08091D30D811113C022E433E778
:10C9E00048EB5BE060E070E08091790E90917A0E08
:10C9F0000E94768090936A0E8093690E81E0809306
:10CA0000D30D81E08D83DF91CF9108958091800EC9
:10CA1000882329F06CED75E081E00C94978184E027
:10CA200090E00C94B7718091800E882329F068EE15
:10CA300073E081E00C94978160E084E090E00C94D6
:10CA4000F5718091800E81111BC08091600E88234A
:10CA5000B9F068EE73E081E00E9497811092600E59
:10CA600025EB30E748E95AE360E070E08091790E09
:10CA700090917A0E0E9476809093D50D8093D40D7C
:10CA800008956CED75E080E00C94978124EF31E01F
:10CA9000DB010E9426B02FEF30E040E050E00E9422
:10CAA0007BB5CA01B90164527A4F8F4F9F4F80E026
:10CAB0000C9497818091800E882331F060ED77E0AF
:10CAC00081E00E94978169CA61E083E090E00C9464
:10CAD000F5712091800E211103C002960C9473739E
:10CAE00008952091800E222389F06FE676E080E0A1
:10CAF0000E94978128EE3EE542E350E060E070E05E
:10CB00008091790E90917A0E0C94768002960C9416
:10CB1000737380E00E94BE8181E00E94BE8180919B
:10CB2000800E811103C082E00E94BE816CED75E031
:10CB300080E00E9497816CED75E081E00E94978112
:10CB40008091800E81110DC080E594E8A1E0BB27A3
:10CB5000ABBFFC016791769182E00E9497810C94B3
:10CB60009E700895FC0180899189938782878289CC
:10CB7000938995878487848995899787868708957F
:10CB800026E00C94F44B08950895FC018281938172
:10CB90008830910529F410922B0110922A010895F2
:10CBA000099721F410922901109228010895FC019F
:10CBB000178A168A6CED75E082810C945E82CF93A1
:10CBC000DF93EC011F8A1E8A8A810E94D7818B8D98
:10CBD000882331F08A810E944E829A8F898F1B8E22
:10CBE000DF91CF910895DF92EF92FF920F931F9301
:10CBF000CF93DF93EC018A81893010F40E94BE81CB
:10CC0000DD8C6B8D7C8D098D1A8DEA80FB8089E02F
:10CC10008E1508F466C00F30110538F001369DE618
:10CC2000190728F000E61DE602C00FE010E06F30A3
:10CC3000710538F061368DE6780728F060E67DE60C
:10CC400002C06FE070E080E090E00E9436B420E027
:10CC500030E04AE754E40E9491B020E030E04CE834
:10CC600052E40E9497B49B01AC0160E070E08AEF4F
:10CC700094E40E9491B00E94F9B0FF2425E12E9D1A
:10CC8000F0012F9DF00D1124E558FE4EDD2071F0CE
:10CC900023813481AB0177FF04C044275527461B0D
:10CCA000570B88279927841B950B0AC0258136814D
:10CCB000AB0177FF04C044275527461B570BCA0119
:10CCC0004FB7F89455E15E9DF0015F9DF00D112482
:10CCD000E558FE4E108B0787328B218B948B838B0C
:10CCE0004FBF9D8D6B8D7C8D8A819923F9F08A30A1
:10CCF00058F495E1899FF0011124E558FE4E058115
:10CD000016811695079502C00EEE12E041E00E94D2
:10CD1000058261E070E080E090E00E94D24D8A815F
:10CD20000E944E8208171907A0F31EC08A3058F4DB
:10CD300095E1899FF0011124E558FE4E038114818D
:10CD40001695079502C00AEC18E040E00E940582A3
:10CD500061E070E080E090E00E94D24D8A810E9404
:10CD60004E8280179107A0F38A810E94D781B80173
:10CD70008A81DF91CF911F910F91FF90EF90DF900B
:10CD80000C945E82CF93DF93EC018A81893010F49A
:10CD90000E94BE8148EE53E05B874A8720ED37E072
:10CDA0003D872C878CED95E09F878E87598B488B2C
:10CDB0003B8B2A8B9D8B8C8BDF91CF910895CF93EA
:10CDC000DF93EC017F8B6E8B8885998568177907D7
:10CDD00069F48A810E94D7818B8D882329F18A8109
:10CDE0000E944E829A8F898F1B8E1EC0CE010E9498
:10CDF000BD4FEA81EA30B0F49C01C39714F022E3FE
:10CE000030E02E3C8FEF380714F42EEC3FEF8FB755
:10CE1000F89495E1E99FF0011124E558FE4E318721
:10CE200020878FBF81E08B8FDF91CF910895CF93C3
:10CE3000DF93EC018BA19CA1892B11F01CA21BA2FA
:10CE40009B0177FF03C0319521953109B901CE01CE
:10CE50000E94BD4F90932D0180932C019F8B8E8B50
:10CE6000A2D66F8F78A389A39AA3DF91CF9108955B
:10CE70000F931F93CF93DF938C01FC01778B668B0D
:10CE80000E94BD4FEC01F8018281938188309105A9
:10CE9000D1F4D7FF06C060E08AE00E94814C61E0D7
:10CEA00005C061E08AE00E94814C60E086E00E945B
:10CEB000814CD7FF03C0D195C195D109D0932B01E7
:10CEC000C0932A011BC00997C9F4D7FF06C060E0D0
:10CED0008DE00E94814C61E005C061E08DE00E9420
:10CEE000814C60E08BE00E94814CD7FF03C0D1955C
:10CEF000C195D109D0932901C0932801DF91CF9129
:10CF00001F910F910895CF93DF93EC018A818930AF
:10CF100010F40E94BE812EEC3FEF3B872A8782E30C
:10CF200090E09D878C871F861E86398B288B9B8B74
:10CF30008A8B1D8A1C8A6EEE72E08A810E944A8268
:10CF40006AEC78E08A810E9446828CED95E09A8FA7
:10CF5000898F1B8EDF91CF910895CF93DF93EC01E2
:10CF60008BA19CA1892B11F01CA21BA2CE01FADD82
:10CF700010922D0110922C011F8A1E8A14D66F8FD9
:10CF800078A389A39AA3DF91CF9108950F931F935C
:10CF9000CF93DF93FC0123A134A1232B81F1EC017A
:10CFA00002D60F8D18A129A13AA1DC01CB01801B6B
:10CFB000910BA20BB30B4097A105B10500F18BA11A
:10CFC0009CA10197E1F46E897F89615071097F8B83
:10CFD0006E8BCE01161617062CF0DF91CF911F91A4
:10CFE0000F91BBCF0E94BD4F90932D0180932C01D8
:10CFF0009F8B8E8BD8D56F8F78A389A39AA3DF914F
:10D00000CF911F910F910895CF93DF93EC018D8DF8
:10D010009E8D1B861A869D878C871F861E86198A81
:10D02000188A9B8B8A8B1D8A1C8A61E08CE20E9485
:10D03000B04C8A819B81089721F410922D011092A7
:10D040002C011CA21BA2DF91CF910895CF93DF93F7
:10D05000EC0121E03FEF3B872A878FEF90E09D872F
:10D060008C871F861E86398B288B9B8B8A8B1D8A0B
:10D070001C8A61E08AE00E94B04C61E086E00E9478
:10D08000B04C61E08DE20E94B04C61E08DE00E9406
:10D09000B04C61E08BE00E94B04C61E08EE20E94F7
:10D0A000B04C8A819B818830910529F410922B0124
:10D0B00010922A0106C0099721F4109229011092BA
:10D0C0002801DF91CF9108950F931F93CF93DF93A2
:10D0D000EC0169D50C8D1D8D2E8D3F8DDC01CB01B2
:10D0E000801B910BA20BB30B853F9140A105B105AD
:10D0F00048F06E897F89CE01DF91CF911F910F910A
:10D100000C943650DF91CF911F910F9108950F939A
:10D110001F93CF93DF938C01FC01178A168AEC01D1
:10D12000699640E068E0CE010E94088F4FE766E014
:10D13000CE010E94088F40E06CE0CE010E94088F73
:10D140004FE767E0CE010E94088F2DD5F801648F6C
:10D15000758F868F978FDF91CF911F910F910895D3
:10D160006F927F928F929F92AF92BF92CF92DF92F7
:10D17000EF92FF920F931F93CF93DF938091F5125D
:10D180009091F612DC01ED91FC910480F581E02D87
:10D190001995B12C181619060CF0D4C0AA24A39422
:10D1A0008091F5129091F612DC01ED91FC910480D2
:10D1B000F581E02D1995892B09F4C4C0C0913B0E6F
:10D1C00081E08C0F80933B0E8091F5129091F612C6
:10D1D000DC01ED91FC910680F781E02D1995EC2F93
:10D1E000F0E0E550F24F80838A30D1F6E0903B0EBC
:10D1F000F12C10923C0D10923B0D1092370D1092B5
:10D20000380D1092390D10923A0D1092360D109281
:10D21000350D1092340D8BEFC82E8DE0D82E00E026
:10D2200010E0D0E0C0E00E151F050CF06EC0F60156
:10D2300091916F019D3009F465C09C3799F19A3046
:10D2400009F054C0CC2351F16C2E712CC30101970D
:10D250000E946D8970933C0D60933B0DA4D4609344
:10D26000F8127093F9128093FA129093FB12809146
:10D27000E10D882309F462C080903B0D90903C0D35
:10D28000B801661977098BEF9DE00E944B908816D4
:10D29000990609F453C01092FA0D52C01092FA0D7B
:10D2A000D0E030C08C2F90E0FC01E852FD4E10829F
:10D2B000D13099F068F0D230B1F40E946D8960935A
:10D2C000370D7093380D8093390D90933A0D0BC044
:10D2D0000E946D896093340D06C00E946D89709321
:10D2E000360D6093350DDF5FC0E00CC00F331105C4
:10D2F0003CF4EC2FF0E0E852FD4E9083CF5F02C08B
:10D300001092FA0D0F5F1F4F8ECF8091FA0D811191
:10D310000EC08091310D9091320D01969093320D97
:10D320008093310D60E087E80E94EE9002C0BB243C
:10D33000B3941092FB0D10923B0E32CFA092FA0DD7
:10D34000D1E0E0CF8B2DDF91CF911F910F91FF9016
:10D35000EF90DF90CF90BF90AF909F908F907F9095
:10D360006F900895CF931092330D1092300D10925C
:10D37000320D1092310D61E089E30E94814C0E94D0
:10D38000EE8F8091F5129091F612DC01ED91FC91F7
:10D390000480F581E02D1995892B61F08091F512BB
:10D3A0009091F612DC01ED91FC910680F781E02D61
:10D3B0001995E7CF0E9469918091F5129091F6122C
:10D3C000DC01ED91FC910284F385E02D199510921A
:10D3D000F712E9D36093F8127093F9128093FA125E
:10D3E0009093FB12C1E0BCDE81110E94EA2F0E94E3
:10D3F0002E900E9431858091310D9091320D0A97C7
:10D4000024F48091F712882331F060E08AE80E94CA
:10D41000EE90C093330D8091330D882321F38091DA
:10D42000300D882341F040ED51E060E070E08AE883
:10D430009EE00E944BB560E089E30E94814C60E071
:10D440008AE3CF910C94814CEF92FF920F931F933C
:10D45000CF93DF9300D000D0CDB7DEB767EE75E095
:10D46000CE0101960E94CA480D811E81F02EEE2445
:10D47000E3948091F5129091F612DC01ED91FC910C
:10D480000480F581E02D1995892B21F18091F51209
:10D490009091F612DC01ED91FC910680F781E02D70
:10D4A00019958F3439F4E092F90D8093EE0DE092E6
:10D4B000ED0DDFCF9091F90D9923D9F2E091ED0DAB
:10D4C00091E09E0F9093ED0DF0E0E251F24F8083DA
:10D4D0009F1578F28091ED0D8F1510F4F12C21C07D
:10D4E0004BE050E062EE7DE0CE0101960E946E7945
:10D4F000AEEEBDE0E7EEF5E0FF24F3941127CF0197
:10D50000875E95408017910734F49D91819198171B
:10D51000B1F3F12CF4CF1092EE0D1092F90D1092A0
:10D52000ED0DCE0101960E949A488F2D26960FB6DA
:10D53000F894DEBF0FBECDBFDF91CF911F910F9149
:10D54000FF90EF900895DC01ED91FC910190F08146
:10D55000E02D1994CF93DF93EC017F8B6E8B0E94AB
:10D56000BD4FBC018A81DF91CF910C945E82809186
:10D570000D02882311F0729801C0729A90910D02E9
:10D5800081E0892780930D0208951092060610927B
:10D5900000061092F70510920106109202061092F2
:10D5A00003061092040681E08093C30A40910C06A2
:10D5B00050910D0660E070E024EE3AE68091F805A7
:10D5C0009091F9050C9476808091D60981111CC048
:10D5D00010920E0A10920F0A1092100A1092110A5D
:10D5E0001092120A1092130A1092160A8091C10A20
:10D5F0009091C20ADC01ED91FC910190F081E02D47
:10D6000019951092C30A089524EE3AE645E050E0D9
:10D6100060E070E08091F8059091F9050C947680B7
:10D620006091490E70914A0E8091F8059091F9052C
:10D630000E940F80882319F081E08093480E08959E
:10D6400060E087E00E94814C1092C40A089561E076
:10D6500087E00E94814C81E08093C40A0895CF93B3
:10D66000DF938091560E811110C084EF91E090936A
:10D67000550E8093540E8BE290E09093530E80935E
:10D68000520E81E08093560E20C08091520E9091F0
:10D69000530E8532910514F0049709C0833191052A
:10D6A00014F0029704C0823091052CF001979093FA
:10D6B000530E8093520E8091520E9091530E97FF0D
:10D6C00004C01092530E1092520EC091510ECC23F2
:10D6D00011F0B6DF01C0BBDF81E08C278093510ED3
:10D6E000C091540ED091550E1C161D0654F0109288
:10D6F000560EA6DF2FE93BE64AEF50E060E070E00F
:10D7000007C02FE23BE6AE010D2E000C660B770B37
:10D710008091F8059091F9050E9476809093500EC3
:10D7200080934F0E8091520E9091530EC81BD90BCF
:10D73000D093550EC093540EDF91CF9108950F935F
:10D740001F93CF93DF938091C50A882329F0DF913F
:10D75000CF911F910F9183CF00914F0E1091500EDA
:10D76000C091F805D091F905B801CE010E940F8053
:10D77000882321F0B801CE010E942780DF91CF914C
:10D780001F910F915DCFCF92DF92EF92FF92109297
:10D79000C50A2091FC053091FD054091FE05509190
:10D7A000FF05609101067091020680910306909139
:10D7B00004060E942CB06B017C0120E030E0A9013E
:10D7C0000E9432B487FD09C0C0920106D0920206C1
:10D7D000E0920306F092040608C01092010610922F
:10D7E00002061092030610920406FF90EF90DF905D
:10D7F000CF90A5CF0F931F93CF93DF9380914E0EC1
:10D800009091060681112AC0992309F456C000910F
:10D810004C0E10914D0EC091F805D091F905B8014C
:10D82000CE010E940F80882321F0B801CE010E9412
:10D8300027800DDF2AEF3BE642EC51E060E070E02C
:10D840008091F8059091F9050E947E8090934D0E8D
:10D8500080934C0E81E080934E0E5AC08091C40A92
:10D86000992361F0882329F0DF91CF911F910F91C7
:10D87000E7CEDF91CF911F910F91E9CE8823C9F3B5
:10D8800060914C0E70914D0E8091F8059091F905C4
:10D890000E9427802AEF3BE644E150E060E070E020
:10D8A0008091F8059091F9050E947E8090934D0E2D
:10D8B00080934C0E10924E0E2BC0C0910E02D09150
:10D8C0000F022297D0930F02C0930E021C161D0662
:10D8D00074F4BE01772787E00E94EC4CCC2321F042
:10D8E00081E08093C40A14C01092C40A11C06091F0
:10D8F0004C0E70914D0E8091F8059091F9050E94A3
:10D9000027809EDE8FEF90E090930F0280930E02AF
:10D91000DF91CF911F910F9108950F931F93CF9394
:10D92000DF930091440E1091450EC091460ED091A8
:10D93000470EC00FD11FD093470EC093460EBE01B5
:10D94000772787E00E94EC4CCC2321F081E0809384
:10D95000C40A02C01092C40A10161106ECF5809198
:10D96000420E9091430EC817D9070CF485C08091E0
:10D97000480E882371F01092430E1092420E8CEFE5
:10D980009FEF9093450E8093440E81E08093410E6B
:10D9900073C068E770E080E090E00E94DE48DC0140
:10D9A000CB010A96A11DB11D9093430E8093420EA8
:10D9B00068E270E080E090E00E94DE48DC01CB018C
:10D9C0000A96A11DB11D66277727681B790B7093F6
:10D9D000450E6093440E50C0012B09F44DC0809158
:10D9E000420E9091430E8C179D070CF445C0809118
:10D9F000410E882311F10091490E10914A0EC091F9
:10DA0000F805D091F905B801CE010E940F80882356
:10DA100099F1B801CE010E94278012DE1092470EC4
:10DA20001092460E1092410E80910606882321F135
:10DA3000DF91CF911F910F91DDCE69E670E080E01C
:10DA400090E00E94DE48DC01CB018A569F4FAF4F29
:10DA5000BF4F9093430E8093420E68E270E080E0E7
:10DA600090E00E94DE48DC01CB010A96A11DB11DA9
:10DA70009093450E8093440EDF91CF911F910F91AB
:10DA80000895EF92FF921F93CF93DF9300D0CDB70D
:10DA9000DEB784E689838CE38A8388E28B831091E6
:10DAA0004B0E1330E8F4E12EF12C10FF02C0C8DD5C
:10DAB00001C0CDDDE1E0F0E0EC0FFD1FEE0DFF1D3C
:10DAC000408150E060E070E021E43DE68091F8059F
:10DAD0009091F9050E9476801F5F10934B0E03C052
:10DAE000AFDD10924B0E0F900F900F90DF91CF9102
:10DAF0001F91FF90EF90089560E088E00C94814CB6
:10DB000061E089E20C94814C0F931F93CF93DF93D4
:10DB100060E08BE20E94814C00913F0E1091400E1C
:10DB2000C091F805D091F905B801CE010E940F808F
:10DB3000882341F0B801CE01DF91CF911F910F9161
:10DB40000C942780DF91CF911F910F91089581E070
:10DB50008093C30A80911406ECD536CD3FB7F89474
:10DB600080915C0E90915D0EA0915E0EB0915F0E63
:10DB700026B5A89B05C02F3F19F00196A11DB11D28
:10DB80003FBFBA2FA92F982F8827820F911DA11D63
:10DB9000B11DBC01CD0142E0660F771F881F991FA0
:10DBA0004A95D1F708952FB7F8946091580E709167
:10DBB000590E80915A0E90915B0E2FBF08951F93BE
:10DBC000CF93DF93CDB7DEB765970FB6F894DEBF7E
:10DBD0000FBECDBF11E01093C70A80913C0E882381
:10DBE00091F10E94C7761092F40982E390E09A8343
:10DBF000898328E230E03C832B832EE630E03E83AD
:10DC00002D8324EF31E038872F831D8A25E1FE0123
:10DC10003196A5EFB9E001900D922A95E1F7909326
:10DC2000F3098093F20984E08093F1090E94BC76A5
:10DC3000BADF6093E3097093E4098093E509909358
:10DC4000E6091093EF0965960FB6F894DEBF0FBE94
:10DC5000CDBFDF91CF911F9108951F920F920FB604
:10DC60000F9211242F933F938F939F93AF93BF9362
:10DC70008091580E9091590EA0915A0EB0915B0E62
:10DC80003091570E23E0230F2D3720F40196A11D6C
:10DC9000B11D05C026E8230F0296A11DB11D2093DA
:10DCA000570E8093580E9093590EA0935A0EB0932E
:10DCB0005B0E80915C0E90915D0EA0915E0EB09116
:10DCC0005F0E0196A11DB11D80935C0E90935D0EB9
:10DCD000A0935E0EB0935F0EBF91AF919F918F9115
:10DCE0003F912F910F900FBE0F901F9018950F939B
:10DCF0001F93CF93DF9300914F0E1091500EC09160
:10DD0000F805D091F905B801CE010E940F80882353
:10DD1000A1F0B801CE010E94278020E13BE648EB4C
:10DD20005BE060E070E08091F8059091F9050E9459
:10DD300076809093500E80934F0E6091490E7091B3
:10DD40004A0E8091F8059091F9050E940F8081118B
:10DD50004BC01092480E8FEF90E09093470E809347
:10DD6000460E75DC68E770E080E090E00E94DE48D7
:10DD7000DC01CB010A96A11DB11D9093430E809347
:10DD8000420E68E270E080E090E00E94DE48DC0134
:10DD9000CB010A96A11DB11D66277727681B790B59
:10DDA0007093450E6093440E2DE83CE644E150E04C
:10DDB00060E070E08091F8059091F9050E947E8006
:10DDC00090934A0E8093490E20E13BE648EB5BE0DE
:10DDD00060E070E08091F8059091F9050E947680EE
:10DDE0009093500E80934F0EDF91CF911F910F9122
:10DDF00008958F929F92AF92BF92CF92EF92FF922F
:10DE00000F931F93CF93DF9320911706223008F0D2
:10DE10007AC07B018C018090010690900206A09050
:10DE20000306B090040620E030E0A901C501B4016A
:10DE30000E9432B4181654F520E030E0A901C50163
:10DE4000B4010E942AB1181654F420E030E048E4EE
:10DE500052E4C501B4010E9432B41816D4F420E093
:10DE600030E048E452E4C501B4010E942AB118161A
:10DE70009CF420E030E048EC52E4C501B4010E947B
:10DE800032B487FF09C0CBE4D0E008C0C0E0D0E0E6
:10DE900005C0C2E3D0E002C0C4E6D0E08FEF8C0D35
:10DEA000823070F4209739F06C2FC8010E94304FF7
:10DEB0006C2FC7010DC0C8010E94B265C70116C012
:10DEC0008DEF8C0D8330F8F4209779F06C2FC8011A
:10DED000DF91CF911F910F91FF90EF90CF90BF9066
:10DEE000AF909F908F900C94304FC801DF91CF91ED
:10DEF0001F910F91FF90EF90CF90BF90AF909F90A8
:10DF00008F900C94B265DF91CF911F910F91FF908C
:10DF1000EF90CF90BF90AF909F908F9008958F9289
:10DF20009F92AF92BF92CF92DF92EF92FF92C090FA
:10DF30000106D0900206E0900306F090040620E06F
:10DF400030E0A901C701B6010E942AB120E030E00B
:10DF500040E05FE387FD0BC0C701B6010E942DB012
:10DF60004B015C010E94F9B097FD27C010C0C701AA
:10DF7000B6010E942CB00E94F9B097FD1EC0653614
:10DF8000710581059105DCF424E6822F14C0C501DA
:10DF9000B4010E94F9B065367105810591057CF4E4
:10DFA00020E030E040E05FE3C701B6010E942DB001
:10DFB0000E94F9B084E6861B03C084E601C080E0BD
:10DFC000FF90EF90DF90CF90BF90AF909F908F9099
:10DFD00008950F931F93CF93DF930091F105109154
:10DFE000F205C091F805D091F905B801CE010E9463
:10DFF0000F80882321F0B801CE010E9427808091F4
:10E00000C50A882339F01092C50ADF91CF911F917C
:10E010000F9195CBDF91CF911F910F91089560E003
:10E0200089E20E94814C20E83DE642E350E060E056
:10E0300070E08091F8059091F9050C9476801F921C
:10E040000F920FB60F9211240BB60F922F933F939E
:10E050004F935F936F937F938F939F93AF93BF93F0
:10E06000EF93FF9380913E0E8823A9F0669917C025
:10E07000EE9824E83DE64CE251E060E070E08091EB
:10E08000F8059091F9050E94768080913D0E8823D5
:10E0900031F0C6D004C0669B02C0EE9835DDFF911A
:10E0A000EF91BF91AF919F918F917F916F915F9110
:10E0B0004F913F912F910F900BBE0F900FBE0F907D
:10E0C0001F90189561E08BE20E94814CEE9A24E843
:10E0D0003DE648E853E160E070E08091F8059091FA
:10E0E000F9050E9476809093400E80933F0E08952C
:10E0F00061E08BE20E94814CEE9A24E83DE648E81C
:10E1000053E160E070E08091F8059091F9050E947C
:10E1100076809093400E80933F0E08951092C70A28
:10E1200040910A0650910B0660E070E02FED3DE64D
:10E130008091F8059091F9050C9476808091800E7D
:10E14000811112C080E594E8A1E0BB27ABBFFC01C0
:10E150006791769182E00E94978181E08093610EC1
:10E160001092650E1092620E089581E08093600E09
:10E170006CED75E00C94978181E20E94594C21E08E
:10E18000892B09F420E0822F0895809110068823BE
:10E1900009F445C081E08093C30AEEDF882329F0AB
:10E1A000809113068823D1F106C080911106811158
:10E1B00004C080911006BDD231C0909110069630F7
:10E1C00069F5823081F08330D1F0813039F5E0910A
:10E1D000310AF091320A72978081918145E550E0D1
:10E1E00060E070E017C0E091310AF091320A729756
:10E1F000808191814AE550E060E070E00BC0E091E1
:10E20000310AF091320A7297808191814FE550E096
:10E2100060E070E08F5C954F0E94EB52D5C9089585
:10E2200080913E0E882339F080913D0E882319F0AD
:10E2300081E08093C00A8091FA059091FB05DC0192
:10E24000ED91FC910688F789E02D19958091860E55
:10E250008111E5DE8091850E882391F061E088E0F0
:10E260000E94814C4091830E5091840E60E070E0DA
:10E270002CE73DE68091F8059091F9050E947680A3
:10E2800080913E0E882321F080913D0E811101C0C6
:10E290007CDF80913D0E882379F080913E0E8823AB
:10E2A00059F08091890E882339F0E091870EF09122
:10E2B000880E82810E94E58131CF8091C50A81114B
:10E2C00055C05ADF8823E9F081E08093C50A809128
:10E2D000FA059091FB05DC01ED91FC910288F38930
:10E2E000E02D19952CDA23EC3BE648E95AE360E08F
:10E2F00070E08091F8059091F9050E9476800EDF1C
:10E3000009C080913D0E882329F180913E0E88231B
:10E3100011F0EEDE3ACFD6DE8091890E882339F0F7
:10E32000E091870EF091880E82810E94E5814091F4
:10E33000810E5091820E14161506BCF4052E000CA9
:10E34000660B770B20E131E78091F8059091F90594
:10E350000C9476808091890E882339F0E091870EA5
:10E36000F091880E82810E94E5815ACF08950F9323
:10E370001F932091800E211135C040E554E861E0E3
:10E3800077279C01220F331F820F931F092E000C49
:10E39000AA0BBB0B0296A11DB11D840F951FA61FD2
:10E3A000B71FABBFFC01879100E514E821E03327DC
:10E3B0004091650E93E0499FA0011124052E000CA9
:10E3C000660B770B4E5F5F4F6F4F7F4F040F151F2C
:10E3D000261F371F2BBFF8010791801718F01F91D8
:10E3E0000F91ACCE1F910F9108958F929F92AF9293
:10E3F000BF92CF92DF92EF92FF920F931F93CF9332
:10E40000DF93EC01A62E8091800E81116BC040E558
:10E4100054E861E077276E01CC0CDD1CCC0EDD1ECC
:10E420000D2C000CEE08FF08D701C6010296A11DB5
:10E43000B11D480F591F6A1F7B1F6BBFFA018791DF
:10E4400040E554E861E07727B090650E93E0B99E0F
:10E4500080011124012E000C220B330B0E5F1F4F85
:10E460002F4F3F4F400F511F621F731F6BBFFA01A9
:10E470004791481708F036C08090630E9090640E64
:10E480000091790E10917A0EB401C8010E940F809C
:10E49000882321F0B401C8010E94278080E594E818
:10E4A000A1E0BB278C0D9D1DAE1DBF1DABBFFC01A8
:10E4B0006791769182E00E949781B092620EC0933C
:10E4C000650EAA2079F01092610E2EE930E742E342
:10E4D00050E060E070E0C8010E9476809093640E86
:10E4E0008093630EDF91CF911F910F91FF90EF907A
:10E4F000DF90CF90BF90AF909F908F900895CF9274
:10E50000DF92EF92FF928091800E811134C0809152
:10E510007F0E882381F161E08EE090E066DF6091FC
:10E520007D0E70917E0ECB01A0E0B0E0C0907B0E1E
:10E53000D0907C0EE12CF12CC816D906EA06FB0619
:10E5400064F4BC01CD016C197D098E099F090E94FC
:10E55000DE48C60ED71EE81EF91E2FE732E7B701C8
:10E56000A6018091790E90917A0E0E947680909308
:10E57000780E8093770EFF90EF90DF90CF90089504
:10E58000CF92DF92EF92FF928091800E811134C082
:10E590008091760E882381F161E08DE090E025DFA7
:10E5A0006091740E7091750ECB01A0E0B0E0C09048
:10E5B000720ED090730EE12CF12CC816D906EA0623
:10E5C000FB0664F4BC01CD016C197D098E099F091D
:10E5D0000E94DE48C60ED71EE81EF91E20EC32E768
:10E5E000B701A6018091790E90917A0E0E947680F3
:10E5F0009093710E8093700EFF90EF90DF90CF900C
:10E600000895CF92DF92EF92FF928091800E811158
:10E6100034C080916F0E882381F161E08CE090E03E
:10E62000E4DE60916D0E70916E0ECB01A0E0B0E063
:10E63000C0906B0ED0906C0EE12CF12CC816D90650
:10E64000EA06FB0664F4BC01CD016C197D098E0954
:10E650009F090E94DE48C60ED71EE81EF91E21E063
:10E6600033E7B701A6018091790E90917A0E0E944E
:10E67000768090936A0E8093690EFF90EF90DF9002
:10E68000CF9008958091800E81112CC08091680EEA
:10E69000882341F080916F0E811104C081E0809346
:10E6A0006F0EAFDF8091670E882361F08091800E3E
:10E6B000811108C08091760E811104C081E08093A1
:10E6C000760E5EDF8091660E882361F08091800E69
:10E6D000811108C080917F0E811104C081E0809378
:10E6E0007F0E0DCF08958091800E81110BC0809117
:10E6F000600E882339F060ED77E081E00E94978119
:10E700000C94CD5F08950F931F93CF93DF93EC018B
:10E71000AB0160E070E02AE00E9442498C01CE012A
:10E720000E94674A800F911FDF91CF911F910F9137
:10E7300008958F929F92AF92BF92CF92DF92EF9205
:10E74000FF920F931F93CF93DF931F921F92CDB72A
:10E75000DEB7082E000C990BAA0BBB0BFC013197FE
:10E76000ED30F10508F033C28827E159FE4F8F4F95
:10E770000C9418B084E08093D2098AE08093D30986
:10E7800086E28093D50981E08093D8098093D909E6
:10E790008093D70943E457E120E030E08091D2092B
:10E7A00090E0281739070CF059C1FA01859194912E
:10E7B000A0E0B0E0880F991FAA1FBB1FF901EE0F60
:10E7C000FF1FEE0FFF1FE759F64F80839183A2834F
:10E7D000B3832F5F3F4F4E5F5F4FE0CF84E0809366
:10E7E000D2098AE08093D30986E28093D50981E03B
:10E7F0008093D8098093D90982E08093D7094BE3AD
:10E8000057E120E030E08091D20990E028173907E5
:10E810000CF024C1FA0185919491A0E0B0E0880F3A
:10E82000991FAA1FBB1FF901EE0FFF1FEE0FFF1F5D
:10E83000E759F64F80839183A283B3832F5F3F4FC5
:10E840004E5F5F4FE0CF84E08093D30985E28093F1
:10E85000D50981E08093D80988E08093D90983E0C5
:10E860008093D70980E090E0FC01ED5CF84EE491E4
:10E87000DC01A652B64FEC93019688309105A1F7C2
:10E880000E949651EBC088E08093D20986E0809385
:10E89000D30986E28093D50981E08093D8098093DB
:10E8A000D90984E08093D70943E257E120E030E0C2
:10E8B0008091D20990E0281739070CF0CFC0FA01F7
:10E8C00085919491A0E0B0E0880F991FAA1FBB1F0B
:10E8D000F901EE0FFF1FEE0FFF1FE759F64F808380
:10E8E0009183A283B3832F5F3F4F4E5F5F4FE0CF93
:10E8F00088E08093D20986E08093D30986E28093F2
:10E90000D50981E08093D8098093D90985E0809367
:10E91000D70943E157E120E030E08091D20990E04F
:10E92000281739070CF09AC0FA0185919491A0E05C
:10E93000B0E0880F991FAA1FBB1FF901EE0FFF1F40
:10E94000EE0FFF1FE759F64F80839183A283B383B5
:10E950002F5F3F4F4E5F5F4FE0CFE091310AF09164
:10E96000320A72978081918140E550E060E070E06A
:10E970008F5C954F0E94EB522AC182E18093D209AD
:10E9800085E08093D30982E28093D50981E080936A
:10E99000D8098093D90987E08093D70980E993E368
:10E9A000A0E0B0E08093690990936A09A0936B0995
:10E9B000B0936C09F2E08F2E912C01E010E080E022
:10E9C00090E0A0E0BBE54CE454E060E070E024EEB1
:10E9D000C22E2CE0D22EE12CF12C9801220F331FF5
:10E9E000220F331F5401AA0CBB1CAA0CBB1C2759B5
:10E9F000364FF901B7FF0DC0C082D182E282F382A7
:10EA000095012759364FF9014083518362837383FF
:10EA10000CC0408351836283738395012759364F1D
:10EA2000F901C082D182E282F382880F991FAA1F66
:10EA3000BB1F0E5F1F4FF2E08F0E911C22E182166A
:10EA4000910459F688E79FEFA0E0B0E08093AD090C
:10EA50009093AE09A093AF09B093B0090E940552FC
:10EA6000B6C0CE0101960E94845123E040E150E0FF
:10EA700060E070E072C084E08093D20982E380930A
:10EA8000D30986E28093D50981E08093D8098093E9
:10EA9000D9098AE08093D7094BE057E120E030E0C4
:10EAA0008091D20990E028173907C4F6FA018591C0
:10EAB0009491A0E0B0E0880F991FAA1FBB1FF90135
:10EAC000EE0FFF1FEE0FFF1FE759F64F8083918374
:10EAD000A283B3832F5F3F4F4E5F5F4FE1CF84E050
:10EAE0008093D20980E28093D30986E28093D5098E
:10EAF00081E08093D8098093D9098BE08093D7096E
:10EB000043E057E120E030E08091D20990E02817FF
:10EB100039070CF0A3CFFA0185919491A0E0B0E001
:10EB2000880F991FAA1FBB1FF901EE0FFF1FEE0FE1
:10EB3000FF1FE759F64F80839183A283B3832F5F32
:10EB40003F4F4E5F5F4FE0CFCE0101960E94845150
:10EB500021E040E154E060E070E0CE0101960E94C7
:10EB60005F5235C084E08093D20983E08093D3095B
:10EB700086E28093D50981E08093D8098093D909F2
:10EB80008DE08093D7094BEF56E120E030E0809193
:10EB9000D20990E0281739070CF060CFFA0185916F
:10EBA0009491A0E0B0E0880F991FAA1FBB1FF90144
:10EBB000EE0FFF1FEE0FFF1FE759F64F8083918383
:10EBC000A283B3832F5F3F4F4E5F5F4FE0CF0F9025
:10EBD0000F90DF91CF911F910F91FF90EF90DF90F9
:10EBE000CF90BF90AF909F908F9008950F931F93F9
:10EBF000CF93DF93EC01462F50E060E070E02AE015
:10EC00000E9442498C01CE010E94674A800F911FE9
:10EC1000DF91CF911F910F9108952FB7F89488231A
:10EC200081F08091BD119091BE119093CC11809391
:10EC3000CB118091CD119091CE1118161906ACF020
:10EC40000FC08091BF119091C0119093CC1180930F
:10EC5000CB118091CD119091CE11181619062CF47C
:10EC60008091CD119091CE1107C08091CD119091DE
:10EC7000CE119195819591099093CE118093CD11EC
:10EC80002FBF0895AF92BF92CF92DF92EF92FF9283
:10EC90000F931F93CF93DF931F921F92CDB7DEB7D1
:10ECA0008C017A836983CE0101966C01580192E050
:10ECB000A90EB11CE12CF12CC8010E945BB5F60134
:10ECC00061916F01861731F0C8010E946DB5FFEFA9
:10ECD000EF1AFF0A0F5F1F4F0A151B0569F781E046
:10ECE000EF2809F480E00F900F90DF91CF911F91F2
:10ECF0000F91FF90EF90DF90CF90BF90AF9008956D
:10ED0000EF92FF920F931F93CF93DF931F921F9267
:10ED1000CDB7DEB78C017B018AEA8A8341E050E0FF
:10ED2000BE016E5F7F4FC8010E948740D701ED9101
:10ED3000FC910284F385E02DC701199582E889834F
:10ED400041E050E0BE016F5F7F4FC8010E948740E5
:10ED50000F900F90DF91CF911F910F91FF90EF9047
:10ED600008958091EE09882311F061E001C060E010
:10ED70008091ED090C94814C8091EE09882311F06B
:10ED800060E001C061E08091ED090C94814CCF936B
:10ED9000DF93C3EED9E01C861D861E86188A1F8667
:10EDA0000E94D36D688379838A839B831986188632
:10EDB0001C86DF91CF910895CF92DF92EF92FF9260
:10EDC0000F931F930E94D36D6B017C0160933912E6
:10EDD00070933A1280933B1290933C128091DC0A1C
:10EDE0000E94594C809338129091DE0A992329F0A1
:10EDF00091E0811190E0909338128091E60A909111
:10EE0000E70AA091E80AB091E90A97018601081B78
:10EE1000190B2A0B3B0B4091EA0A5091EB0A6091C7
:10EE2000EC0A7091ED0A9091DF0A04171507260786
:10EE3000370760F4C092E20AD092E30AE092E40A53
:10EE4000F092E50A1092E10A892F1EC09093E00A21
:10EE5000809138128093DF0AC092E20AD092E30ACE
:10EE6000E092E40AF092E50A891761F0C092E60A9E
:10EE7000D092E70AE092E80AF092E90A91E09093D2
:10EE8000E10A02C01092E10A1F910F91FF90EF90EA
:10EE9000DF90CF900895462F50E060E070E02AE0C8
:10EEA0000C9442490F931F93CF93DF93EC012AE018
:10EEB0000E9442498C01CE010E94674A800F911F37
:10EEC000DF91CF911F910F910895CF92DF92EF9232
:10EED000FF920F931F93CF93DF936B01770FEE0891
:10EEE000FF08F7FE1BC0EC016DE20E9402498C0195
:10EEF00044275527BA014C195D096E097F092AE09C
:10EF0000CE010E944249800F911FDF91CF911F9146
:10EF10000F91FF90EF90DF90CF9008952AE0B70116
:10EF2000A601DF91CF911F910F91FF90EF90DF909D
:10EF3000CF900C944249CF92DF92EF92FF920F93C1
:10EF40001F93CF93DF938C016B01770FEE08FF08BF
:10EF5000F7FE12C06DE20E940249EC0144275527DA
:10EF6000BA014C195D096E097F092AE0C8010E94A7
:10EF70004249C80FD91F06C02AE0B701A6010E9466
:10EF80004249EC01C8010E94674A8C0F9D1FDF9126
:10EF9000CF911F910F91FF90EF90DF90CF90089548
:10EFA0000F931F93CF93DF931F92CDB7DEB78C01E2
:10EFB00069830E945BB56981861729F0C8010E94A8
:10EFC0006DB581E001C080E00F90DF91CF911F917E
:10EFD0000F910895CF930E94488584E090E090932C
:10EFE000D90A8093D80A8BE89EE090935C118093B5
:10EFF0005B11109256118091D70A90918B0E891750
:10F0000018F091E09093531124E93EE0309366119B
:10F0100020936511109260119091940E891718F049
:10F0200091E090935D112DE93EE0309370112093B3
:10F030006F1110926A1190919D0E891718F091E04E
:10F040009093671126EA3EE030937A11209379116C
:10F05000109274119091A60E891718F091E0909378
:10F0600071111092D60A20E030E0F901E55DF04F11
:10F0700040815181415051094432510520F491E0C1
:10F080009093D60A05C02D5F3F4F2837310569F7A9
:10F090009091D60A992341F120919E0E30919F0EB6
:10F0A0002D5D3F4F30939F0E20939E0E2091A00E1A
:10F0B0003091A10E235231093093A10E2093A00E5E
:10F0C0002091A70E3091A80E2D5D3F4F3093A80ED2
:10F0D0002093A70E2091A90E3091AA0E2352310938
:10F0E0003093AA0E2093A90E9091A40F9F3049F45B
:10F0F0009091A50F9F3029F4109252111092511146
:10F1000008C02091F80F3091F90F309352112093DD
:10F11000511122E130E030934F1120934E11209194
:10F12000D80A3091D90AAFEABEE0EAEFF0E141E057
:10F13000B683A5839C91992329F0891718F0408301
:10F140002F5F3F4F1A96379691E1EE34F90781F71A
:10F150003093D90A2093D80A2131310534F080E167
:10F1600090E09093D90A8093D80A0E94338587E56E
:10F1700091E190935D1080935C1080915B11909170
:10F180005C1190935B1080935A1084E591E1909309
:10F190005F1080935E1085E591E1909361108093FC
:10F1A000601083E591E1909363108093621081E693
:10F1B00091E1909367108093661080916511909112
:10F1C000661190936510809364108EE591E19093A1
:10F1D0006910809368108FE591E190936B10809394
:10F1E0006A108DE591E190936D1080936C108BE621
:10F1F00091E1909371108093701080916F119091B4
:10F20000701190936F1080936E1088E691E1909347
:10F2100073108093721089E691E19093751080933A
:10F22000741087E691E1909377108093761085E7CC
:10F2300091E190937B1080937A1080917911909155
:10F240007A11909379108093781082E791E19093EE
:10F250007D1080937C1083E791E190937F108093E1
:10F260007E1081E791E1909381108093801020912E
:10F27000D80A3091D90A2450310960E07AE0C7E019
:10F28000462F50E04217530724F5CA010496789F91
:10F29000F001799FF00D1124E65AFF4EC49FC00182
:10F2A000C59F900D1124AC0144505F4E538342839F
:10F2B000DC01A650BF4E15964D915C911697518377
:10F2C000408385509F4E95838483B187A0876F5F6D
:10F2D000D7CF81E08093DA0ACF9108950F931F93DF
:10F2E000CF93DF93FC01248135812115310519F479
:10F2F000FB01108211C0EA0121972C173D0708F489
:10F30000E9018B01FC0160817181AE01C8010E949D
:10F3100062B3C00FD11F1882DF91CF911F910F915F
:10F320000895FC01128213821482158216821782BC
:10F330001286089580E008950F931F93CF938C0158
:10F3400069E078E18CEC98E00E940949D8011896B0
:10F35000ED91FC911997608171818CEC98E0D3D983
:10F36000C1E0D8011A968C91C81700F564E078E1E5
:10F370008CEC98E00E9409496C2F8CEC98E08BDDB6
:10F3800061E078E18CEC98E00E940949F8019085F1
:10F390008185E92FF82FEC0FF11DEC0FF11D608135
:10F3A00071818CEC98E0AFD9CF5FDBCFCF911F910B
:10F3B0000F910895CF93DF93CDB7DEB76E970FB659
:10F3C000F894DEBF0FBECDBF8F300CF080E029EF88
:10F3D00037E13A83298322EF37E13C832B8324EE04
:10F3E00037E13E832D8328ED37E138872F832EECDC
:10F3F00037E13A87298727EC37E13C872B8723ECD5
:10F4000037E13E872D872CEB37E1388B2F8721EBB7
:10F4100037E13A8B298B24EA37E13C8B2B8B29E9A6
:10F4200037E13E8B2D8B2DE837E1388F2F8B2BE783
:10F4300037E13A8F298F2AE637E13C8F2B8F25E67B
:10F4400037E13E8F2D8FE82FEE0FFF0BEC0FFD1FE6
:10F45000818192816E960FB6F894DEBF0FBECDBF4C
:10F46000DF91CF910895AF92BF92CF92DF92EF924A
:10F47000FF920F931F93CF93DF938AE492E17EE193
:10F48000D72ED80ECC24C39402E010E0C3E0D0E025
:10F49000E2E0BE2EEE24E394F12C8091890D909150
:10F4A0008A0DDC01ED91FC910480F581E02D199528
:10F4B000892B09F4ADC0A09030018091890D909105
:10F4C0008A0DDC01ED91FC910680F781E02D199504
:10F4D00096B3B39A2091840030918500285A344E17
:10F4E00030938D0020938C002A2D2C7119F01092EE
:10F4F000730D4BC093FB992790F9E091730DE111C7
:10F5000016C0992351F2803241F6C092730D809358
:10F510004A128091AB0D9091AC0D892B09F0BDCFB3
:10F52000F092AC0DE092AB0D1092750DB6CF91112B
:10F53000DECFE13041F4803409F0AFCFB092730DEB
:10F5400080934B12E6CF91E09E0F9093730DF0E005
:10F55000E65BFD4E8083903209F09FCF1092730DD1
:10F56000EAE4F2E12FEF3FEF8191281B3109DE122F
:10F57000FBCF409168128091691290E0982F882704
:10F58000840F911D2817390729F0D093AC0DC09333
:10F59000AB0D83CF8091AB0D9091AC0D019739F4F9
:10F5A0008091750D8F5F8093750D843020F01093DE
:10F5B000AC0D0093AB0D8091740D8F5F8093740D33
:10F5C0009091720D981708F5C092AD0D20E030E0D3
:10F5D000F901E65BFD4E4281838190E0982F8827F8
:10F5E000840F911DAC014F5E52404B3D554028F4B5
:10F5F000F901E557F24F918380832E5F3F4F2C3105
:10F60000310531F71092740D48CF1092AD0D45CFF2
:10F61000DF91CF911F910F91FF90EF90DF90CF90EE
:10F62000BF90AF900895EF92FF920F931F93CF93E7
:10F63000DF9310928A0E82E080938B0E68EE73E067
:10F6400070938D0E60938C0E40ED57E050938F0EAB
:10F6500040938E0E2CED35E03093910E2093900E5A
:10F660008FE08093920E1092930E94E09093940EFC
:10F670007093960E6093950E5093980E4093970E4C
:10F6800030939A0E2093990E80939B0E10929C0EAD
:10F6900093E090939D0E70939F0E60939E0E5093F7
:10F6A000A10E4093A00E3093A30E2093A20E809340
:10F6B000A40E1092A50E91E09093A60E7093A80E42
:10F6C0006093A70E5093AA0E4093A90E3093AC0EF0
:10F6D0002093AB0E8093AD0E1092AE0EEFEAFEE0DB
:10F6E000A8EBBEE080E008EE13E060ED77E04CEDC3
:10F6F00055E031E022E095E0980F9083128301837A
:10F700007483638356834583ED01229791E03883A8
:10F71000219628831C928F5F3A961A968C3059F75F
:10F720001092270F9093280F1092290F90932A0F71
:10F7300080E090E09C012657314FF901EF55FF4FD3
:10F74000118210823296108203968837910591F7C4
:10F7500084E290E090932C0F80932B0F81E08093B4
:10F760002D0F2CE030E030932F0F20932E0F94E0DC
:10F770009093300F21E230E03093320F2093310F1D
:10F7800027E02093330F29E030E03093350F2093AA
:10F79000340F20E12093360F7AE07093A30F2BE013
:10F7A0002093A40F2093A50F48EE53E05093A70F8A
:10F7B0004093A60F20ED37E03093A90F2093A80FB8
:10F7C0001092AA0F64E66093AB0F6093AC0F509356
:10F7D000AE0F4093AD0F3093B00F2093AF0F109248
:10F7E000B10F5093B30F4093B20F3093B50F2093E6
:10F7F000B40F1092B60F1092B70F8093B80F1092FB
:10F80000BA0F1092B90F8093BB0F8093BC0FE8EC36
:10F81000F0E0F093BE0FE093BD0FE0E2F3E0F09371
:10F82000C00FE093BF0F5093C20F4093C10F3093AE
:10F83000C40F2093C30F8093C50FE9E5F0E0F09368
:10F84000C70FE093C60FE0E8F0E0F093C90FE09334
:10F85000C80FEFEFF0E0F093CB0FE093CA0FF093F7
:10F86000CD0FE093CC0F8093CE0F9093CF0F1092DB
:10F87000D00F8093D10F9093D20F1092D30F10928C
:10F88000D40F8093D50F1092D60F1092D70F80937C
:10F89000D80F1092D90F98E29093DA0F5093DC0FA3
:10F8A0004093DB0F5093DE0F4093DD0F3093E00F5A
:10F8B0002093DF0F8093E10F92E39093E20FE2E059
:10F8C000E093E30F8093E40F6093E50FE6E4E093A9
:10F8D000E60F9093E70F1092E80F1092E90F109245
:10F8E000EA0F1092EB0F1092EC0F1092ED0FEAEF6F
:10F8F000F0E0F093EF0FE093EE0F1092F00F109204
:10F90000F10F6093F20F61E46093F30F1092F40F24
:10F910009093F50F1092F60F9093F70FEEE5F1E04C
:10F92000F093F90FE093F80F1092FA0FACEDB5E0F9
:10F93000B093FC0FA093FB0F00EA1FE01093FE0FA3
:10F940000093FD0F309300102093FF0FC8E8D3E120
:10F95000D0930210C093011068EBE62E6BE0F62EF8
:10F96000F0920410E0920310E0E4FFE1F09306103F
:10F97000E0930510109207101092081010920910D1
:10F9800069E160930A1080930B1080930C108093B0
:10F990000D1050930F1040930E10309311102093C0
:10F9A0001010F0921310E0921210109315100093A3
:10F9B0001410D0931710C093161020E737E130933E
:10F9C00019102093181010921A1010921B101092F8
:10F9D0001C1090931D1090931E1090931F10109266
:10F9E000201080932110109231101092221099E073
:10F9F000909323101092241010922510109226102C
:10FA000010922710B0932910A0932810F0932B1078
:10FA1000E0932A1080932C1070932D1010922E10CA
:10FA200021E030E03093301020932F1040E052EC72
:10FA300061E070E0409332105093331060933410C3
:10FA400070933510409336105093371060933810F0
:10FA50007093391040E056E960E070E040933A104E
:10FA600050933B1060933C1070933D1040933E10B8
:10FA700050933F10609340107093411010924210C9
:10FA800020E039E130934410209343101092451048
:10FA90009EE190934610109247102EE130E0309393
:10FAA00049102093481030934B1020934A10309304
:10FAB0004D1020934C1090934E1090934F108093C4
:10FAC00050108093511010925210909353108093C5
:10FAD00054108093551088E293E1A0E0B0E0809349
:10FAE000561090935710A0935810B09359100AE8ED
:10FAF0001EE0C0E0D0E0CE010E945BB5F80161914C
:10FB00008F01861719F0CE010E946DB52196C03D78
:10FB1000F1E0DF0781F7DF91CF911F910F91FF9007
:10FB2000EF9008954F925F926F927F928F929F9283
:10FB3000AF92BF92CF92DF92EF92FF92CF93DF937B
:10FB4000EB01A0914812B09149129D012F5F3F4FE8
:10FB500045E0429F2001439F500C1124052C000CCE
:10FB600066087708812C912C54012F33E1E03E0781
:10FB7000ECF443E854E861E0772775016401C40CB4
:10FB8000D51CE61CF71C4C0D5D1D6E1D7F1D6BBF4B
:10FB9000FA014791569165E0860E911CA11CB11C9B
:10FBA000C417D50729F12F5F3F4FDFCF25E0822E05
:10FBB000912CA12CB12C21E030E0A217B30708F45E
:10FBC0004CC043E854E861E07727480D591D6A1D91
:10FBD0007B1D6BBFFA0147915691F5E08F0E911C8A
:10FBE000A11CB11CC417D50719F02F5F3F4FE5CFFB
:10FBF00043E854E861E07727E5E0E29F6001E39F96
:10FC0000D00C11240D2C000CEE08FF084E5F5F4F46
:10FC10006F4F7F4F4C0D5D1D6E1D7F1D6BBFFA0139
:10FC200047915691FC015383428343E854E861E0D5
:10FC300077274C5F5F4F6F4F7F4FC40ED51EE61E78
:10FC4000F71EEBBEF601C790FC01C4823093491247
:10FC500020934812C901019606C0109249121092D1
:10FC6000481280E090E0DF91CF91FF90EF90DF901D
:10FC7000CF90BF90AF909F908F907F906F905F904C
:10FC80004F9008950F931F938091431281111EC0CE
:10FC90000E94D36D0091441210914512209146129A
:10FCA00030914712AB01BC01401B510B620B730B2F
:10FCB0008091411290914212A0E0B0E08417950724
:10FCC000A607B70718F481E0809343121F910F91A4
:10FCD00008958091411290914212892B89F0809170
:10FCE0004312882381F00E94D36D60934412709375
:10FCF0004512809346129093471210924312089532
:10FD000081E08093431208951F920F920FB60F92D5
:10FD100011242F938F939F9310929500109294002B
:10FD20008091CF0A8F5F8093CF0A9091C712891775
:10FD300084F01092CF0A2091D10A8091D212909132
:10FD4000D312820F911D27FD9A959093D312809321
:10FD5000D2128091CE0A8F5F8093CE0A9091D712F3
:10FD6000891784F01092CE0A2091D00A8091D51282
:10FD70009091D612820F911D27FD9A959093D612DD
:10FD80008093D5129F918F912F910F900FBE0F905E
:10FD90001F9018958091CD0A811104C08091CC0AE2
:10FDA000882321F080917100826003C080917100EE
:10FDB0008D7F8093710008951F93CF93DF931F92DF
:10FDC000CDB7DEB710E0181731F089830E94673A8B
:10FDD0001F5F8981F8CF0F90DF91CF911F91089518
:10FDE000CF93DF9360E088E00E94814C1092401234
:10FDF000C0913E12D0913F12BE0180EF9AE00FD128
:10FE0000882321F0BE0180EF9AE021D181E0809328
:10FE10003D1280919206882341F06BE477E1809156
:10FE20009006909191060E947A4ADF91CF912EC759
:10FE3000609143107091441080E090E00E9436B4CD
:10FE400020E030E04AE754E40E9491B0AB01BC01ED
:10FE500021E080919006909191060C948A49482F58
:10FE600050E095E1899FF0011124E558FE4E218173
:10FE7000328180859185280F391F83819481821773
:10FE8000930728F08581968128173907E8F485E1E2
:10FE9000849FF001859FF00D1124E558FE4E858169
:10FEA00096812817390728F52581368185E1849FB9
:10FEB000F001859FF00D1124E558FE4E82858230B9
:10FEC00019F411861086128685E1849FF001859FC2
:10FED000F00D1124E558FE4E328321838091840079
:10FEE00090918500280F391F309389002093880056
:10FEF00008958381948182179307C0F6238134810A
:10FF0000D5CF6CE20C947E614F925F926F927F929C
:10FF10008F929F92AF92BF92CF92DF92EF92FF9219
:10FF20000F931F93CF93DF936C01A4ECCA1AADEF2C
:10FF3000DA0AD601ED91FC917E970CF05DC0FC01D0
:10FF4000E858FF4F812C912CA191B191AB2B21F45A
:10FF50002115310549F450C0BFEF8B1A9B0AAEE161
:10FF60008A16910489F748C0EC015401AA0CBB1C05
:10FF7000AA0CBB1CAC0EBD1EF501EC54FF4F408318
:10FF80005183628373837401EE0CFF1CEC0EFD1E23
:10FF9000F701E858FF4F31832083EC54FF4F118362
:10FFA0000083BE01680D791DFB01EC55FE4F81E019
:10FFB00080830E94D36DF501608371838283938374
:10FFC000C65CDD4F88819981F701E250FE4F918335
:10FFD0008083D6012D913C9111972F5F3F4F2D9338
:10FFE0003C939C012F5F3F4F1216130614F021E043
:10FFF00030E03983288302C08FEF9FEFDF91CF91EC
:020000021000EC
:100000001F910F91FF90EF90DF90CF90BF90AF9036
:100010009F908F907F906F905F904F900895DC013C
:10002000A250BE4F20E030E04D915D91461757073A
:1000300039F4280F391FF901EC55FE4F80810895DE
:100040002F5F3F4F2E31310579F780E00895CF9330
:10005000DF93EC01C45CDD4FA881B981109709F4EE
:1000600042C0FC01E250FE4F20E030E0419151914E
:100070004617570799F5A901440F551F480F591FF7
:10008000FA01E858FF4F60817181672B61F111829D
:100090001082FC01E20FF31FEC55FE4F1082FA01B3
:1000A000EE53FE4F11821082235D3F4F220F331F0C
:1000B000220F331FFC01E20FF31F10821182128204
:1000C0001382FA01E859FE4F11821082EA56FF4F5F
:1000D000118210821197B983A88305C02F5F3F4F0B
:1000E0002E31310519F6DF91CF9108950F931F93AB
:1000F00001E010E009DF1F910F9108950F931F9306
:1001000000E010E001DF1F910F9108952F923F92C0
:100110004F925F926F927F928F929F92AF92BF9217
:10012000CF92DF92EF92FF920F931F93CF93DF93C3
:1001300000D000D0CDB7DEB78C010E94D36D9801FE
:100140002E533E4F3C832B831E830D83D801AC5529
:10015000BE4FBA83A9831801B2E02B1ABEEF3B0A47
:10016000F901AA24A394B12C32E0832E912C1182A0
:1001700010829F012A543140D9012D913C91232BAB
:1001800009F44DC0AD81BE812D913D914D915C91A1
:1001900013977D01B4EBEB0EF11CD701CD90DD90F0
:1001A000ED90FC902B013C01421A530A640A750A37
:1001B0004C145D046E047F0490F1C20ED31EE41E45
:1001C000F51EAD81BE81CD92DD92ED92FC9213972A
:1001D000A981BA812C91222311F19F01265931095D
:1001E000D9012D913C912115310519F4B182A082DC
:1001F00016C07F01BAE5EB1AF108D7014D915C9169
:100200001197421753075CF4B182A0824F5F5F4F92
:100210004D935C934217530714F09182808232967B
:100220002D813E812C5F3F4F3E832D83A981BA8172
:100230001196BA83A983E215F30509F098CFEB81F3
:10024000FC8181919191FC83EB838130910599F040
:100250000297C9F4EB81FC81EC54F1400190F081EC
:10026000E02D1995AB81BC81DA966D917C91DB977D
:10027000C801EDDE08C0EB81FC81EC54F140019037
:10028000F081E02D19952B813C8122153305B9F6BB
:1002900026960FB6F894DEBF0FBECDBFDF91CF918B
:1002A0001F910F91FF90EF90DF90CF90BF90AF9094
:1002B0009F908F907F906F905F904F903F902F9086
:1002C00008956E3E22E0720738F06B3C98E07907A3
:1002D00028F06AEC78E002C06EEE72E0660F771FDD
:1002E0009FB7F89425E1829FF0011124E558FE4E56
:1002F000748363839FBF08956E3E22E0720738F0D7
:100300006B3C98E0790728F06AEC78E002C06EEE6A
:1003100072E0660F771F9FB7F89425E1829FF00186
:100320001124E558FE4E768365839FBF0895660FBE
:10033000771F282F30E095E1899FF0011124E558BF
:10034000FE4E858196816817790718F4658176815C
:1003500007C0838194818617970710F463817481A5
:100360008FB7F89495E1929FF001939FF00D1124BF
:10037000E558FE4E728361838FBF0895982F8FB723
:10038000F89425E1929FF0011124E558FE4E21E0FA
:1003900027838FBF41B121E030E0B90102C0660F71
:1003A000771F9A95E2F7CB01842B81B908958A30A3
:1003B00058F49FB7F89425E1829FF0011124E55885
:1003C000FE4E118610869FBF08951F93CF93DF9333
:1003D00025E1829FC0011124EC01C558DE4E8A85BB
:1003E00081110FC01FB7F89481E08A8789899A89A3
:1003F0009A8389830E94D36D6B877C878D879E87C4
:100400001FBFDF91CF911F910895CF93DF938A3063
:10041000D0F56233710538F061369DE6790728F032
:1004200060E67DE602C062E370E0D42FC82F80E072
:1004300090E00E9436B420E030E04AE754E40E94A5
:1004400091B020E030E04CE852E40E9497B49B0168
:10045000AC0160E070E08AEF94E40E9491B00E94E9
:10046000F9B09B01DD2321F022273327261B370B10
:100470008FB7F89495E1C99FF0011124E558FE4E1D
:10048000318720878FBFDF91CF9108958A3008F49C
:1004900018CF08958A3008F42FCF08958A3058F481
:1004A00095E1899FF0011124E558FE4E81819281EA
:1004B00096958795089580E090E008958A3008F435
:1004C00036CF08951F920F920FB60F9211240BB6DC
:1004D0000F920F931F932F933F934F935F936F93BD
:1004E0007F938F939F93AF93BF93CF93EF93FF939C
:1004F0008091B412893048F01092B41280912A127F
:10050000882399F0809123120DC0E091B412E1503C
:1005100025E1E29FF0011124E558FE4E87818823F2
:1005200021F0808192B1892782B9E091B41285E1EE
:10053000E89FF0011124E558FE4E8781882321F0C1
:10054000808192B1892B82B9E091B412C5E1CE9F2E
:10055000F0011124E558FE4E80859185892B09F024
:100560004DC0E091B412CE9FF0011124E558FE4E2B
:100570008285813009F060C00E94D36DE091B41291
:10058000CE9FF0011124E558FE4E03851485258584
:100590003685E091B412CE9FF0011124E558FE4E4D
:1005A0000784F089E02DAB01BC01401B510B620BAD
:1005B000730BCF01A0E0B0E084179507A607B7073B
:1005C000D8F5E091B412A091B412CA9FD0011124C1
:1005D000A558BE4E53968D919C915497CE9FF00195
:1005E0001124E558FE4E91878087E091B412CE9F8A
:1005F000F0011124E558FE4E82E082878091B4120A
:100600002EDC8091B4128F5F8093B412FF91EF9132
:10061000CF91BF91AF919F918F917F916F915F919A
:100620004F913F912F911F910F910F900BBE0F9003
:100630000FBE0F901F901895E091B4128091840026
:100640009091850025E1E29FF0011124E558FE4ECE
:1006500021813281820F931F9093890080938800BB
:10066000D0CF1F93CF93DF938091B312811173C0CA
:100670001092B4129FB7F89485E128EB3BE04CED63
:1006800055E064E971E1A1E0B0E0E091B412E93035
:1006900008F052C0E091B4128E9FF0011124E55889
:1006A000FE4E32832183E091B4128E9FF00111241B
:1006B000E558FE4E56834583E091B4128E9FF001BB
:1006C0001124E558FE4E74836383E091B412F091D7
:1006D000B412ED0101C0CC0FFA95EAF78E9FF0013C
:1006E0001124E558FE4EC083E091B4128E9FF001B4
:1006F0001124E558FE4E1782E091B4128E9FF0014E
:100700001124E558FE4E11861086E091B4128E9F9A
:10071000F0011124E558FE4E1286E091B4128E9F2E
:10072000F0011124E558FE4E148A138AE091B412A8
:10073000EF5FE093B412A9CF9FBF8FB7F89420EA80
:100740003FE03093251220932412109223128FBF82
:1007500081E08093B312DF91CF911F9108950F93A1
:100760001F93CF93DF938C01C62FD42FDC011196FA
:100770008D919C911297DC01ED91FC910190F0819B
:10078000E02DD8016C911995F80181819281DC01ED
:10079000ED91FC910190F081E02D6C2F1995F801FD
:1007A00081819281DC01ED91FC910190F081E02D3D
:1007B0006D2F1995F80180816C2F70E0680F711D05
:1007C0006D0F711D6F77772781819281DF91CF91B6
:1007D0001F910F910C94A36A0F931F93CF93DF93F4
:1007E0008C01C62FD42FDC0111968D919C9112970C
:1007F000DC01ED91FC910190F081E02DD8016C912C
:100800001995F80181819281DC01ED91FC910190B3
:10081000F081E02D6C2F1995F80181819281DC0126
:10082000ED91FC910190F081E02D6D2F1995F8016B
:1008300080816C2F70E0680F711D6D0F711D6F77D7
:10084000772781819281DF91CF911F910F910C9435
:10085000A36A4F925F926F927F92AF92BF92CF92B4
:10086000DF92EF92FF921F93CF93DF93DD24D39417
:1008700045E0C42E52E0A52EB12CC3E0D0E0EE241A
:10088000E394F12C8091971290919812DC01ED91F4
:10089000FC910480F581E02D1995892B09F4BEC0E7
:1008A000109130018091971290919812DC01ED9196
:1008B000FC910680F781E02D199596B3B39A2091AB
:1008C0008400309185002059384E30938D0020935C
:1008D0008C00212F2C7139F01092B212D093961205
:1008E000C0939512CFCF93FB992790F9E091B21264
:1008F000E11116C0992331F28F3021F6D092B21255
:10090000809399128091951290919612892B09F0FB
:10091000B9CFF0929612E092951210929412B2CF43
:100920009111DACF91E09E0F9093B212F0E0E7566A
:10093000FD4E8083993109F0A5CF81116CC0809163
:10094000B01282FF05C0D0939612C093951263C077
:1009500083FDF9CF8091951290919612019739F409
:10096000809194128F5F80939412843020F0B09223
:100970009612A0929512809193128F5F809393129A
:1009800090919212981708F044C0D0929112A1E76A
:10099000B2E1EAE9F2E140E050E0BA0110E0CF0153
:1009A000FC011B3098F401964080512C612C712C75
:1009B000012E04C0440C551C661C771C0A94D2F707
:1009C0004429552966297729185FEACF9A0137709B
:1009D000205E3340C29EC001C39E900D112497FD3E
:1009E000079623E0959587952A95E1F784529A4FCB
:1009F0008D939D931B503BE0769567955795479552
:100A00003A95D1F782E1A139B80749F610929312CD
:100A100002C0109291121092B21234CFDF91CF9196
:100A20001F91FF90EF90DF90CF90BF90AF907F909D
:100A30006F905F904F9008958091DB0A833031F47E
:100A400080916F12909170120C94337A0895809176
:100A5000DB0A823029F480916D1290916E12F9CEEA
:100A60000895F5DFE9CF1092541110925E111092A3
:100A70006811109272111092501180E090E0FC0108
:100A8000E650FF4E1182079684359105C1F708950F
:100A90008091DB0A823039F0833049F0813049F4AB
:100AA00080916A1201C080E18093D70A04C08EE071
:100AB000FBCF1092D70A8091D70A089560E089E3AE
:100AC0000E94814C60E08AE30E94814C60E085E3F3
:100AD0000E94814C60E085E00E94814C60E084E0EF
:100AE0000E94814C60E087E00E94814C72980895DA
:100AF000CF93C09112026C2F89E30E94814C81E058
:100B0000C8276C2F8AE30E94814CC0931202CF91B8
:100B10000895CF93DF93C09111026C2F89E30E9457
:100B2000814CD1E0DC276D2F8AE30E94814C6C2F31
:100B300085E30E94814C6D2F85E00E94814C6D2FD2
:100B400084E00E94814C6C2F87E00E94814CCC2372
:100B500011F0729801C0729A9091110281E0892778
:100B600080931102DF91CF910895CF93DF9380910D
:100B7000C61281110DC01092C5121092C41281E0EC
:100B800090E09093C3128093C2128093C61236C035
:100B90008091C4129091C512863191057CF18F38F5
:100BA000910534F48091C2129091C312019609C04C
:100BB0008D3521E0920754F48091C2129091C312B6
:100BC00002969093C3128093C21218C0863222E01C
:100BD000920734F48091C2129091C3120496F1CF1F
:100BE000883E93403CF48091C2129091C3128A5B7C
:100BF0009F4FE7CF1092C3121092C2128ADFC091AA
:100C0000C412D091C512C93E83E0D80754F01092A7
:100C1000C61254DF2CE236E848EE53E060E070E0A4
:100C200007C025EB35E8AE010D2E000C660B770BE7
:100C300080EF9AE05BDA9093C1128093C0128091AA
:100C4000C2129091C3128C0F9D1F9093C512809376
:100C5000C412DF91CF910895CF93DF9380919506D1
:100C6000882319F0DF91CF9180CFC091C012D0912D
:100C7000C112BE0180EF9AE0D2D9882321F0BE01D3
:100C800080EF9AE0E4D9DF91CF9118CFCF93C09154
:100C9000BD126C2F70E088E00E94EC4C89E18093DB
:100CA000BC1290911002992311F0CD5F01C0C35086
:100CB000C093BD128091BD12873970F0992321F045
:100CC0008FEF8093BD1208C08D3D30F086E9809390
:100CD000BD1288E78093BC128091BD128F3F19F43A
:100CE0001092100205C08A3118F481E0809310023E
:100CF0004091BC1250E060E070E026E436E880EFFE
:100D00009AE0F4D990933F1280933E12CF910895C8
:100D1000CF92DF92EF92FF92CF93DF93EC019C0191
:100D2000AFEFB0E00E94C9B5CC24CA9423E0D22E24
:100D3000E12CF12CA70196010E947BB5B90188E056
:100D40000E94EC4C9E01A4E6B0E00E94C9B5A70148
:100D500096010E947BB580914E10821320934E1015
:100D6000DF91CF91FF90EF90DF90CF900895CF93D8
:100D7000DF93C0913E12D0913F12BE0180EF9AE006
:100D80004ED9882321F0BE0180EF9AE060D960E05F
:100D900088E00E94814C809192068823D1F0809156
:100DA0004012882319F066EA78E10DC080913D1267
:100DB000882319F06DE878E106C08091091381114C
:100DC00008C06EE778E180919006909191060E94AC
:100DD0007A4A1092401210923D12DF91CF910895FD
:100DE00061E088E00E94814C80919206882361F046
:100DF00080914012811108C060E778E180919006EF
:100E0000909191060C947A4A089580914012811134
:100E100010C0ADDF81E0809340128091920688235C
:100E200041F065ED78E180919006909191060E94E5
:100E30007A4A8091BB12882329F060E088E00E9402
:100E4000814C01C0CDDF9091BB1281E08927809356
:100E5000BB12882329F040914A1050914B1004C0D6
:100E600040914C1050914D1060E070E025E037E863
:100E700080EF9AE03BD990933F1280933E12089501
:100E8000CF938091B91281110FC081E08093B91284
:100E900080919206882341F06EE378E1809190067C
:100EA000909191060E947A4AC091B8126C2F85E009
:100EB0000E94814C4091531050E060E070E020E4CB
:100EC00037E880EF9AE012D99093B7128093B61268
:100ED00081E06C2F68276093B812CF910895CF936B
:100EE000DF93C091BE12D091BF12BE0180EF9AE095
:100EF00096D8882359F0BE0180EF9AE0A8D81092C6
:100F0000BF121092BE12DF91CF91D8CDDF91CF9159
:100F100008956091BE127091BF1280EF9AE07FD861
:100F200081112DC060E089E30E94814C60E08AE37A
:100F30000E94814C60E085E30E94814C60E085E086
:100F40000E94814C60E084E00E94814C60E087E078
:100F50000E94814C729880915010882319F029E8E2
:100F600035E802C028E735E842E350E060E070E091
:100F700080EF9AE0C3D89093BF128093BE12089579
:100F800060E08AE30C94814C61E08AE30C94814C2C
:100F90000F931F93CF93DF938C01C1E0D0E00C1728
:100FA0001D079CF0F1DF64E670E080E090E00E94B5
:100FB000D24DE6DFC017D10734F46AE570E080E077
:100FC00090E00E94D24D2196EACFDF91CF911F9100
:100FD0000F91089583E090E0DBCF82E090E0D8CFDE
:100FE00081E090E0D5CF60E089E30C94814C61E032
:100FF00089E30C94814C0F931F93CF93DF938C0163
:10100000C1E0D0E00C171D079CF0F1DF64E670E052
:1010100080E090E00E94D24DE6DFC017D10734F4A3
:101020006AE570E080E090E00E94D24D2196EACF20
:10103000DF91CF911F910F91089583E090E0DBCF76
:1010400082E090E0D8CF81E090E0D5CF60914E1063
:1010500070E088E00E94EC4C80919206882341F079
:101060006FEB78E180919006909191060C947A4A0A
:1010700008951092BA1280917E06811104C060E03A
:1010800084E00E94814C80919206882341F06DE5B6
:1010900078E180919006909191060C947A4A089597
:1010A00081E08093BA1280917E06811106C0609122
:1010B000B51270E084E00E94EC4C80919206882387
:1010C00041F06BE478E180919006909191060C9448
:1010D0007A4A089510927E068091BA12811104C056
:1010E00060E084E00C94814C6091B51270E084E083
:1010F0000C94EC4CCF93DF9360E085E00E94814C30
:101100008091B91281110BC080918C0690918D064F
:10111000DC01ED91FC9102ACF3ADE02D1995C0918D
:10112000B612D091B712BE0180EF9AE00E940F80F4
:10113000882329F0BE0180EF9AE00E9427808091E9
:101140009206882379F02091B912809190069091AF
:101150009106222319F062E378E102C066E278E1A9
:101160000E947A4A1092B912DF91CF91089561E0FE
:1011700085E00E94814C80918C0690918D06DC0167
:10118000ED91FC9102ACF3ADE02D199580919206A2
:10119000882341F06BE178E180919006909191066F
:1011A0000C947A4A089560E085E30E94814C809116
:1011B0008C0690918D06DC01ED91FC9106A8F7A9B3
:1011C000E02D199580919206882341F06FE078E137
:1011D00080919006909191060C947A4A0895411559
:1011E000510529F06115710511F00C946E7908957F
:1011F000EF92FF920F931F93CF93DF931F921F9253
:10120000CDB7DEB78C018CE789831A82F801E480C0
:10121000F580FFEFEF1AFF0AB701C8010E94F947F6
:10122000882381F0F8012081318184819581BE017C
:101230006F5F7F4F820F931F0E945BB3F801F582AF
:10124000E48281E00F900F90DF91CF911F910F9179
:10125000FF90EF900895AF92BF92CF92DF92EF92FE
:10126000FF920F931F93CF93DF9300D01F92CDB7C0
:10127000DEB78C0149835A836B837C83CE01019650
:101280006C01580194E0A90EB11CE12CF12CC801AD
:101290000E945BB5F60161916F01861731F0C801BC
:1012A0000E946DB5FFEFEF1AFF0A0F5F1F4F0A157F
:1012B0001B0569F781E0EF2809F480E00F900F909B
:1012C0000F900F90DF91CF911F910F91FF90EF90B2
:1012D000DF90CF90BF90AF900895CF92DF92EF92C2
:1012E000FF920F931F93CF93DF93EC010091D812DD
:1012F000E0E0F0E020E030E0A90110E0CE17DF07E9
:101300001CF1309711F40D32E1F0DF01A852BD4E0F
:10131000FC9080ED8F0D8A30A8F4AAE0B0E00E9426
:1013200097B52F2DFF0C330B205331096901330F73
:10133000EE08FF089B01AC012C0D3D1D4E1D5F1DED
:1013400001C011E03196DACFCA01B901112339F099
:1013500090958095709561957F4F8F4F9F4FDF914E
:10136000CF911F910F91FF90EF90DF90CF90089554
:101370008091DF0A811105C081E09091E10A91110D
:1013800001C080E00895CF93DF9320910A0A309145
:101390000B0AE9012697A881B981A65FB54F12967D
:1013A0001C92082E000C990BAA0BBB0BFC01319769
:1013B000EE30F10508F057C18827E458FE4F8F4FF3
:1013C0000C9418B0F9013A9780819181865F954F0E
:1013D0000E94F6AD882309F44BC1E0910A0AF0910E
:1013E0000B0A36970190F081E02DE65FF54F81E022
:1013F000A0C0F9013C9780819181865F954F0E9442
:1014000033AD882309F434C1E0910A0AF0910B0A44
:1014100036970190F081E02DE65FF54F82E089C0BC
:10142000F9013E9780819181865F954F0E9476AC4D
:10143000882309F41DC1E0910A0AF0910B0A36973E
:101440000190F081E02DE65FF54F83E072C0F90175
:10145000709780819181865F954F0E94F9AB8823B8
:1014600009F406C1E0910A0AF0910B0A369701903F
:10147000F081E02DE65FF54F84E05BC0F9017297E3
:1014800080819181865F954F0E94B4AB882309F4D7
:10149000EFC0E0910A0AF0910B0A36970190F081B3
:1014A000E02DE65FF54F85E044C0F9017497808137
:1014B0009181865F954F0E943BAB882309F4D8C089
:1014C000E0910A0AF0910B0A36970190F081E02D25
:1014D000E65FF54F86E02DC0F90176978081918116
:1014E000865F954F0E94B5AA882309F4C1C0E09198
:1014F0000A0AF0910B0A36970190F081E02DE65F21
:10150000F54F87E016C0F901789780819181865F59
:10151000954F0E94A7AA882309F4AAC0E0910A0A5D
:10152000F0910B0A36970190F081E02DE65FF54FC0
:1015300088E082839DC0F901B09780819181865FA8
:10154000954F0E94C9A7882309F492C0E0910A0A26
:10155000F0910B0A36970190F081E02DE65FF54F90
:1015600083819481A581B6814097A105B10509F0D9
:101570007FC08EC0F9017A9780819181865F954FF7
:101580000E94DCA9882309F473C0E0910A0AF09153
:101590000B0A36970190F081E02DE65FF54F8AE067
:1015A000C8CFF9017C9780819181865F954F0E9419
:1015B00011A9882309F45CC0E0910A0AF0910B0A92
:1015C00036970190F081E02DE65FF54F8BE0B1CFCB
:1015D000F901B09780819181865F954F0E94C9A7DC
:1015E000882309F445C0E0910A0AF0910B0A369766
:1015F0000190F081E02DE65FF54F83819481A58114
:10160000B68180319440A105B10591F543C0F9013F
:101610007E9780819181865F954F0E9442A88823A2
:1016200039F1E0910A0AF0910B0A36970190F081A6
:10163000E02DE65FF54F8DE07CCFF901B09780811A
:101640009181865F954F0E94C9A7882389F0E09118
:101650000A0AF0910B0A36970190F081E02DE65FBF
:10166000F54F8EE066CFE881F981E65FF54F128293
:10167000E0910A0AF0910B0A36970190F081E02D73
:10168000E65FF54F81E09281911106C080E004C0D1
:1016900089E04FCF8CE04DCFDF91CF910895EF924D
:1016A000FF920F931F93CF93DF931F921F92CDB79B
:1016B000DEB741110AC07C0197FF03C0F194E194A9
:1016C000F108E616F70664F402C0E12CF12C81E083
:1016D0008093CC0A8FEF633371059CF425E012C030
:1016E0006E157F0534F01092CC0A81E091E021E084
:1016F0000AC06D337105BCF381E08093CC0A23E00E
:1017000001C024E092E03091CC0A332379F03FB756
:10171000F894899F902D11249093D00A2093D7128A
:101720000091D5121091D6123FBF0AC09FB7F8940E
:101730001092D00AF092D612E092D5129FBF870184
:101740004A8389830E94CA7E4A818981442319F091
:1017500017FF19C014C0813031F417FD10C0E01616
:10176000F1068CF40FC08F3F71F40E151F0554F075
:101770000F3F110541F03CF00FEF10E004C000E016
:1017800010E001C08701C8010F900F90DF91CF9149
:101790001F910F91FF90EF900895CF92DF92EF92FB
:1017A000FF920F931F93CF93DF93042FE22E4330CA
:1017B00049F0453039F0443041F4F92EFF1CFF2444
:1017C000FF1C04C0FF24F39401C0F12CFC0197FF1F
:1017D00003C0F195E195F109EF011092CD0A0130B6
:1017E00009F432C1053009F06EC08091E712811111
:1017F00018C0C091D412D0E0D093E612C093E51285
:1018000081E08093CD0A21E030E03093E412209310
:10181000E3123093D3122093D2128093E71211E097
:10182000B9C08091D2129091D31281159640E8F5FB
:1018300081E08093CD0A8091D2129091D3122091B1
:10184000E3123091E412821B930BC091E512D09108
:10185000E612089720F1BE0180E090E00E9436B4C5
:101860002091CE123091CF124091D0125091D112CE
:101870000E9497B420E030E040E05FE30E942DB08A
:101880000E94F9B0EB017093E6126093E51280912B
:10189000D2129091D3129093E4128093E312CF313D
:1018A000D1050CF075C0E1E001C0E0E01092CD0A76
:1018B0001092E6121092E5121092E7128E2F11E0AC
:1018C000C0E0D0E061C0EE20E1F0023029F4809168
:1018D000C80A9091C90A04C08091CA0A9091CB0AA3
:1018E000E817F9070CF0B3C081E08093CD0A80912E
:1018F000CD1294E0F595E7959A95E1F7EE5F1FEF2D
:1019000043C0DB0177FF03C0B195A195B109AE17C4
:10191000BF07C4F48091CC12882309F49CC081E0F5
:101920008093CD0A8091CB129091CA129130A1F58B
:10193000EA1BFB0BFD970CF0845011E054976CF5FB
:10194000E4E02CC0EA17FB070CF085C08091C912B7
:10195000882309F480C0043009F47DC081E08093BD
:10196000CD0A8091CD129091C812913009F07CC0BF
:10197000E233F10514F48E5F77C0AE1BBF0BD39733
:101980000CF472C0825070C01E1644F0E1E006C034
:1019900011E081E0E1E006C011E0E2E0181614F089
:1019A0006E0160C06E019091CD0A9923D9F02FB7D6
:1019B000F8941E9F902D11249093D10A8093C71202
:1019C0001C161D063CF48091D2129091D312892BE3
:1019D00009F44CC0053021F0C091D212D091D3123D
:1019E0002FBF09C08FB7F8941092D10AD093D312A9
:1019F000C093D2128FBF0E94CA7EEE2019F0D7FF8B
:101A00001DC018C0113031F4D7FD14C0CC16DD064E
:101A1000ACF413C01F3F91F4023011F0033071F4A5
:101A2000CC15DD0554F0CF3FD10541F03CF0CFEFB0
:101A3000D0E004C0C0E0D0E001C0E601FF2001F129
:101A4000D195C195D1091CC090E080E006C090E01E
:101A500080E01FEF03C09E2F8F2F11E06F01C92F71
:101A6000D82FE1E081E09FCF1FEF97CF8091D10A7F
:101A7000082E000C990B9093D3128093D212AACF08
:101A8000CE01DF91CF911F910F91FF90EF90DF90EA
:101A9000CF900895CF92DF92EF92FF9297FF26C0EA
:101AA000CC24DD24C61AD70A0D2C000CEE08FF0842
:101AB000092E000CAA0BBB0B9C01AD0121503F4F1E
:101AC0004F4F5F4FC701B601609570958095909517
:101AD0000E94E2AF2EEF30E040E050E00E947BB584
:101AE000C20ED31EE41EF51EC60126C0009711F1DA
:101AF000092E000CAA0BBB0B9C01AD012150310932
:101B000041095109CB01770FAA0BBB0BBC01CD01D9
:101B100061507109810991090E94E2AF2EEF30E016
:101B200040E050E00E947BB5DA01C9010196A11D99
:101B3000B11D02C080E090E0FF90EF90DF90CF9069
:101B4000089580910702813019F485E0809307029F
:101B500008951092870608958091C00A8823C1F0E5
:101B60006091B60D7091B70D80EF9AE00E942780CA
:101B70001092B70D1092B60D1092C00A8091070214
:101B80008130D9F48091F10F8823B9F0DADF15C0E4
:101B90008091E8128F5F8093E812803580F0609129
:101BA000B60D7091B70D80EF9AE00E9427801092D9
:101BB000B70D1092B60D1092C00A1092E812089557
:101BC000CF93823069F49091D80F2091D50F309146
:101BD000D90F4091D60F5091D70F6091D40F0CC000
:101BE0009091D20F2091CF0F3091D30F4091D00F11
:101BF0005091D10F6091CE0F6093CC125093C912C7
:101C00004093CA123093C8122093CB129093CD12F6
